:020000040800F2
:10000000002000105D070308014902088D55010812
:10001000FD480208F9480208F548020800000000FF
:10002000000000000000000000000000F14802088D
:10003000ED48020800000000E9480208A92F010865
:10004000C5070308C5070308C5070308C507030854
:10005000C5070308C5070308ED5E0108196001081C
:10006000DD5F0108A15F0108655F01089153000889
:100070008153000871530008615300085153000870
:100080003D53000829530008C5070308C5070308A6
:100090008D4C0208C5070308C5070308295F01083E
:1000A000351A0108951A0108C5070308A51A0108A1
:1000B000851A0108751A0108651A0108C5070308A1
:1000C000C5070308C5070308C5070308C5070308D4
:1000D000C50703081552000809520008FD51000821
:1000E000B15E0108C5070308D9480208C50703081F
:1000F000451A0108C5070308551A0108C507030872
:10010000000000000000000000000000C507030818
:10011000C5070308C5070308C5070308C507030883
:100120001553000801530008ED520008D952000889
:10013000C5520008C50703080000000000000000C9
:10014000C5070308C5070308C5070308000000002A
:10015000000000000000000000000000000000009F
:100160000000000000000000C5070308C5070308E1
:10017000C5070308000000000000000000000000A8
:0801800000000000C5070308A0
:100190002DE9F04FB54CB64B2768A3FB07239B080E
:1001A00003EB8303791CFF1A8DB0216040F00E81B0
:1001B000B04D23792A7802F004029342064600F0FB
:1001C0003C81002A40F0148167693B6838469B688F
:1001D0009847FF236069FB710268A74BD2F814802F
:1001E00001210222B9711146C047A44B1B789A071E
:1001F00000F1498207230293062303934FF0050879
:100200004FF004094FF0030A04AF60699C4B026889
:100210000221D2F814B05246D847B4F90A309948AE
:10022000994980FB0320DA17C2EBA00202EB82009F
:10023000A3EB40031BB212B2384616F0F7FD60691B
:10024000036852461621D3F814A03B46D047606994
:100250008E4B02680221D2F814A04A46D047394694
:10026000B4F90E002AF09EFD38462FF0A5FB884A0F
:10027000636912883A5219684A461846D1F81490B0
:100280003B461621C847834B1B681B0500F1BE8106
:100290006069814B02680221D2F814904246C84737
:1002A0007E4BB4F9100093F86A34002B40F0918132
:1002B00000EB800300EBC300794AC00082FB0031F1
:1002C000C317D3EB611100F1058282FB012ECA171F
:1002D000C2EB6E124FF06409DFF8A8E1DFF8D4C179
:1002E00009FB12128EFB02E18CFB00E0D217C2EB7D
:1002F000A10EC3EB203120220F20CDF800E00B46E9
:1003000001906849384616F091FD606901683B46E6
:1003100042464F691621B8474FF43471B4F90800CA
:10032000B4F90A20B4F90C90B4F90EC0B4F910E095
:10033000E1802B7803F00403237100285A4FDFF883
:100340007881DFF85CA1BCBF002020813888904212
:10035000D8F80020B8BF60818AFB02BAD217C2EB7E
:100360006A1212B24A45C8BFA281227EDFF84C91C0
:100370006245B8BFE281D9F818207245C8BF228211
:100380008BB1DFF83CE194F819C0AEFB06AECEF3BA
:10039000874EF44507D0B4F81AC084F819E00CF180
:1003A000010EA4F81AE0002900F08C803F4AB2F94F
:1003B000060040F2D66398424BDCB2F902209A4222
:1003C00047DC013989B2E18021B944E06069036802
:1003D000DB689847636943B193F90830002B04DD6B
:1003E000244D2B7823F001032B700DB0BDE8F08F66
:1003F000D4F81480D8F8003040469B689847FF2313
:10040000606988F807300268294BD2F814900122FD
:1004100088F806200C210722C84706214FF4FA72FB
:100420004FF0630CBE46A78127812782B946384624
:10043000E1806281A4F80EC07BE7E188B4F908008E
:10044000B4F90A20B4F90C90B4F90EC0B4F910E074
:1004500073E70023E38065692B6828469B6898470B
:100460000122FF23AA71EB71B4E700BFA020002096
:10047000CDCCCCCC1B8E0020287503084A8E0020E2
:100480004C7503086766666660750308687503083F
:10049000487F0308B47E0020AC75030894610020F7
:1004A0001F85EB51C0750308344500207488002077
:1004B00020750308AD8BDB68582400203024002011
:1004C00083DE1B439149DFF87CA2D4F814B0B6094F
:1004D000A1FB0616C6F380168AF80060BBF1000F78
:1004E00004D09BF9081000293FF77BAF884D95F8A1
:1004F0006A1449B94FF4A471864E01FB02F286FBDF
:100500000261D217C2EB61128349DFF808C2B1F869
:1005100000E064218CFB026C01FB0EF17F4E95F82C
:1005200062E4C1F387218E452176B6F800E0E169E7
:100530008CBF41F0010121F0010170457848B5F808
:1005400066E40078B4BF41F4001121F400114FEAD1
:10055000E272B4BF41F0020121F00201C2EB6C1261
:100560008007DFF8E4C1608BACFB006054BF41F44E
:10057000804121F48041BEEB501F40F2A58021F064
:1005800040036849B5F8640409688842B5F86814FE
:10059000D4BF43F4805323F480538A42DBF8002015
:1005A000ACBF43F4004323F40043E361584693682F
:1005B00098475D4B1B680121FF228BF80610190339
:1005C0008BF8072040F1C480606903681B6A984774
:1005D00000E7504B554983FB0023C217C2EB63135E
:1005E000642202FB130281FB021ED117C1EBAE0194
:1005F00081EAE17E0028AEEBE17E83EAE371ACBFE5
:1006000020222D220C20A1EBE37176E66069484B95
:1006100002680221D2F814904246C8473946B4F91C
:100620000C002AF0BFFB38462FF0C6F9414A636937
:1006300012883A52196842461846D1F814803B464F
:100640001621C0476069DDF80C9002683A4BD2F879
:10065000148002214A46C047324B394618682AF0B6
:10066000A1FB38462FF0A8F9344A636912883A5240
:1006700019681846D1F814804A463B461621C047EF
:10068000DDF8088004E660692D4B02680221D2F88B
:10069000148004AF0322C0473946B4F908002AF099
:1006A00081FB606903680322D3F8148016213B465E
:1006B000C04708230293072303934FF006084FF027
:1006C00005094FF0040AA0E5002B3FF458AF41F0B4
:1006D000400356E782FB012ECA17C2EB6E12DFF809
:1006E0006CC04FF0640E0EFB121210498CFB00E040
:1006F00081FB02E1C3EB2033D217A2EBA10E83EA08
:10070000E371A1EBE3710F202D22F6E5632D3E0589
:10071000946100201F85EB51A4450020E047002094
:100720004A8E002030450020148E002067666666E1
:100730007C7503089075030894750308A875030871
:10074000387503080000002089888888AD8BDB6835
:10075000B54B1B689A0705D463692BB393F908302E
:10076000002B21DD032018F0A7FFB5F83A341B0554
:100770001AD5E3695E0702D59AF80030A3B960691B
:1007800003681B6998470CABA84A43F8202D6169A0
:10079000B0F5F07F086808BF0722D0F814B018BF82
:1007A000062208460D21D847B5F838B41BF4006F6F
:1007B00024D0E369980702D59AF80030F3B93B8852
:1007C0009B4A9C49A2FB0302D20802EB8200A3EBE6
:1007D00040030CA806469BB24FF0910E0DF111009C
:1007E00006F820ED16F022FB606902685269334674
:1007F0000BF01F011646CBF34412B047B5F836B4E0
:100800001BF4006F21D0E369D90702D59AF80030B4
:10081000DBB9894B89491B88642202FB03F29212DF
:100820000CAE632A4FF00103A8BF63220DF1110043
:1008300006F8203D16F0FAFA6069026833460BF0BC
:100840001F015669CBF34412B047B5F84264320534
:1008500024D5E3695B0602D59AF80030F3B9638BBF
:10086000774A7849A2FB03025209C2EB02100DF14C
:10087000300BA3EB80039BB24FF09C0E0DF11100E7
:100880000BF820ED16F0D2FA606902685B4606F0BC
:100890001F01D2F814B0C6F34412D847B5F840B4DB
:1008A0001BF4006F2CD0E369980602D59AF800304B
:1008B00033BB12F02DFB644B614ADFF8B0E16149B4
:1008C000A3FB00639B0CA2FB0362060A5009C0EB6A
:1008D0000010AEFB06620CAEA3EB8003920A4FF051
:1008E0009B0E0DF1110006F820ED16F09FFA6069DD
:1008F000026833460BF01F015669CBF34412B04730
:10090000B5F8443419051FD5E269120602D59AF8E4
:100910000020CAB94D4A106803F01F01C3F3441206
:10092000C30040F1E6814A4B4A480088460500F181
:10093000C181C60700F1E681474E10F0020F18BFD3
:100940003346606915F09EFBB5F84864300530D534
:10095000E369990502D59AF8003053BB3F4B404AF2
:10096000B3F906303549B3F5FA6FA8BF4FF4FA630F
:10097000B3F57A7FB8BF4FF47A73A3F57A7382FB2D
:100980000302DB17C3EBA2024FF0040E05230DF1A7
:1009900012008DF811308DF810E016F047FA6069FA
:1009A0000368C6F34412D3F814B006F01F0104AB79
:1009B000D847B5F84C6432052AD5E3691B0502D542
:1009C0009AF8003023BBD8F800302648264983EA3D
:1009D000E37EAEEBE37E80FB0E304FEAEE72C2EBBD
:1009E00060120DF1300B642000FB12E34FF09A0E01
:1009F0000DF111000BF820ED16F018FA606902688D
:100A00005B4606F01F01D2F814B0C6F34412D84773
:100A1000B5F84E64300541D5E369D90428D59AF874
:100A20000030002B3AD123E0248A0020267E2700C4
:100A3000CDCCCCCC60750308A445002098A7030852
:100A400089888888CC75030883DE1B43148E0020B8
:100A50000C750308C06000201C7503087488002012
:100A6000676666661F85EB51D8750308C7541E017B
:100A7000B44BB5491A680DF1300B07230DF1110085
:100A80000BF8203D16F0D2F9606902685B4606F06B
:100A90001F01D2F814B0C6F34412D847082018F04A
:100AA0000BFEB5F85464320545D5E3691B0403D544
:100AB0009AF80030002B3ED195F86A34D9F8182006
:100AC00006F01F09C6F34416002B40F0F5804FF4E2
:100AD000A4719E4B01FB02F183FB0120CA17D2EBEC
:100AE000601000F1118183FB00E34FEAE07ECEEB62
:100AF00063134FF0640BDFF884E2DFF894C20BFB62
:100B000013038EFB030ED8178CFB0113C0EBAE0E44
:100B10000F21C2EB2330202203460191CDF800E0E3
:100B20008B4904A816F082F960693246066804AB66
:100B300049467669B047B5F85664300519D5E3697A
:100B4000D90302D59AF800309BB9824B82491868C4
:100B5000837A0278007D009004A816F067F9606936
:100B6000026804ABD2F8149006F01F01C6F34412D9
:100B7000C847B5F85864320519D5E3699B0302D517
:100B80009AF800309BB9734B74491868C37A42785D
:100B9000407D009004A816F049F96069026804AB32
:100BA000D2F8149006F01F01C6F34412C847B5F8F6
:100BB0005A64300519D5E369590302D59AF8003013
:100BC0009BB9644B66491868037B8278807D0090EE
:100BD00004A816F02BF96069026804ABD2F81490EF
:100BE00006F01F01C6F34412C847B5F85C6432052D
:100BF0001ED5E3691B0302D59AF80030C3B93888C3
:100C0000D8F80030574A584903FB00F382FB03022F
:100C1000DB17C3EBA21204A816F008F9606902689A
:100C200004ABD2F8148006F01F01C6F34412C0478B
:100C3000B5F85E6430051CD5E369D90202D59AF88F
:100C40000030B3B995F8D0254849742303FB02530B
:100C500004A893F8C0340132013316F0E7F8606954
:100C6000026804ABD2F8148006F01F01C6F34412E8
:100C7000C047B5F860542A057FF5A6ACE3699B022E
:100C800004D59AF80030002B7FF49EAC384B1A88BC
:100C90003B889A427FF798AC04A8364916F0C6F80C
:100CA0006069026804AB566905F01F01C5F3441280
:100CB000B04789E4304B44E6244B304883FB0213B1
:100CC000D117C1EB6313642101FB132180FB010EDB
:100CD000C817C0EBAE0080EAE07E002AAEEBE07EF3
:100CE00083EAE370ACBF20222D220C21A0EBE3703D
:100CF00012E7234B23481E68234B16F4800F08BFCE
:100D0000034611E6214B1CE683FB003C4FEAE07EE4
:100D1000CEEB6C1E1E4B4FF0640C0CFB1E00DFF87C
:100D20005CE083FB0113C2EB23328EFB00E1C017B2
:100D3000A0EBA10E82EAE270A0EBE2700F212D225F
:100D4000EAE600BF3045002098A703081F85EB5155
:100D5000C07503088C410020E0750308F075030896
:100D600000760308D34D621010760308147603084A
:100D7000E04700201C760308107503086766666666
:100D8000B47E0020047503080C750308147503086D
:100D9000AD8BDB6810B40268047B11680223A340AA
:100DA000194209D00649406800240C7001684FF6CA
:100DB000FE742140016053605DF8044B704700BF32
:100DC00034680020FF207047012380F845307047C9
:100DD000014B1868704700BF145200200120704773
:100DE000704700BF704700BF2DE9F04FDFF81CB21D
:100DF000DFF81CE2BBF80020DEF80060BBF904302D
:100E0000BBF90250BBF90A80C2EB261404FB04F4C0
:100E100024135200C2EBE60203FB04F305FB02F2CB
:100E20009B1303EBE223B3F5FA364FEAE37589B07F
:100E300045F1FF373246A6FB0645CDE9024502FBE8
:100E400007F205EB4202CDE90467029EBBF90840B8
:100E5000039208FB02FC4FEAE87906FB09CC3A460C
:100E6000A8FB0689049ECBF81830E51704FB02F2B4
:100E700006FB0522A4FB0667E14417444FEA18224B
:100E800042EA096200924FEA292201923D03DDE91C
:100E90000078340345EA16553F19BBF80660069002
:100EA00048EB05083C1C48F5004503EB8302A4FB16
:100EB000068906FB0599803213124FEA69064FEA4C
:100EC000E977079356EA07038A4600F09280DDE946
:100ED0000489BBF90E20DEF80440BBF91000494636
:100EE000C4F5801ED317DDE9024502FB01F108FBC2
:100EF0000311A2FB08230B444FEA43492B46C117B9
:100F000000FB03F304FB0133A0FB0401BBF90C401D
:100F10001944E30001937346DC170023009349EA68
:100F2000D2394FEA4248DDE9002310EB080041EBDB
:100F30000901E50712184FEACE744B4145EA5E05F8
:100F4000A41A65EB0305221945EB050312196B4141
:100F500099019001801841EA926159418B00820009
:100F600043EA9073101943EB05018B00820043EABA
:100F7000907310460019194632463B4669412FF0DE
:100F800019FABBF916204C13450B45EAC14502FB83
:100F900004F6D31705FB0366A2FB05233344BBF914
:100FA000146002FB04F405FB034406FB01FEA2FBF4
:100FB0000523F717234400FB07EE540EA6FB00673A
:100FC000774444EAC3144FEAD64800194FEA6365F0
:100FD00048EA473869414FEAE74918EB0008BBF98E
:100FE000124049EB01094FEA182646EA096620013A
:100FF0003618069B0BB1360A1E60BAF1000F02D0FC
:10100000079BCAF8003009B0BDE8F08FCC30002053
:10101000C0200020704700BF704700BF4FF400633E
:101020000381704750F8043C01224274143803B124
:101030001847704790F82530024603F0FF0013B1BF
:10104000002382F82530704770B582B00446036BE8
:1010500090F844006A4606219847C0B19DF8040004
:101060009DF800609DF801109DF802509DF8032046
:101070009DF8053041EA062143EA002342EA0522B1
:1010800009B212B21BB2A1830120E283238402B011
:1010900070BD00BFF0B583B0044643696A460621BF
:1010A0003B209847A0B19DF800709DF801109DF875
:1010B00002609DF803209DF804509DF8053041EA38
:1010C000072142EA062243EA05236181A281E381E6
:1010D00003B0F0BD036D026B70B50446DD69C2B1AB
:1010E000636B2BB12B0702D5236D08221A6270BDEA
:1010F0002A06F7D5A26A616A8A421FD0511CA069EC
:10110000A162825C2069266D81423285EAD3A362A6
:10111000E8E7A906E4D5C26A1AB1988C80B2904774
:10112000DEE7C1699B8C4069DBB24E1CE66143542B
:10113000E169E368994228BFE261D1E7226D136853
:1011400023F080031360CDE770B40468037B22684A
:10115000022101FA03F31A4213D042690A49456891
:10116000582000FB021229685068528900684FF627
:10117000FE7631402960C168D24392B20A40C26013
:10118000636070BC704700BFC85B00200A4B1B78CF
:101190008BB130B4094B1C7864B1094B002503EBCB
:1011A000C4041A6899885562D06808330143A34281
:1011B000D160F6D130BC70472C600020E85F002081
:1011C000EC5F00201B4B70B41C788CB31A4E582572
:1011D00005FB00656C685CB3E4684CB32B7B43EAA9
:1011E00041039AB2131283EA121300EB80015340B9
:1011F00000EB4100C00003F00F0343EA021300219B
:1012000000F10C024C309BB232443044297313F489
:10121000004F14BF0E21072142F8041F5B008242D9
:101220009BB2F4D112236360236843F0010323606F
:1012300070BC70472C600020C85B002010B40268AE
:10124000047B11680223A340194209D00649406873
:1012500000240C7001684FF6FE7421400160536059
:101260005DF8044B704700BF2E3E002010B51A4BAE
:1012700093F87D36022B82B006D0184B18680368AD
:101280001B68984702B010BD154B8DF80710186801
:101290000A4690F91A104B1C0FD0436840F2FF1415
:1012A000C3F30803A34208D003EB41230D495A546A
:1012B00043680133436002B010BD037E13F0060F94
:1012C000E0D090F82830002BDCD101220DF107018D
:1012D00023F04CFBD6E700BF94610020547D002032
:1012E0003C7D0020246B00202DE9F8438D498E4A77
:1012F0008E4B8F4CD1ED024A246892ED026AD3EDF9
:10130000027A91ED014AD2ED015A93ED017AD1EDC5
:10131000003A92ED005AD3ED006A864B2060FDEE54
:10132000E33ABDEEC44AFDEEE44ABDEEC55AFDEE19
:10133000E55ABDEEC66AFDEEE66ABDEEC77AFDEE81
:10134000E77A04F1280204F1300003F10801914228
:1013500088BF9842C4ED013A84ED024AC4ED034AC5
:1013600084ED045AC4ED055A84ED066AC4ED076A9B
:1013700084ED087AC4ED097A00F28F801A43500791
:1013800040F08B801A685B68A262E3626A4D95ED5B
:10139000130A30F0C3FF95ED140A814630F0BEFF0A
:1013A00095ED150A804630F0B9FF644A644BD2F8D7
:1013B00034E0966B176B00210025002260F30F05C7
:1013C00069F30F016EF30F0204F13C0068F31F4153
:1013D00066F31F4240EA030667F31F452163710766
:1013E0006563A26304F144055CD19D4203F10801E9
:1013F0008CBF00220122884228BF42F00102002A4D
:1014000050D01A685B68E26323644E4B1A782AB3A3
:101410004D4B04F14801181DA84288BF994246D897
:101420000A2A44D9911E49080131052998681E6885
:101430005D68E0644FEA410018BF59696664A564BD
:10144000DE681D6918BFA16590422665656505D0F7
:1014500004EB400233F81030A2F844303B4D3C4BD3
:101460003C4E3D483D493E4A2D8837688069DE68DC
:1014700009885289A4F86C501D695B69A4F86E70E4
:10148000A4F87460A4F87650A4F878302067A4F823
:101490007A10A4F86620BDE8F8835A681B68E262F7
:1014A000A36273E75A681B682264E363ADE7198897
:1014B000A4F84410012AD1D05988A4F84610022A71
:1014C000CCD09988A4F84810032AC7D0D988A4F8AA
:1014D0004A10042AC2D01989A4F84C10052ABDD09C
:1014E0005989A4F84E10062AB8D09989A4F850104A
:1014F000072AB3D0D989A4F85210082AAED0198A85
:10150000A4F85410092AA9D0598AA4F856100A2A16
:10151000A4D0998AA4F858100B2A9FD0DB8AA4F88B
:101520005A309BE778600020846000206C600020C7
:10153000307D002054490020CC8900208C89002077
:10154000148800208887002060490020C0470020C0
:10155000505200200848002030240020A4450020DC
:101560003C600020F0B585B0002833D0404C238982
:10157000B3F5805F2ED33F4B3F4D1B78E3743F4B59
:101580003F484049404A93F87D362D68007891F8ED
:1015900020101278E560022B20746174A27401ADF2
:1015A00040D03A4B1868036853211B689847E0689D
:1015B0000CF00EF9207C0CF00BF9E37C617CA27C32
:1015C00003932846019102920BF090FF00232381A0
:1015D00005B0F0BD2B4D2849294A2B48254B2C4CF2
:1015E0000968127895F8207006781B78019101AD92
:1015F0008DF808202146284608228DF809708DF8BC
:101600000A608DF80B3032F06BFF0028E0D01B4BE6
:1016100095E8030093F87D36022B84E80300A4F1DB
:101620000C04BED11B4B186890F91A1053224B1CA6
:101630008DF803200ED0436840F2FF16C3F3080371
:10164000B34207D003EB412313495A544368013393
:101650004360ACE7037E13F0060FA8D090F8283063
:10166000002BA4D101220DF1030123F07FF99EE7A5
:10167000C020002070460020148E002094610020BD
:101680004A8E00201C8E0020D88D0020547D002022
:10169000CC2000203C7D0020246B0020274B1B78B1
:1016A00013B1274B1B7803B9704770B5254C2378CD
:1016B00003F0FF05002B40D1234E7369C31A002BA2
:1016C0003BDBB269214B995C01324FF47A730E2AED
:1016D000B26103FB01F11E4A88BFB56100F58C536E
:1016E000143305460B441068736114F0D7FB18B12E
:1016F00005F5C335A035756123784BB115480368EE
:10170000013300E00B462278591C002AFAD103600D
:10171000114B124A19681268114D01264FF43473A7
:1017200000202670536048620B8828809BB23343A8
:101730000B8013683343136070BD70BD9526002085
:101740000C31002034680020C0200020304D0308F8
:101750000431002038680020503D00204C3D00201E
:10176000366800202DE9F04190F84450002280F8BE
:10177000442015B90120BDE8F08118490B6813B960
:101780001846BDE8F0810B68052B02D01046BDE875
:10179000F081134EDFF84C80376800F13004D8F840
:1017A00000302946204683B923F0ACF83368DB1BB0
:1017B000322BA5EB000504440BD8002DDAD0D8F865
:1017C000003029462046002BEED03368DB1B322B3D
:1017D000E5D9B5FA85F04009BDE8F081B4510020A3
:1017E0004488002018520020002280F84520B9E7E4
:1017F00090F844305A1C0344D2B280F8442083F855
:10180000301090F845300BB1132A00D9AAE7704781
:10181000134B186800B970471B68052BFBD12DE9E5
:10182000F041104E002A1446376816DDDFF8388084
:101830000D460AE023F066F83368DB1B322BA4EB7D
:101840000004054409D8002C07DDD8F800302146F3
:101850002846002BEED00020EEE7BDE8F08100BF67
:10186000B451002044880020185200202DE9F04196
:10187000254D264E264F82B02B68002B3DD12C687B
:101880005FFA84FC002C3CD00023307FDFF884E03A
:101890001A460EEB03010DF1080801334244DBB296
:1018A000095C02F8041CA3421A46F2D32B681B1BE6
:1018B0002B60D5F8008060443077B8F1000F06D077
:1018C000002CD9D09DF8040002B0BDE8F081402181
:1018D000032021F081FB3B6886F81C8023F48043C1
:1018E00023F070039BB283F4405343F4004343F06E
:1018F00080033B60002CBFD0E4E74FF0010C64464E
:10190000C2E7307FA446D1E714520020C020002057
:101910000C5C0040D451002070B5084C064620688D
:101920000D4614F0A5FA30462CF094FB28462CF016
:1019300091FB206814F0A2FA012070BD848A002077
:10194000F0B583B004466B46062203211E202CF01E
:101950005DF900283CD09DF800509DF801109DF8DD
:1019600002709DF803209DF804609DF8053041EA5F
:10197000052142EA072243EA062309B212B21BB24A
:10198000144D06EE901A07EE102A07EE903AF8EE84
:10199000E66A95ED005AD5ED025A95ED016AB8EE6A
:1019A000C77AF8EEE77A66EE856A27EE257A67EE63
:1019B000867AFDEEE66ABDEEC77AFDEEE77A16EEB0
:1019C000901A17EE102A17EE903A2180A2806380B9
:1019D00003B0F0BD040000202DE9F043322083B0B5
:1019E00010F0F8FC112200211E202CF005F96022D5
:1019F00001211E202CF000F9642010F0EBFC684659
:101A0000FFF79EFF0024DFF83881254626460A2787
:101A1000012202211E202CF0EFF8322010F0DAFC17
:101A20006846FFF78DFFBDF90000BDF90210BDF952
:101A3000042088420346A8BF0B469342A8BF134622
:101A4000434506440D4414446EDB013FE0D14FF0A2
:101A50000109122200211E202CF0CEF8DFF8E080D0
:101A60000A27012202211E202CF0C6F8322010F095
:101A7000B1FC6846FFF764FFBDF90000BDF9021034
:101A8000BDF9042088420346A8BF0B469342A8BF75
:101A900013464345A6EB0006A5EB0105A4EB0204A3
:101AA00045DB013FDDD107EE906AF8EEE76A07EE0D
:101AB000905AB8EEE77A07EE904ADFED1E5A9FED96
:101AC0001E5A1E4EF8EEE77A85EEA66A70220021B5
:101AD0001E20C5EE876A85EE277AB0EEC66AF0EE64
:101AE000E66AF0EEC77A86ED006AC6ED016AC6EDD9
:101AF000027A2CF081F8202201211E202CF07CF8A3
:101B0000002202211E202CF077F8642010F062FCE5
:101B1000B9F1000F04D14FF07E5333607360B360AE
:101B2000012003B0BDE8F0834FF0000991E74FF0CA
:101B30000009B8E700406F4601C05E46040000207F
:101B400001F0FFFFF0B585B005460DF10703012256
:101B500002210C202CF05AF818B19DF80730DB0751
:101B600003D40024204605B0F0BD02AB06220321B9
:101B70000C202CF04BF80DF10703012209210C2059
:101B80002CF044F804460028EBD09DF8073013F001
:101B90000C0FE6D19DF80D009DF809709DF8081016
:101BA0009DF80B609DF80A209DF80C3041EA072152
:101BB00042EA062243EA0023C1EB8131C2EB8232C2
:101BC000C3EB8333890092009B0029806A80AB803D
:101BD00001220A210C202CF00FF8C3E700B50022E7
:101BE00083B00A210C202CF007F8142010F0F2FB2F
:101BF0000F220A210C202BF0FFFF0A2010F0EAFB35
:101C000001AB032210210C202CF000F80A2010F068
:101C1000E1FB00220A210C202BF0EEFF0A2010F03D
:101C2000D9FB0DF10303012202210C202BF0EEFF62
:101C30000DF10303012209210C202BF0E7FF012203
:101C40000A210C202BF0D8FF012003B05DF804FB23
:101C5000F0B583B004466B46012202210C202BF024
:101C6000D5FF18B19DF80030DA0702D4002003B088
:101C7000F0BD6B46072203210C202BF0C7FF002884
:101C8000F4D09DF806309B07F0D19DF801709DF8C7
:101C900000109DF803609DF802209DF805509DF806
:101CA00004301D4841EA072142EA062243EA05239F
:101CB00009B212B21BB2494252425B4206EE901A7E
:101CC00007EE102A07EE903A90ED035AD0ED045A31
:101CD00090ED056AF8EEE66AB8EEC77AF8EEE77AB4
:101CE00066EE856A27EE257A67EE867AFDEEE66A6D
:101CF000BDEEC77AFDEEE77A16EE901A17EE102ABF
:101D000017EE903A21806280A38001220A210C20E4
:101D10002BF072FFABE700BF0400002000B50022EB
:101D200083B00A210C202BF067FF142010F052FB27
:101D30000F220A210C202BF05FFF0A2010F04AFB33
:101D400001AB032210210C202BF060FF0A2010F0C1
:101D500041FB9DF90430DFED2B7ADFED2B5A06EEC7
:101D6000103A9DF9053006EE903A9DF9063007EEDF
:101D7000103AB8EEC66AF8EEE66AB8EEC77A76EEC2
:101D8000E76A36EE676A37EE677AF7EE007AB0EE0A
:101D9000675AA6EE255A1D4B0022B0EE456AB0EEFA
:101DA000675AA6EEA55A0A210C20E7EE257AF3EE33
:101DB0000E5A26EE256A25EE257A67EEA57A83ED82
:101DC000036A83ED047AC3ED057A2BF015FF0A2030
:101DD00010F000FB0DF10303012202210C202BF077
:101DE00015FF0DF10303012209210C202BF00EFF3A
:101DF00001220A210C202BF0FFFE012003B05DF828
:101E000004FB00BF000000430000803B04000020F2
:101E100028F038BCF8B50B4C074620680E4615462E
:101E200014F026F847F080002CF014F933462946C8
:101E30000022054814F046F9206814F01FF801202C
:101E4000F8BD00BF848A002000300140C36A70B52D
:101E50000446F3B118780EF025FC2023002183718D
:101E6000C171054613F048FE2146454B41F8143F29
:101E700028462CF01FF8AB88B3FA83F3C3F11F0395
:101E80005A1C06D03F490122086802FA03F30343B3
:101E90000B603D4D6E7F002E52D14FF480702CF0C0
:101EA00003F980216B20FFF737FD962010F092FA9E
:101EB00003216820FFF730FD962010F08BFA0321F4
:101EC0006B20FFF729FD0F2010F02AFA10216A205D
:101ED000FFF722FD0F2010F023FA31466C20FFF7A8
:101EE0001BFD0F2010F01CFA94F824101920FFF7A6
:101EF00013FD0F2010F014FA18211B20FFF70CFD22
:101F00000F2010F00DFA18211C20FFF705FD0F20FF
:101F100010F006FA10213720FFF7FEFC0F2010F01A
:101F2000FFF901213820FFF7F7FC0F2010F0F8F936
:101F300002202CF0B9F8012010F0F2F901236B77A0
:101F40004FF480702CF0B0F894F822101A20FFF7AC
:101F5000E3FC012010F0E4F902202CF0A5F8204663
:101F6000FFF772F8E38B5BB2013300D070BDA38B37
:101F70005BB20133FAD10620BDE870400FF054BFC8
:101F80002510000800040140C020002010B51A4BA5
:101F900093F87D36022B82B0014606D0174B1868A5
:101FA00003681B68984702B010BD154B8DF80700F9
:101FB000186890F91A20531C0FD0436840F2FF14A0
:101FC000C3F30803A34208D003EB42230D4A9954FC
:101FD00043680133436002B010BD037E13F0060F67
:101FE000E1D090F82830002BDDD101220DF107015E
:101FF00022F0BCFCD7E700BF94610020547D002094
:102000003C7D0020246B00202DE9F04FDFF8F482A6
:10201000B8F81E3091B00546002B40F02A83B44C2E
:1020200094F87B26012A00F034841846FFF79AFAC8
:102030002846FFF759F9AF4B02931A4694F87D36BC
:102040001768022B60D0AC4B1868036849211B68E5
:102050009847D8F82000DFF8A8B2A74DA74E0BF09C
:10206000B7FB38680BF0B4FB07F10C0394F87D263E
:102070000193BA46039799465AF8047FF91781EA03
:1020800047077F2F09D863E028680368FF091B68AA
:1020900098477F2F94F87D265AD967F07F01022A4E
:1020A000C9B2F1D1306840F2FF1E90F91A308DF8B4
:1020B00017105A1C18D04268C2F30802724502EB8E
:1020C000432311D003F80B104368FF0901337F2F1E
:1020D000436067F07F0140F25A8190F91A30C9B22B
:1020E0005A1C8DF81710E6D1037E13F0060F02D0AC
:1020F00090F8283013B3FF097F2F67F07F0140F27B
:102100004681C9B23068D0E77C4B186890F91A1044
:1021100049224D1C8DF8162000F0C483436840F21C
:10212000FF15C3F30803AB4200F0BC8303EB41236C
:1021300073495A544368013343608AE701220DF121
:102140001701FF0922F012FC7F2F94F87D26A4D8F6
:10215000022AF9B200F01C81286803681B689847BE
:1021600094F87D26CA4587D1039FDFF894A1624D7C
:10217000624EDDF80490019707F118039B4659F869
:10218000047FFB1783EA47077F2F09D83DE02868C3
:1021900003681B68984794F87D26FF097F2F34D980
:1021A00067F07F01022AC9B2F1D1306840F2FF1E08
:1021B00090F91A308DF819105A1C17D04268C2F3E2
:1021C0000802724502EB432310D003F80A1043685B
:1021D000FF0901337F2F436067F07F0129D990F910
:1021E0001A30C9B25A1C8DF81910E7D1037E13F0CA
:1021F000060F02D090F828309BB1FF097F2F67F0BF
:102200007F0116D9C9B23068D2E7022AF9B211D0DB
:10221000286803681B689847D94525D094F87D261F
:10222000ADE701220DF1190122F0A0FB94F87D2603
:10223000B3E7F9B230688DF81A1090F91A20571CDC
:1022400000F0EC80436840F2FF1EC3F308037345BF
:1022500000F0E48003EB4223D94503F80A104368F9
:1022600003F101034360D9D1D8F82430019FDD0385
:1022700000F1E382980300F1D782590300F1CD8287
:1022800007F1280028F064FBB4F8CC30B7F92E0031
:10229000C01A0BF09DFAD8F82430DA0400F1ED8270
:1022A0009E0400F1E3825D0500F1D982180500F17A
:1022B000CD82190400F1AC8207F1300028F048FB10
:1022C00007F1360028F044FBDFF834A00A4D0B4E2E
:1022D000019707F1420307F13A099B4639F9021FBA
:1022E00094F87D26CB1783EA41077F2F16D8A5E007
:1022F00094610020307D0020547D00203C7D002032
:10230000246B0020C0200020286803681B689847C1
:1023100094F87D26FF097F2F40F2908067F07F01BF
:10232000022AC9B2F0D1306840F2FF1E90F91A308B
:102330008DF81B105A1C18D04268C2F3080272456F
:1023400002EB432311D003F80A104368FF0901335D
:102350007F2F436067F07F0140F2428190F91A308D
:10236000C9B25A1C8DF81B10E6D1037E13F0060F7C
:1023700004D090F82830002B00F01281FF097F2F45
:1023800067F07F0140F22C81C9B23068CEE7F9B224
:10239000306840F2FF1E90F91A208DF81810571C73
:1023A00021D04368C3F3080373451CD003EB4223D9
:1023B000CA4503F80B10436803F10103436000F0C2
:1023C00024825AF8043FD91781EA43017F290F4636
:1023D0004FF002023FF661AE90F91A20C9B2571CC5
:1023E0008DF81810DDD1037E13F0060F00F02B815D
:1023F00090F82830002B00F03581CA4500F00582A6
:102400005AF8043F590081EAE3717F290F464FF0E3
:1024100002023FF642AEC9B23068BCE7037E13F059
:10242000060F3FF4F9AE90F82830002B7FF4F4AE9D
:1024300001220DF11A0122F099FAEDE6022AF9B211
:1024400000F0CF80286803681B689847CB457FF46D
:1024500045AF019FBB4BB7F944001B88C01A0BF076
:10246000B7F9B94B1B78012B67DD213307EB430329
:10247000DFF800A3B54DB64E019307F1440939F9D1
:10248000023FB7F9441094F87D26591ACB1783EA16
:10249000410BBBF17F0F0BD844E0286803681B6831
:1024A000984794F87D264FEADB1BBBF17F0F39D9A3
:1024B0006BF07F01022AC9B2EFD1306840F2FF1EF3
:1024C00090F91A308DF81D105A1C19D04268C2F3C9
:1024D0000802724502EB432312D003F80A10436846
:1024E0004FEADB1B0133BBF17F0F43606BF07F01D1
:1024F0005ED990F91A30C9B25A1C8DF81D10E5D179
:10250000037E13F0060F03D090F82830002B3FD045
:102510004FEADB1BBBF17F0F6BF07F0148D9C9B2DB
:102520003068CDE7022A5FFA8BF143D02868036850
:102530001B689847019B9945A1D1D8F8243099058B
:1025400008D5B7F96630A3F2DC53D81780EA430008
:102550000BF03EF9029D7F4928687F4B7F4A6860F7
:10256000441AA41003FB04F3013382FB0342A2EBE1
:10257000E37202EB42029B1AC3EB431301EB8303AA
:102580000122A8602B6088F8A02111B0BDE8F08F6F
:1025900001220DF11D0122F0E9F994F87D2682E770
:1025A00001220DF11B0122F0E1F994F87D26B1E63C
:1025B0005FFA8BF130688DF8201090F91A20531CC7
:1025C00025D0436840F2FF1EC3F3080373451ED0B5
:1025D00003EB422303F80A10436801334360A9E781
:1025E000F9B230688DF81C1090F91A20571C1BD0D6
:1025F000436840F2FF1EC3F30803734514D003EB96
:10260000422303F80A104368013343601EE7037E48
:1026100013F0060F8ED090F82830002B8AD10122BB
:1026200008A922F0A3F985E7037E13F0060F3FF413
:102630000DAF90F82830002B7FF408AF012207A9D6
:1026400022F094F902E7CA4500F0DF805AF8043F0F
:10265000D91781EA43017F290F464FF002023FF666
:102660001CADD8E6012206A922F080F994F87D2657
:1026700078E53B4AD8F8A4311468A34207D0394B17
:10268000C8F8A4411B78093B012B40F2AD82364BC0
:10269000D8F8A8611C68B44207D0324BC8F8A841EA
:1026A0001B78093B012B40F20E81304CB8F81E30EC
:1026B00094F87B1694F87C060B44013BB3FBF0F2D4
:1026C00000FB123399427FF660AF0120FEF74AFF0C
:1026D000274B02931F462846FEF706FE502097E838
:1026E0000006FFF753FC3B68BA68796812681B68FC
:1026F0000868164D164E1344A3EB40000AF0D2FFB3
:10270000DAF80420D9F804309B1A0893DAF8082084
:10271000D9F808309B1A0993D9F80C30DAF80C2054
:102720009B1A0A9308AB01931F4657F8043B4FEAE4
:10273000E37B8BEA430BBBF17F0F94F87D3627D800
:10274000D0E000BF6657002088870020547D00201D
:102750003C7D0020EC200020DF7BEFBD5655555519
:102760006048002048950020148E002094610020CD
:10277000307D0020246B0020286803681B68984780
:1027800094F87D364FEADB1BBBF17F0F40F2AA8045
:102790006BF07F01022BC9B2EED1306840F2FF1E10
:1027A00090F91A308DF81E105A1C1AD04268C2F3E4
:1027B0000802724502EB432313D0494A99544368F7
:1027C0004FEADB1B0133BBF17F0F43606BF07F01EE
:1027D00040F2E28190F91A30C9B25A1C8DF81E10ED
:1027E000E4D1037E13F0060F04D090F82830002BBC
:1027F00000F0CA814FEADB1BBBF17F0F6BF07F015A
:1028000040F2CA81C9B23068CAE7039F0222ACE431
:10281000B7F87A000AF0DCFF4EE57B6AD81780EA49
:1028200043000AF0D5FF2BE53B6A580080EAE370CD
:102830000AF0CEFFD8F824301FE5FB69580080EA83
:10284000E3700AF0C5FFD8F8243013E53B6FD817C2
:1028500080EA43000AF0BCFFD8F8243029E507F1EC
:10286000740028F075F8D8F824301FE5B7F86E002A
:102870000AF0AEFFD8F8243015E5B7F86C30B8F898
:102880002800C01AC0F30D000AF0A2FFD8F82430C7
:1028900006E594F87C36A3F12000B0FA80F04009F8
:1028A000FFF7C4BB037E13F0060F3FF4D2AB90F8E2
:1028B0002830002B7FF4CDAB01220DF1160122F060
:1028C00055F8FFF7C6BB4520FFF760FB1E20FFF75A
:1028D0005DFB20460AF07CFF30460AF079FFE4E613
:1028E000246B0020022B5FFA8BF100F057812868DF
:1028F00003681B6898470BABBB427FF416AFDAF84E
:102900001020D9F810309B1A0893DAF81420D9F85F
:1029100014309B1A0993D9F81830DAF8182008A84F
:102920009B1A0A930AF0E2FDD8F82430DC0300F188
:102930000382980300F1F681590300F1EB81BAF9A3
:102940002830B9F92820D21A0892BAF92A30B9F9F0
:102950002A10C91A0991BAF92C30B9F92C00C01AF9
:102960000A90B9F92E30BAF92E401B1B0B932BB1EC
:1029700003F108040F2C00F2598101239B0030B1B0
:1029800000F108040F2C00F2498143F001039B0081
:10299000DBB231B101F108000F2800F2378143F0BA
:1029A00001039C00E4B232B102F108030F2B00F2E4
:1029B000258144F001042046FFF7E8FA04F0030300
:1029C000022B00F00B82032B00F02282012B00F07F
:1029D0000A82A40804F00303022B00F0E081032B19
:1029E00000F0B481012B00F0338100231846A508C4
:1029F00005F00302022A00F0D781032A00F0E381E8
:102A0000012A40F06382002B40F059820A9B1B018F
:102A1000D8B2AD08022D00F02B82032D00F02F82DA
:102A2000012D00F02E81FFF7B1FAD8F8243013F40D
:102A3000805400F06D81BAF86C10B9F86C20521A0D
:102A40000892022101249A040AD5B9F86E20BAF836
:102A50006E5010A800EB8400521B0C4640F8202C4E
:102A60005F051ED5BAF97400B9F9742010A901EBFD
:102A70008401121A41F8202CBAF97600B9F97620AF
:102A800010A901EB8401121A41F81C2CB9F9782025
:102A9000BAF9780010A901EB8401121A41F8182C38
:102AA00003341E0500F1F480180400F1FF80002CAF
:102AB00040F00781302027F089FE362027F086FE7F
:102AC000029A54689768166804F13A053A37423416
:102AD0003A3635F9023F37F9021F36F9022F0B4417
:102AE00003EBD373A2EB6303D81780EA43000AF029
:102AF0006FFEA542EDD1CB4B02991B780E684D6855
:102B00008F68BBB1213305EB43044237423542366F
:102B100035F9023F37F9021F36F9022F0B4403EB58
:102B2000D373A2EB6303D81780EA43000AF050FE88
:102B3000A542EDD1D8F824309B0506D5B9F9660039
:102B4000BAF96630C01A0AF0ADFD029EB649306887
:102B50007468B460B54BB64A7060441AA41003FBA5
:102B600004F3013382FB0342A2EBE37202EB420265
:102B70009B1AC3EB431301EB83030122336088F8F4
:102B8000A02111B0BDE8F08F01220DF11E0121F04E
:102B9000EDFE94F87D36F5E55FFA8BF130688DF83F
:102BA0001F1090F91A20531C0ED0436840F2FF1EEC
:102BB000C3F30803734507D003EB42239D4A99549E
:102BC00043680133436096E6037E13F0060F3FF43B
:102BD00092AE90F82830002B7FF48DAE01220DF1DB
:102BE0001F0121F0C3FE86E64520FFF7CFF9002044
:102BF000FFF7CCF920460AF0EBFD48E58032FF2ACA
:102C000094BF44F0020444F00304D4E68031FF2969
:102C10008CBF43F0030343F00203C2E68030FF2879
:102C20008CBF43F0030343F00203B0E68033B3F5F7
:102C3000807F34BF02230323A0E6099BC3F3033341
:102C40001843FFF7A3F90998C0F30710FFF79EF99F
:102C5000099B1B01D8B2A50805F00303022B00F065
:102C60001D81032B00F0F280012B00F02881240944
:102C7000022C00F0FD80032C00F00181012C7FF478
:102C8000D2AE0B9B03F00F031843FFF77FF9CCE69E
:102C9000D9F87020DAF8701010A800EB8400521AEE
:102CA0001D0440F8202C04F101040AD5B9F87A304B
:102CB000BAF87A1010AA02EB84025B1A42F8203CA0
:102CC0000134012C00F0F48008AB03EB84020020F7
:102CD000631E52F8041D40000029C0B203F1FF3307
:102CE00018BF40F00100591CF3D1FFF74FF9002540
:102CF000019E02E0A542BFF6DDAE56F8043B013569
:102D0000002BF7D0D81780EA43000AF061FDF1E705
:102D1000012198E6D9F82400DAF82430C01A0AF024
:102D2000C1FC0CE6DAF82030D9F82000C01A0AF00D
:102D3000B9FCD8F82430FFE5DAF81C30D9F81C00CB
:102D4000C01A0AF0AFFCD8F82430F2E59DF825004F
:102D5000FFF71CF99DF82400FFF718F9A50805F006
:102D60000303022B22D0032B2FD0012B3FF44EAEB6
:102D70002409022C0ED0032C08D0012C7FF455AE70
:102D80000B9B1B01D8B24EE6002B78D19DF82D008D
:102D9000FFF7FCF89DF82C00FFF7F8F845E69DF8E2
:102DA0002400FFF7F3F8D9E7002B77D19DF828002E
:102DB000FFF7ECF8AD08022DECD0032DE6D0012D85
:102DC0007FF433AEDCE7002B40D19DF82900FFF7FC
:102DD000DDF89DF82800FFF7D9F8EBE79DF8200013
:102DE000FFF7D4F8F5E5089AA408100104F00302EF
:102DF000022AC0B220D0032A3FF41FAF012A7FF479
:102E0000F6AD099B03F00F031843FFF7BFF8A5E7E2
:102E10009DF82100FFF7BAF89DF82000FFF7B6F8FB
:102E2000D7E500BF88870020EC200020DF7BEFBDC6
:102E300056555555246B0020099BC3F303131843C3
:102E4000FFF7A4F8099B1B01D8B204E70A9BC3F360
:102E500003331843FFF79AF80A98C0F30710FFF7F7
:102E600095F80A9BAD081B01022DD8B27FF4D5ADB1
:102E70000B9BC3F303131843FFF788F880E70B9B02
:102E8000C3F303331843FFF781F80B98C0F307101F
:102E9000FFF77CF80B9B1B01D8B2C4E50A9BC3F378
:102EA00003131843FFF772F80A9B1B01D8B2B0E571
:102EB000089BD81780EA43000AF08AFCFAE50A9BCF
:102EC00003F00F031843FFF761F873E72409022C9E
:102ED00008D0032C3FF458AF012C07D1002B3FF44E
:102EE0004FAFCEE6002B3FF455AFC1E7002B3FF4C8
:102EF0009CAD98E52DE9F04F89B0904D139F149E3D
:102F0000D5F8B041DDF848A09B1A0293F31B904618
:102F1000019300290CBF04230623621C049300F0D4
:102F2000CD80A24562DDDFF82C9247B1019B04FB06
:102F300003F20123B95C6A6A8B40134251D0029BB1
:102F4000D5F8AC2104FB03F408EB0406002A40F09A
:102F5000868058F8040003922CF02EFD039A053069
:102F6000D9F8003083424EDA012009B0BDE8F08F75
:102F7000734B1B6893F91AE02C20BEF1FF3F8DF8CC
:102F80001F0000F08780596840F2FF1CC1F3080160
:102F900061457FD001EB4E21DFF8C0E101F80E0062
:102FA000596801315960002A5BD158F804400393F5
:102FB00020462CF001FD039B197E11F0060F07D06F
:102FC00093F8282022B902462146184621F0CEFC6B
:102FD00096F904104B1C39D05A480AF00FFED5F868
:102FE000B0410134A245C5F8B0419EDCA24500F0D5
:102FF0009180D5F8AC01049B834294BF002001204E
:1030000009B0BDE8F08F95F8B4111B1AC9F800306B
:1030100079BB012385F8B4311ABB4B4B58F80440F7
:1030200093F87D36022B46D021780029D0D0DFF8E6
:1030300030B1DBF8000003681B68984714F8011FE3
:103040000029F6D196F904104B1CC5D1D5F8B04132
:103050000134A245C5F8B0413FF767AFC6E703208A
:103060007EE71644394831790AF0C8FDD5F8B041F9
:10307000EEE7354B93F87D36022B3FF479AFDFF85E
:10308000E0B0DBF8000003682C211B689847D5F8F6
:10309000AC21C1E7197E11F0060F84D093F82810F7
:1030A000002980D1012218460DF11F0121F05EFC9C
:1030B000D5F8AC21B0E7224B1B6878E7D5F8AC41D6
:1030C000A34203D8002009B0BDE8F08F204B059142
:1030D00003EB840381461A69039210462CF06CFCC2
:1030E0001C4E039A336805990B3098423FF73CAF6A
:1030F000032C98BF494618480AF080FD3368D5F87C
:10310000B0411B1A013400223360C5F8B04185F884
:10311000B42106E70F4A1368002B7FF76AAF013B23
:103120000A201360FEF732FFD5F8AC014FF0FF33F1
:103130000130C5F8AC01C5F8B0315CE7C020002013
:103140003C7D0020387603089461002098A703088E
:10315000304D0308642E002028760308246B0020DD
:10316000547D002070B5204C23780B2B08D8012209
:103170009A4040F603010A4209D112F4C06F07D108
:103180001A4A1B4B1268C3F8B0210B23237070BD81
:10319000093B012BF4D84520FEF7F8FEFF20FEF78F
:1031A000F5FE144B93F87D36022B0ED0124D134EC4
:1031B0004521306803681B68984715F8011F0029EE
:1031C000F7D10020FEF7E2FEDAE70D4B1868037E28
:1031D00013F0060FF5D090F82830002BF1D10A2219
:1031E000054921F0C3FBECE7489500204488002006
:1031F000C02000209461002040760308547D002008
:103200003C7D0020A54B1B78012B00D070472DE999
:10321000F04FA34D95F87B0685B018B195F87C6604
:10322000002E31D1012385F87B3685F87C3695F860
:103230007D3623B1022B3DD0002385F87D36994B96
:1032400099491B6800220A701A88160600F17F83CC
:103250001A89140600F1AC831A8A100600F1AF83B4
:103260001A8B160600F1B1831A8C140600F1AA839A
:103270001A8D100600F1AC8306230B70874A0023D9
:10328000137005B0BDE8F08FB042CBD20146324694
:1032900000E01A4691FBF2F302FB13131146002BD8
:1032A000F7D190FBF2F096FBF2F285F87B0685F8F9
:1032B0007C26BCE77D4B5A78012ADFD941F2B51252
:1032C0009B5C002BDAD17A4E402386F8B6317949DF
:1032D000794A0F68DFF8F8C195F87B167748784B84
:1032E0000291C7F3C031A2F5887EBCF800C00391FB
:1032F0007449D3F800A0C0F804E095F8B332A6F8FA
:1033000028C0A2F1940EA2F5C67C95F87C86C0F880
:1033100000C0C0F808E00020D1F800E00299C6F82B
:10332000B801DFF8B09195F8674250609060D060C6
:103330001061A3F119024145B2FA82F207F4006C60
:10334000C7F3400B4FEA5212CAF3800799F8009076
:1033500095F84452CAF3C00A2CBF00210121002C69
:103360007ED0012B00F09281BCF1000F40F0F18083
:1033700001256046A8466B1EDBB203F1FF3CBCF1A1
:10338000130F14D8DFE80CF00A0A0A0A0A0A0A0A1C
:1033900037321B201816132525253C169945B4BF36
:1033A0004FF0000C4FF0010CBCF1000F02D008FAF6
:1033B00003F31843142D29D80135EDB2DBE7BC46E1
:1033C000BCF1000FF3D1F7E7DC46BCF1000FEED102
:1033D000F2E70EEB030C9CF804C01CF1000C18BFC4
:1033E0004FF0010CBCF1000FE1D1E3E7D446BCF192
:1033F000000FDCD1E0E79446BCF1000FD7D1DBE74A
:103400008C46BCF1000FD2D1D6E7029E244B7062ED
:1034100003F1500102E0043399421FD093F8D12503
:103420001A2AF8D193F8D30593F8D4259042F2D212
:1034300001232549254A86F8CC3100233362F383E2
:10344000A6F8CE3186F8A031144B08681168C6F88A
:10345000A4010222C6F8A8111A7012E70023E8E7B7
:10346000012B00F05381BCF1000F40F0B880012522
:103470006046A8466B1EDBB203F1FF3CBCF1130FA4
:1034800036D8DFE80CF051515151515151514C3D5A
:1034900042473A385B292929613800BF4895002006
:1034A00094610020947E0020987E00200C6B002008
:1034B000C0200020B47E002078220020307D002033
:1034C000248A00208C41002060480020148E0020B7
:1034D000C0470020888700200EEB030C9CF804C036
:1034E0001CF1000C18BF4FF0010CBCF1000F02D012
:1034F00008FA03F31843142D88D80135EDB2B9E763
:10350000D446BCF1000FF3D1F7E7BC46BCF1000F85
:10351000EED1F2E7DC46BCF1000FE9D1EDE79446CD
:10352000BCF1000FE4D1E8E74B45CCBF4FF0000CF5
:103530004FF0010CBCF1000FDAD1DCE7DDF80CC074
:10354000BCF1000FD4D1D8E78C46BCF1000FCFD12D
:10355000D3E7012D00F05D814FF0010CE0460CF146
:10356000FF33DBB25D1E132D10D8DFE805F00A0A29
:103570000A0A0A0A0A0A27231B1F16120F2B2B2BD3
:1035800034129945B4BF0025012515B108FA03F39B
:103590001843BCF1140F3FF639AF0CF1010C5FFA80
:1035A0008CFCDCE73D46002DF0D1F6E75D46002DB2
:1035B000ECD1F2E75546002DE8D1EEE71546002D97
:1035C000E4D1EAE70EEB03052D79003518BF01259C
:1035D000002DDBD1DDE70D46002DD7D1DDE7012D34
:1035E00000F0F98101252046A8466B1EDBB203F1ED
:1035F000FF3CBCF1130F17D8DFE80CF03333333343
:10360000333333332E1F24291C193D0A0A0A431968
:103610000EEB030C9CF804C01CF1000C18BF4FF01B
:10362000010CBCF1000F02D008FA03F31843142D6B
:103630003FF6ECAE0135EDB2D7E7D446BCF1000F52
:10364000F2D1F7E7BC46BCF1000FEDD1F2E7DC4662
:10365000BCF1000FE8D1EDE79446BCF1000FE3D1D7
:10366000E8E79945B4BF4FF0000C4FF0010CBCF1F6
:10367000000FD9D1DBE7DDF80CC0BCF1000FD3D1CE
:10368000D8E78C46BCF1000FCED1D3E7012D00F076
:10369000E981BCF1000F00F082809C465A1ED2B234
:1036A000551E132D12D8DFE805F0262626262626DD
:1036B0002626111A221E1714110A0A0A2D140EEBBF
:1036C00002052D79003518BF012515B10CFA02F25B
:1036D0001043142B3FF69AAE0133DBB2DEE75546BA
:1036E000002DF3D1F8E75D46002DEFD1F4E73D461C
:1036F000002DEBD1F0E79145B4BF00250125002D49
:10370000E4D1E6E70D46002DE0D1E5E7BCF1000F7E
:1037100040F0CB80DDF80C80029660461D465A1EB4
:10372000D2B202F1FF3CBCF1130F10D8DFE80CF06D
:103730000A0A0A0A0A0A0A0A0F2B271815122F1C4E
:103740001C1C33129145B4BF0026012616B105FAA0
:1037500002F21043142B3FF658AE0133DBB2DEE722
:103760005E46002EF3D1F8E70EEB020C9CF804C085
:103770001CF1000618BF0126002EE8D1EAE73E46FC
:10378000002EE4D1E9E75646002EE0D1E5E74646B3
:10379000002EDCD1E1E70E46002ED8D1DDE76046F1
:1037A0009C465A1ED2B2551E132D10D8DFE805F0E4
:1037B0000A0A0A0A0A0A0A0A0F201C1815120F24FC
:1037C00024242D129145B4BF0025012515B10CFA12
:1037D00002F21043142B3FF619AE0133DBB2E0E7DF
:1037E0005D46002DF3D1F8E73D46002DEFD1F4E71B
:1037F0005546002DEBD1F0E70EEB02052D79003593
:1038000018BF0125002DE2D1E4E70D46002DDED1E1
:10381000E3E7A8466B1EDBB203F1FF3CBCF1130FDC
:1038200017D8DFE80CF02E2E2E2E2E2E2E2E291F2E
:1038300024381619160A0A0A3D190EEB030C9CF8D7
:1038400004C01CF1000C18BF4FF0010CBCF1000FBC
:1038500002D008FA03F31843142D3FF6D7AD013513
:10386000EDB2D7E7D446BCF1000FF2D1F7E7BC4682
:10387000BCF1000FEDD1F2E79446BCF1000FE8D1A6
:10388000EDE79945B4BF4FF0000C4FF0010CBCF1CF
:10389000000FDED1E0E7DC46BCF1000FD9D1DEE756
:1038A0008C46BCF1000FD4D1D9E7012D204600F0A1
:1038B0005981DDF80C801D465A1ED2B202F1FF3C40
:1038C000BCF1130F14D8DFE80CF00A0A0A0A0A0A3E
:1038D0000A0A132B261C1916213030303D1691454B
:1038E000B4BF4FF0000C4FF0010CBCF1000F02D040
:1038F00005FA02F21043142B3FF688AD0133DBB218
:10390000DAE7DC46BCF1000FF2D1F7E7C446BCF1C0
:10391000000FEDD1F2E7BC46BCF1000FE8D1EDE7B6
:10392000D446BCF1000FE3D1E8E70EEB020C9CF8A3
:1039300004C01CF1000C18BF4FF0010CBCF1000FCB
:10394000D6D1D8E78C46BCF1000FD1D1D6E7012003
:1039500008707F495E7993F9020051F826307D4E58
:10396000802A14BF02270127B3F5613F14BF00214D
:1039700002210222019100928021002286F8B57175
:103980001DF034FD744B75491B68754A03EB430306
:10399000A1FB03135B09106008D0402BA8BF402394
:1039A00086F8B63100287FF492AC67E40123F7E78C
:1039B0000226012013EBC0030E70CAD15EE4032679
:1039C0000220F7E705260420F4E704260320F1E7A8
:1039D00006260520EEE72046A84602966B1EDBB2BF
:1039E00003F1FF3CBCF1130F10D8DFE80CF00A0A1A
:1039F0000A0A0A0A0A0A2F2B181C0F123320202049
:103A000037129945B4BF0026012616B108FA03F310
:103A10001843142D3FF6F9AC0135EDB2DEE73E4612
:103A2000002EF3D1F8E75E46002EEFD1F4E70EEB5F
:103A3000030C9CF804C01CF1000618BF0126002EE0
:103A4000E4D1E6E75646002EE0D1E5E71646002E23
:103A5000DCD1E1E7039E002ED8D1DDE70E46002E33
:103A6000D4D1D9E7BCF1000F38D0AC466B1EDBB225
:103A70005A1E132A10D8DFE802F00A0A0A0A0A0AB4
:103A80000A0A0F2925180F120F1C1C1C2D124B455A
:103A9000CCBF0022012212B10CFA03F31843142DFB
:103AA0003FF6B4AC0135EDB2E0E75A46002AF3D157
:103AB000F8E70EEB03021279003218BF0122002A48
:103AC000EAD1ECE73A46002AE6D1EBE75246002A73
:103AD000E2D1E7E70A46002ADED1E3E76046AC46DA
:103AE0006B1EDBB25A1E132A12D8DFE802F026261C
:103AF000262626262626111A221E1714110A0A0A1D
:103B00002D140EEB03021279003218BF012212B1FC
:103B10000CFA03F31843142D3FF678AC0135EDB2DF
:103B2000DEE75246002AF3D1F8E75A46002AEFD1E1
:103B3000F4E73A46002AEBD1F0E79945B4BF0022FA
:103B40000122002AE4D1E6E70A46002AE0D1E5E7AF
:103B500038730308C02000206C480020D34D621049
:103B6000547D00202A466B1EDBB203F1FF3CBCF102
:103B7000130F17D8DFE80CF03434343434343434D1
:103B80001629241F16192E0A0A0A3E190EEB030CD9
:103B90009CF804C01CF1000C18BF4FF0010CBCF1E4
:103BA000000F02D002FA03F31843142D3FF62EAC97
:103BB0000135EDB2D7E7DC46BCF1000FF2D1F7E7F3
:103BC000BC46BCF1000FEDD1F2E7D446BCF1000FCA
:103BD000E8D1EDE7DDF80CC0BCF1000FE2D1E7E77A
:103BE0004B45CCBF4FF0000C4FF0010CBCF1000F67
:103BF000D8D1DAE78C46BCF1000FD3D1D8E700BFAB
:103C00002DE9F04FAD4DAE4C2B78DA1E052A8DB064
:103C1000064640F2B880023B092B25D8DFE813F0B6
:103C20001901C101F8012400240015022B023602FB
:103C30002B016001A34F7B78032B15D141F2A40225
:103C40000123BA5C3375002A01F0ED8041F2E802ED
:103C5000BA5C002A01F0E88041F22C13FB5C002BD7
:103C600001F065810023337594F87D26022A11D175
:103C7000944A41F2B513D35C5BB1934F97F8D031BE
:103C800001222A7013B1002387F8D0310DB0BDE8AE
:103C9000F08F022294F87E36002BF7D08B4B1968F8
:103CA00011F4805100F0EE82B4F8EC108848B0F9BD
:103CB0000430B0F90270B0F906608F4208BF8B4241
:103CC00014BF01230023B0F908708E4218BF43F0DF
:103CD0000103B0F90A608F4218BF43F00103B0F945
:103CE0000C708E4218BF43F00103B0F90E608F4292
:103CF00018BF43F00103B0F910708E4218BF43F0B3
:103D00000103B0F912608F4218BF43F00103B0F90C
:103D100014708E4218BF43F00103B0F916608F4251
:103D200018BF43F001038E4218BF43F00103002B7C
:103D300040F0E781B0F900308B4240F0E281654EFF
:103D4000614F3368D7F8D411994200F2E2812B78A1
:103D5000012B9BD097F8D021002A97D00B2B0CD8A1
:103D600001229A4040F603010A428CD112F4C06F3E
:103D700003D0093B012B41F267803368C7F8B031AB
:103D80000B232B707FE794F87D26002A00F0A0819A
:103D9000022A40F000824B4F41F22702BA5CD00762
:103DA00040F17A82002241F23701795CC90706D4DA
:103DB00041F23601795C012998BF02F5007241F2A7
:103DC0004701795CC80706D441F24601795C0129B4
:103DD00098BF02F5007241F25701795CC90706D419
:103DE00041F25601795C012998BF02F5007241F257
:103DF0006701795CC80706D441F26601795C012944
:103E000098BF02F5007241F27701795CC90706D4C8
:103E100041F27601795C012998BF02F5007241F206
:103E20008701795CC80706D441F28601795C0129D3
:103E300098BF02F5007241F29701795CC90706D478
:103E400041F29601795C012998BF02F50072104693
:103E500044E194F87D26022A00F055861D4B1A494C
:103E60001B681D4EC1F8B03103200023C1F8AC31EE
:103E700033602870FAE6144F97F8CC3123B1174B12
:103E80001B685B0140F111823046FEF7BDF8FB8BE9
:103E900039893A6A01339BB201310132202BFB830D
:103EA00039813A627FF4E0AEB7F8CE3194F87D26DE
:103EB00001330021A7F8CE31F983D7E648950020D9
:103EC000946100200C6B0020C0200020B47E0020F4
:103ED0004058002044880020642E0020148E0020CA
:103EE00094F87D26AD4F022A41D197F8A031AC4E0F
:103EF000002B40F0E281D6F80080B8F1000F32D0FC
:103F000098F800307BB398F82820002A7FF4B0AEF0
:103F100098F81830D8F82410C8F8382088F83C20D1
:103F200013F008034FF0040288F82820C8F82C107A
:103F3000C8F8301003D09B4A41F29413D358C8F804
:103F400034304FF00009C8F82490C8F80890C8F839
:103F50000C90404626F0D2FE0523C8F8409088F821
:103F6000283094F87D2600210423316033758E4972
:103F7000D7F8B0310968C8338B420CD3002A00F05F
:103F80003B87022A7FF486AE19F0E2F994F87D2689
:103F900000283FF46BAE002A00F00C8701232B7041
:103FA00064E67E4F804AD7F8B0311268643393429A
:103FB000BFF45AAEDFF80092D9F800303F2B5FDD36
:103FC000D7F8AC31794E4FF040080FE0FDF7DEFF37
:103FD000D9F80020D7F8AC31013A0133B8F1010823
:103FE000C9F80020C7F8AC3100F01287334493F8C9
:103FF00028301846002BE9D14FF0FF32002104236E
:10400000C7F8B021C7F8AC112B7094F87D262DE6C7
:10401000674A0292A2F10C03292101930091A2F1B7
:104020000A035021163A4920FEF764FF00287FF466
:104030001BAE5A4B94F87D26C3F8AC0107214FF014
:10404000FF30C3F8B001297010E65A4B002105205B
:104050008DE80300A3F1080202915320FEF74AFF06
:1040600000287FF401AE4D4B94F87D26C3F8AC01D7
:1040700008232B70FAE5504B1B683F2B00F3A880F8
:1040800094F87D26002A7FF4F1AD03E64B4B434FB5
:104090001B6813F0806FFB8B3FF4FAAE002B7FF4AC
:1040A000F7AED7F820804520FDF770FF0E20FDF712
:1040B0006DFF404609F08CFB304609F089FB4FF458
:1040C00080520A2330463A812B70FDF79DFFDEE6D1
:1040D0003B4B186803689B6898472B78DFF8D8E05B
:1040E0002E4FDEF8002097F8B6110A44B2F5807F13
:1040F000A8BF4FF480728242A8BF0246CEF80020CB
:1041000089E5294B254F1B6803F59C530833C7F8F5
:10411000D4312B78012B7FF4B9AD97F8D031002B37
:104120007FF4B4AD8ABB274B2749284893F900C0D8
:1041300093F90CE093F9186093F9245093F9304007
:1041400093F93C800B6802700132D2B2C3B1198876
:1041500001F08101812913D193F90210614500F02A
:10416000C7868E4500F0C186B14200F0BB86A942E9
:1041700000F0B0868C4200F0D786414500F0D18631
:10418000062A03F10803DFD10270FFF73BF8012391
:1041900087F8D0317AE50020A0E700BFC0200020DA
:1041A0003C7D00200C6B002044880020304D03082B
:1041B000CE4D0308AC4F0308642E0020148E00205F
:1041C000547D0020487E0020947E0020907E0020B8
:1041D00094F8D025B24F742303FB0243D7F8AC11F7
:1041E00093F8C0344A2900F2CB85DFE811F0B3011F
:1041F000A7019E0196018B014F0146013D01780206
:104200006F0269025C0254024D0244023B02320218
:1042100021021002FF01EE01DD01CC01BB017A0495
:104220006504550445043504250415040504F50307
:10423000E503D903C903BD03B103A50399038D03A6
:10424000220316030A03FE02F202E602DA02CE029B
:10425000C202B602AA029E0295028C0283023401B7
:104260002B01200115010B010201F900F000E7000C
:10427000DE00D500CC00C300BA00B100A8008F005A
:104280008200A000874B1B681B7A053B032B7FF63F
:104290000DADB4F8D01009E541F22602BA5C022A4D
:1042A00034BF4FF4007200227DE597F8D031002B27
:1042B0007FF4EAAD09232B70E9E5306800283FF46C
:1042C00052AE0378002B3FF44EAE90F82830002B0E
:1042D0007FF4CEAC82684168C3628A4238BF0A4626
:1042E0000323826080F8283018F060F994F87D2666
:1042F00039E694F8F9116C4809F0FEFAD7F8AC31B8
:104300000133C7F8AC3194F87D26AFE4D4ED367AAA
:104310009FED667A664867EE877AFDEEE77A17EEDC
:10432000901A09F0E9FAD7F8AC310133E9E7A1684E
:10433000604809F0E1FAD7F8AC310133E1E7B4F8AD
:10434000D2105D4809F0D8FAD7F8AC310133D8E77C
:1043500094F8D410594809F0CFFAD7F8AC310133AA
:10436000CFE794F8D510564809F0C6FAD7F8AC3123
:104370000133C6E794F85C12524809F0BDFAD7F849
:10438000AC310133BDE7B4F876124F4809F0B4FA06
:10439000D7F8AC310133B4E794F872124B4809F006
:1043A000ABFAD7F8AC310133ABE794F87012484858
:1043B00009F0A2FAD7F8AC310133A2E794F8B012B1
:1043C000444809F099FAD7F8AC31013399E794F8E9
:1043D0000F12414809F090FAD7F8AC31013390E759
:1043E00094F824123D4809F087FAD7F8AC3101332C
:1043F00087E794F819123A4809F07EFAD7F8AC31F9
:1044000001337EE7B4F816329FED287A354807EE7F
:10441000903AF8EEE77A7EE7B4F80A22B4F806128A
:10442000314809F069FAD7F8AC31013369E7B4F8DB
:104430000822B4F804122D4809F05EFAD7F8AC311E
:1044400001335EE794F80112294809F055FAD7F8CC
:10445000AC31013355E794F80012264809F04CFAC4
:10446000D7F8AC3101334CE74FF07E51224809F0C8
:1044700043FAD7F8AC31013343E7B4F8CE101F4804
:1044800009F03AFAD7F8AC3101333AE7B4F8CC1076
:104490001B4809F031FAD7F8AC31013331E700BFDE
:1044A000C020002058570020287C03080000C84284
:1044B000107C0308387C0308FC7B0308E47B0308BA
:1044C000CC7B0308B47B0308947B0308747B03084C
:1044D000607B0308447B0308347B0308207B0308CC
:1044E000107B0308007B0308E87A0308D47A0308EA
:1044F000C07A0308AC7A03082C7703081C770308FA
:104500000C77030894F87C2694F87B16CF4809F0C2
:10451000F3F9D7F8AC310133F3E6CD49CD4809F0D2
:10452000EBF9D7F8AC310133EBE6CB4ACB49CC48B9
:1045300009F0E2F9D7F8AC310133E2E6C94B009358
:10454000C94ACA4BCA49CB4809F0D6F9D7F8AC31A9
:104550000133D6E6C849C94809F0CEF9D7F8AC31DD
:104560000133CEE6742101FB02F203EB430302EBBD
:1045700083032344C24893F8CA1409F0BDF9D7F85D
:10458000AC310133BDE6742101FB02F203EB4303BE
:1045900002EB83032344BB4893F8C61409F0ACF93B
:1045A000D7F8AC310133ACE6742101FB02F203EB26
:1045B000430302EB83032344B34893F8C51409F083
:1045C0009BF9D7F8AC3101339BE6742101FB02F271
:1045D00003EB430302EB83032344AC4893F8CB146F
:1045E00009F08AF9D7F8AC3101338AE6742101FB6E
:1045F00002F203EB430302EB83032344A44893F842
:10460000C31409F079F9D7F8AC31013379E6742194
:1046100001FB02F203EB430302EB830323449D48B7
:1046200093F8C41409F068F9D7F8AC31013368E69F
:10463000742101FB02F203EB430302EB83032344E7
:10464000954893F8C21409F057F9D7F8AC31013303
:1046500057E694F8F811914809F04EF9D7F8AC31C3
:1046600001334EE694F8FE118D4809F045F9D7F86C
:10467000AC31013345E68B4B8B48996C09F03CF922
:10468000D7F8AC3101333CE6884B1B681A0500F1C2
:104690003C840E2335E6398D854809F02DF9D7F88D
:1046A000AC3101332DE694F83B3294F83D2294F876
:1046B0003C12804809F020F9D7F8AC31013320E6EC
:1046C0007B6AD90400F117840D231AE67A4B7B48E4
:1046D000198909F011F9D7F8AC31013311E6784B9B
:1046E000784A19881288784809F006F9D7F8AC3169
:1046F000013306E694F8FF11744809F0FDF8D7F885
:10470000AC310133FDE594F84D12714809F0F4F82D
:10471000D7F8AC310133F4E594F84C126D4809F048
:10472000EBF8D7F8AC310133EBE5742303FB02421D
:104730006948D2F8A41409F0DFF8D7F8AC31013396
:10474000DFE5742303FB02426448D2F8A01409F0A9
:10475000D3F8D7F8AC310133D3E5742303FB02421D
:104760005F48D2F8BC1409F0C7F8D7F8AC31013370
:10477000C7E5742303FB02425A48D2F8B81409F083
:10478000BBF8D7F8AC310133BBE5742303FB02421D
:10479000554892F8B51409F0AFF8D7F8AC310133A9
:1047A000AFE5742303FB0242504892F8B41409F0B9
:1047B000A3F8D7F8AC310133A3E5742303FB02421D
:1047C0004B48D2F8B01409F097F8D7F8AC31013360
:1047D00097E5742303FB02424648B2F8AE1409F091
:1047E0008BF8D7F8AC3101338BE5742303FB02421D
:1047F000414892F8AA1409F07FF8D7F8AC31013398
:104800007FE5742303FB02423C4892F8A91409F0A7
:1048100073F8D7F8AC31013373E5742303FB02421C
:10482000374892F8A81409F067F8D7F8AC3101338B
:1048300067E5742303FB0242324892F89C1409F0A6
:104840005BF8D7F8AC3101335BE500BFF8760308BD
:104850001C680020E8760308BC760308C8760308C5
:10486000D4760308B07603087C76030854900308D6
:1048700084760308907603085C760308687603085C
:1048800030780308247803081878030808780308A8
:10489000F8770308EC770308E0770308C877030884
:1048A000B4770308CC890020A8770308B47E0020E1
:1048B000887703086C7703088C89002050770308F9
:1048C000665700206C5700203C770308A07A030845
:1048D000907A0308947A03087C7A03086C7A0308B8
:1048E000587A0308407A0308287A0308107A0308E4
:1048F000F8790308DC790308C8790308AC79030860
:104900009479030878790308742303FB02428848EA
:10491000B2F89A1408F0F0FFD7F8AC310133F0E4A4
:10492000742303FB02428348B2F8981408F0E4FFB2
:10493000D7F8AC310133E4E4742303FB02427E4830
:10494000B2F8961408F0D8FFD7F8AC310133D8E4A8
:10495000742303FB02427948B2F8941408F0CCFFA8
:10496000D7F8AC310133CCE4742303FB0242744822
:1049700092F8921408F0C0FFD7F8AC310133C0E4CC
:10498000742101FB02416F4891F8913491F887241A
:1049900091F87D1408F0B0FFD7F8AC310133B0E4E2
:1049A000742303FB0242684892F87C1408F0A4FFC9
:1049B000D7F8AC310133A4E4742101FB0241634810
:1049C00091F88F3491F8852491F87B1408F094FFC6
:1049D000D7F8AC31013394E4742101FB02415C4807
:1049E00091F88E3491F8842491F87A1408F084FFB9
:1049F000D7F8AC31013384E4742101FB02415548FE
:104A000091F88D3491F8832491F8791408F074FFAB
:104A1000D7F8AC31013374E4742101FB02414E48F4
:104A200091F88C3491F8822491F8781408F064FF9E
:104A3000D7F8AC31013364E4742101FB02414748EB
:104A400091F88B3491F8812491F8771408F054FF91
:104A5000D7F8AC31013354E4742101FB02414048E2
:104A600091F88A3491F8802491F8761408F044FF84
:104A7000D7F8AC31013344E4742101FB02413948D9
:104A800091F8893491F87F2491F8751408F034FF77
:104A9000D7F8AC31013334E4742101FB02413248D0
:104AA00091F8883491F87E2491F8741408F024FF6A
:104AB000D7F8AC31013324E4742103EB430301FB49
:104AC00002F101EB83012144284891F8C93491F89F
:104AD000C82491F8C71408F00FFFD7F8AC310133A0
:104AE0000FE4742101FB02F203EB430302EB8303A7
:104AF00023441F48B3F8CC1408F0FEFED7F8AC31BD
:104B00000133FFF7FEBB1B4E337D052B3FF6ACA8F0
:104B100001A252F823F000BF353C0008693C0008B0
:104B20000B4D0008D14B00081F4C0008794D0008C0
:104B3000607903084C7903083C7903082C79030851
:104B40001479030804790308F8780308E478030863
:104B5000D0780308BC780308AC7803089C78030875
:104B60008C7803087878030864780308547803087D
:104B7000407803083C7D0020716891F91A305F1C71
:104B80000AD0C54A03F5817302EB0313FF20DA79DB
:104B90006FF30002DA71887691F91B30581C15D03A
:104BA000BD4F03F5817307EB031207EB0317D279AF
:104BB000FB79C2F34502012AC6BF02F1FF32D2B22D
:104BC0000022FF2062F34603FB71C876032333758E
:104BD000B2480378002B7FF447A87768002F00F0D5
:104BE0004F8197F82830002B7FF43EA828384422C4
:104BF00039462DF067F93B787BB197F8283063B9D7
:104C0000BA687968FB628A4238BF0A460323BA60F1
:104C100087F82830384617F0C9FC002373603769DD
:104C2000DFF894E2DFF894B29D4BDFF89492DFF85E
:104C3000948201370497AEFB077C049FABFB077B94
:104C4000049F0FCBA9FB0779049F4FEADC0CA8FB5C
:104C50000778AEFB0C7A4FEADA0A0AEB8A070DF105
:104C6000200AAAE807004FEA5B1B4FEA58384FEAD0
:104C70009919AEFB0B21AEFB0902AEFB080EACEBA3
:104C80004700049F8AF800300CEB8C0CA7EB4C0C0F
:104C900041F2A403C908D2084FEADE0E7E4F01EBB1
:104CA000810102EB82020EEB8E0EABEB4101A9EB10
:104CB0004202A8EB4E0E17F8038001F1300B3030A2
:104CC00002F130010CF1300C0EF1300201238DF8AD
:104CD00026008DF827C08DF825B08DF824108DF8AA
:104CE00023203375B8F1000F00F0D48041F2E802C0
:104CF000BA5C002A6FD041F22C130220FB5C002B1F
:104D00006AD004233375FEF7AFBFDFF8BC91DFF83C
:104D1000BC81DFF8BCA1706807AA494617F0A2FB66
:104D2000012841464FF003027EF49EAF079F3846AC
:104D3000002F3FF421AF3B78002B3FF41DAF2FF045
:104D40009FFC032251460028E5D107F108002FF00F
:104D500097FC03460028DED157F8030F08903A79F4
:104D60008DF8242008A88DF825302DF083F83369BC
:104D7000984248D83361CEE794F87D26FFF76EB8A5
:104D800094F87D2682B1022A7EF484AF18F0E0FA0E
:104D900000283EF469AF4FF480520A233A812B7009
:104DA00094F87D26FEF762BF3E4B186803685B6986
:104DB0009847EDE73B4B0592186804931CF0ECFA1A
:104DC00097F8B511049B059A1A60022928D094F827
:104DD0007D26FFF7E3B8184600EB001007EB8000D4
:104DE000314B009300F5855008A93C232022043064
:104DF00018F01CFAFEF738BF2A4B186803685B6985
:104E00009847FFF7C3B808A82DF034F80346B1E778
:104E1000334493F82830002B7EF426AFFFF7ECB82C
:104E200023F03FFED3E7134603EB031307EB8300A6
:104E300000F585501D4B0093102213231C490430AC
:104E400018F0F4F9FEF710BF4520FDF79FF8FF209A
:104E5000FDF79CF894F87D36022B6AD0114B154C67
:104E600045219846D8F8000002681268904714F867
:104E7000011F0029F6D10020FDF788F8FEF77DBF5D
:104E80002CF09EFF00283EF4EFAE7768002F7FF4F1
:104E9000B2AEC2E640469FE70C6B0020EC7C0020DF
:104EA000447C0308547D002013C7000815D3000874
:104EB0004C76030840760308CDCCCCCC1F85EB5153
:104EC000D34D62105917B7D1447D002054760308A2
:104ED000587603081E4B02705B68002B7EF4D6AE3A
:104EE000FFF753B902701B4BF6E702701A4BF3E75A
:104EF0001A4B0270F0E794F83812194808F0FCFCDD
:104F0000D7F8AC310133FFF7FCB9B4F94022B4F95A
:104F10004212144808F0F0FCD7F8AC310133FFF727
:104F2000F0B90270104BD7E70270104BD4E70223A0
:104F30007AE70F4B1868037E13F0060F9BD090F8AA
:104F40002830002B97D10A220A491FF00FFD92E763
:104F50006C7E0020607E0020547E0020487E002071
:104F60005C77030894770308847E0020787E002015
:104F70003C7D0020407603082DE9F047DFF8A4804F
:104F8000DFF8A490244E0124082088F8004029F07E
:104F90008BF8D9F8000010F06BFF052029F05AF8C3
:104FA000002029F057F8062029F054F8002029F0B5
:104FB00051F8042029F04EF8204629F04BF83388A8
:104FC0008BB1164D164F002415F804A0072029F0C8
:104FD00041F8504629F03EF82A5D33883A550134AD
:104FE000A4B2A342F0D8072029F034F8FF2029F01A
:104FF00031F8042029F02EF8002029F02BF8D9F8F8
:10500000000010F03BFF022029F04EF8002388F842
:105010000030BDE8F08700BFAA00002098260020DD
:105020002C29002096260020708700202DE9F041D1
:10503000494E082029F038F8306810F019FF474B26
:105040001B78012B78D05FD3022B0AD1DFF828819F
:10505000082388F800300D254FF4C373404F3B8080
:1050600010E0DFF814813E4F98F8003003F0400361
:10507000002B14BF4FF4F0734FF4C3733B8014BF85
:1050800010250D25002404F11000C0B228F0E2FF25
:105090000134012028F0DEFFA3B2AB42F3D398F82D
:1050A0000050304C002028F0D5FF284628F0D2FFD1
:1050B0002D4B1D78022028F0CDFF284628F0CAFF8E
:1050C0002A4B1D78032028F0C5FF284628F0C2FF90
:1050D000042028F0BFFF042028F0BCFF306810F047
:1050E000CDFE022028F0E0FF3A88214800212FF071
:1050F00020FA237E33B11F4B1B7833B30023237672
:10510000BDE8F081BDE8F081A02028F0A3FF0020D9
:1051100028F0A0FF00F00603022BDFF85C8007D028
:1051200000F00500012803D1482388F8003008E08A
:10513000082388F800308EE7DFF83C80482388F8A1
:10514000003010254FF4F07388E7FFF715FF0023B8
:105150002376BDE8F08100BF7087002074870020AF
:10516000AA00002004000020758700207687002018
:105170002C29002096260020AC000020F8B50B4C0E
:10518000074620680E46154610F072FE47F0800074
:1051900028F060FF334629460022054810F092FFB0
:1051A000206810F06BFE0120F8BD00BF9061002068
:1051B0000030014070B582B06A460621F720FFF743
:1051C000DDFF9DF801209DF804309DF800609DF8FA
:1051D00003509DF802409DF80500074912011B018C
:1051E00042EA063243EA053342EA141243EA101354
:1051F0004A600B6002B070BDC02000200148FBF780
:1052000069BF00BFC03100200148FBF763BF00BF8A
:105210006C3100200148FBF75DBF00BF1831002052
:10522000F0B5064683B00D460024012714E003299B
:105230000CBF03220122C3F3011E6946C3F381039D
:1052400030468DF805208DF806E08DF807301EF009
:10525000C3F90134102C0FD02B8807FA04F2134243
:10526000F7D0AB78E9780092022903F003028DF8B9
:105270000420DCD10A46DEE703B0F0BD70B50F4C68
:105280000F4DC0EBC00004EB800468692669304311
:10529000686182B09209667BA1600025012101A8A6
:1052A00063618DF804608DF805208DF806508DF847
:1052B000071028F0B5FC02B070BD00BF3C1D0020F7
:1052C000001002400348D0F83C3113B100F59A7049
:1052D000184770473C1D00200348D0F8203113B117
:1052E00000F58C70184770473C1D00200348D0F82B
:1052F00004310BB1FC301847704700BF3C1D002043
:105300000348D0F8E8300BB1E0301847704700BFD1
:105310003C1D00200348D0F8CC300BB1C4301847F6
:10532000704700BF3C1D00200348D0F8B0300BB1DF
:10533000A8301847704700BF3C1D00200348D0F834
:1053400094300BB18C301847704700BF3C1D0020D3
:105350000248836F0BB17030184770473C1D002026
:105360000248C36D0BB15430184770473C1D0020F4
:105370000248036C0BB13830184770473C1D0020C1
:105380000248436A0BB11C30184770473C1D00208F
:105390000248836803B11847704700BF3C1D0020D6
:1053A0001749184B184A194810B4D1F8884044F4EA
:1053B0007004C1F888401C6844F001041C605C68FB
:1053C00022405A601A6822F0847222F480321A60F5
:1053D0001A6822F480221A605A6822F4FE025A6087
:1053E000DA6A22F00F02DA621A6B002410404FF0E2
:1053F000006218639C608A605DF8044B704700BFD0
:1054000000ED00E0001002400CC07FF8CCFC00FF73
:105410002DE9F04F2DED028B8FB0834629F0CCFDA6
:105420007C4B1D7825B10FB0BDEC028BBDE8F08F31
:10543000DFF81492D9F800305F05F4D5764C94F873
:105440005C31002B40F0028194F89C31002B63D03A
:10545000D4F8A031714AABEB0303934201F272809E
:1054600094F8D871002F40F01182D4F8DC01036861
:105470005B689847C0B201280FD9022840F05E82CD
:10548000674E3378002B42F04D81D4F8E031ABEB1E
:105490000303B3F57A6F82F0D782D4F8E421002AAF
:1054A0003AD094F8D831002B40F0F581D4F8F0319F
:1054B0009B780122022B84F8D82101F2C680594939
:1054C000D4F8DC014B68984202F0B2830B69984231
:1054D00001F0D680CB69984202F0B0838B6A984283
:1054E00002F0A9834B6B984202F0AB830B6C98429D
:1054F00001F0C5800022022390F90400009301927C
:105500004FF4964308211BF071FFC4F8DC0100231F
:1055100084F8F431C4F8ECB109F0C2FC94F8F63127
:1055200063B1414E306848B1404AD4F8F831D2F8FE
:1055300000A0AAEB0303632B00F222823C4F3B78CE
:10554000022B01F05380364E96F87430032B01F095
:10555000368094F802326BB1D4F8043253B10DF0B6
:10556000D7FCD4F8083244F61F62C31A934282462D
:1055700000F2A28294F85433002B40F0608194F83A
:105580008E33002B3FF44FAFD4F8903303F5C33381
:10559000A0339B45FFF447AF94F89433254AC4F8F1
:1055A00090B302EB8302526A42B3234E0EADF31C5A
:1055B00045F8203D06F1150100230791A4F8963324
:1055C00080211523A52784F89A33284684F8991357
:1055D00084F8987390472846B4F8961311F010FB9E
:1055E000069D1648AD1B152DA8BF15252A46314628
:1055F0002CF068FC124A94F894331570114A013368
:1056000082FB0312A2EBE37202EB42029B1A84F8C4
:10561000943308E79D410020C02200203F0D030085
:1056200034000020487E0020848700204488002029
:10563000F4440020CC4F0308582600200C430020DF
:105640002143002056555555B47E0020DFF82C83A9
:10565000D4F86031D8F80020D31A7C2B7FF6F4AE52
:1056600094F86431BB4F9FEDBC8AC4F860210133CC
:1056700084F864314FF0240AD4F8680103685E218D
:105680001B689847D4F86801036851461B6898471F
:10569000B24BF7EC016A1B8907EE103AF8EEE66AA6
:1056A000B8EEC77A0AF1010AC6EE877A5FFA8AFA7B
:1056B00067EE887AFDEEE77ACDED027ABDF90860F3
:1056C000F0B229F06BFBC6F3072029F067FBBAF1B3
:1056D000270FD1D1D4F8680103685E211B68984771
:1056E000D4F86801036830211B689847D4F86C61CE
:1056F000F0B229F053FBC6F3072029F04FFBD4F892
:10570000680103685E211B68984794F8643113F0C0
:10571000030643D1D4F8602141F288339A4202F261
:105720003281D4F8680103685E211B689847D4F879
:105730006801036814211B689847894B894AB3F9AB
:10574000043082FB0312DE17C6EBA20636B2F0B2BB
:1057500029F024FBC6F3072029F020FBD4F86801C8
:1057600003685E211B689847D4F8680103681C2110
:105770001B689847D4F86801036800211B689847A4
:10578000D4F86801036800211B689847D4F86801C1
:1057900003685E211B68984794F8643113F007068C
:1057A00001F0BC81282B7FF44FAED4F86801D8F803
:1057B000008003686C4F1B6800265E2184F86461DA
:1057C0009847D4F86801036817211B689847D4F8F4
:1057D0006801036831461B689847644BA3FB0823A4
:1057E0009B0BA7FB03125209C2EB0212A3EB82032D
:1057F000D8B229F0D3FAD4F8680103685E211B6897
:105800009847D4F86801036818211B689847584BDB
:10581000A3FB08239B09A7FB03125209C2EB021248
:10582000A3EB8203D8B229F0B9FA304629F0B6FAD0
:10583000D4F8680103685E211B68984704E694F871
:105840005523002A40F05D86D4F8583303F5C3335E
:10585000A0339B45FFF493AE94F85C53C4F858B35F
:10586000631993F86063F30701F10485B70701F149
:105870002782760700F14C8794F88D23013595FB3C
:10588000F2F302FB135584F85C5378E6D4F8E42174
:10589000002A3FF441AED4F8EC3140F6B731ABEB1F
:1058A00003038B427FF638AE94F8E831002B40F0CA
:1058B000B086D4F8F021C4F8E431927884F8D83175
:1058C000022A01F2FC802B49D4F8DC21486882428C
:1058D00001F00A810B699A4202F0BA81CB699A42BF
:1058E00002F0AC828B6A9A4202F0A5824B6B9A421C
:1058F00002F09E820B6C9A4201F0F58092F904004E
:1059000001230022009301924FF4964308211BF0DB
:105910006DFDC4F8DC0106E0D4F8DC010368DB6847
:105920009847D4F8DC0103685B6898470028F3D1F6
:10593000F0E5D4F8DC010368DB689847D4F8DC01B3
:1059400003685B6898470028F3D10B4E012333703E
:10595000A3E500BFBC89002000007A448C890020A8
:10596000D0600020676666668988888873B2E745DC
:10597000D34D6210487E002034000020448800206F
:10598000494F00233B70036824211B689847306807
:10599000036854211B6898473068036841211B68DD
:1059A0009847424B424AB3F90230306882FB0312F7
:1059B0004FEAE378C8EBA2080FFA88F802685FFAAA
:1059C00088F319461268029390473A78029B306830
:1059D00053403B700368C8F3072841461B6898474B
:1059E0003A78324B3068B3F9003088EA0208304A1E
:1059F00087F8008082FB0312DB17C3EBA2080FFAC3
:105A000088F802685FFA88F3194612680293904793
:105A10003A78029B306853403B700368C8F307280C
:105A200041461B689847214B3A78B3F90430204926
:105A3000306881FB03E188EA0208DB1787F8008001
:105A4000C3EBA1030FFA83F803685FFA88F21146EB
:105A50001B6802929847029A3B78306853403B702B
:105A60000368C8F307281B684146984739783068AF
:105A700088EA0101397003681B68984794F8FC3183
:105A800013F0010200F03A870A4AC4F8F8A1013382
:105A9000DBB2A2FB0312D20802EB8202A3EB4203A9
:105AA00084F8FC314AE500BF5A880020D06000200D
:105AB00067666666CDCCCCCC94F80E32002B40F0F5
:105AC000D985D34B1B6803F00802002A48F603412E
:105AD0004AF60B404BF60F4249F6074504BF024613
:105AE0000D4613F0040F4FF0190118BF15469F061D
:105AF00084F80E1203D545F4804545F02005D9F809
:105B0000003013F00206C5F3090741F01E874FF07D
:105B1000FF3864204FF0000E06950795ADF826601B
:105B20000897ADF828808DF83600ADF824E0CDF860
:105B30002AE0CDF82EE0CDF832E006AE0FCEB54D1E
:105B400084F82DE00FC596E80F0007C525F8023B45
:105B5000294601261B0CFE251F20C82201F81E39EC
:105B600084F82A5084F82B0084F82F6084F82E20C3
:105B700094F81E2284F82C2082F0F10383EA0313A8
:105B8000D8B2030983F0E70343EA002383EAC003A2
:105B90001BB283EA0310C0B2C3F3072383EA1013D6
:105BA00043EA002383EAC0031BB283F0C80080EA03
:105BB0000010C0B2C3F3072383EA101343EA0023A3
:105BC00083EAC0031BB283EA060585EA0515EDB238
:105BD000C3F3072383EA151343EA0523324483EA18
:105BE000C50584F81E22258501F11F0011F8013B2F
:105BF0006B4083EA0313DBB21A0982EA152242EAF8
:105C0000032282EAC3031BB29DB281422585EDD1F6
:105C100083F07C0181EA0111C9B20B0983EA1523E3
:105C200083EA012383EAC1031BB29AB24FEA122E20
:105C3000DFB2DFF8F8C1228584F850E084F84F70B5
:105C400004F12A0504F14A0828686968AA68EB6823
:105C500066460FC610354545B446F5D12868306014
:105C60006D4E2B798CF8043006F1270584F86D729F
:105C700084F86EE2D4F8040216F8011F03681B686A
:105C80009847B542F6D194F80F22002A40F0EE84EE
:105C90006249634B09781B680A2084F80F020029C7
:105CA00000F017875F4D01292888049042F2D180C7
:105CB00068880290022901F0F0860329B5F804E013
:105CC00002F0D280E8880390042902F0D7800529E9
:105CD000288902F0CF8006296F8902F0C280072947
:105CE000AE8900D0EA8994F81E52069385F03003FD
:105CF00083EA0313DBB24FEA13184B4984F82C50A4
:105D000088F07A08098848EA032888EAC303DFF89C
:105D10002081C1EB012188FB01C888444FF0000CB1
:105D2000C917C1EB68216EF30F0C4FF0000E0591FF
:105D30001BB2049960F30F0E002066F30F004FF0C2
:105D4000000883EA0316C3F3072361F30F0819461B
:105D5000029B63F31F48039BCDF81C80F6B263F3EC
:105D60001F4C67F31F4E62F31F4000279DF814205D
:105D7000CDF820C0CDF824E08DF82C7081EA161300
:105D80008DF82D200A900DF1180C43EA062EBCE880
:105D90000F008EEAC60636B286F0C808DFF874E057
:105DA00084F82D7088EA0817AEE80F00FFB2C6F33A
:105DB000072686EA17139CE8030043EA072383EAD1
:105DC000C7031BB24EF8040B83F0230686EA0616BF
:105DD000F6B27046C3F3072282EA161242EA06229E
:105DE00020F8141982EAC606013516224FF0230E58
:105DF000FE27C82384F81E52268584F82FE084F8F5
:105E00002A70811884F82B2084F82E3012E000BF0D
:105E1000248A0020F022002007250020608800202E
:105E20004488002074880020A44500200825002014
:105E30000308208010F8013B734083EA0313DBB2B0
:105E40001A0982EA162242EA032282EAC3031BB23B
:105E50009EB288422685EDD183F0F40181EA0111DA
:105E6000C9B20B0983EA162383EA012383EAC1033B
:105E700026461BB21FFA83FC56F82A0FCC4DA4F815
:105E800028C0DFB24FEA1C2E84F8467084F847E041
:105E90007168B268F3680FC530697169B26904F25C
:105EA000472607C504F2652584F865E284F8647224
:105EB000D4F8040216F8011F03681B689847B5421E
:105EC000F6D194F81662002E40F0CC83B94B94F8CA
:105ED0001E72B3F90010B3F90220B3F904309FED3C
:105EE000B66A84F82D6007EE103AB44B1B6806932F
:105EF00087F06A0383EA031306EE901AD9B20B09FE
:105F000083F0D50343EA012383EAC1031BB283EA8A
:105F100003115242C9B207EE902AC3F3072383EA62
:105F2000111343EA0123F8EEE77AF8EEE66AB8EED9
:105F3000C77A83EAC1031BB267EE867A66EE866A89
:105F400027EE067A002083F0C805CDED087ACDED66
:105F5000076A8DED097A0A900B900C9085EA051E70
:105F60000DF1180C5FFA8EFEC3F30725BCE80F0095
:105F700085EA1E1545EA0E2585EACE05DFF858E2CA
:105F80002DB2AEE80F0085F01E069CE8070086EAF9
:105F90000613DBB2C5F3072686EA131646EA032684
:105FA0008EE8070086EAC3061C21AEF110054FF00B
:105FB00005084FF01E0CFE20C8227B1C84F82B1015
:105FC00084F8168284F82FC084F82A0084F82E20E2
:105FD000691884F82C70268584F81E3215F8013B68
:105FE000734083EA0313DBB21A0982EA162242EAFB
:105FF000032282EAC3031BB29EB28D422685EDD1F5
:1060000083F0270383EA0313DBB21A0982EA16221C
:1060100082EA032282EAC3031BB29AB24FEA122E2B
:10602000DFB2DFF88CC1228584F84DE084F84C7033
:1060300004F12A0504F14A0828686968AA68EB682F
:1060400066460FC610354545B446F5D15C4E2B88E3
:10605000ACF8003006F1240584F86A7284F86BE22B
:10606000D4F8040216F8011F03681B689847B5426C
:10607000F6D194F81782B8F1000F40F0EE82514B40
:106080001B68052213F0140F84F8172240F00485D2
:10609000DFED4D7A94F81EE2464B4C4AB3F90410FA
:1060A000B2F906204A4D4B48CDED087A8EF0220316
:1060B00083EA0313DEB2B2F5FA6F4FEA1613A8BFF4
:1060C0004FF4FA6283F0590343EA0623B2F57A7F6C
:1060D00083EAC603B8BF4FF47A721BB26427A2F5F5
:1060E0007A7283EA031607FB02F285FB0257F6B2C7
:1060F00080FB0150C3F30723D217C9174FF0000CE0
:1061000083EA1613C2EBA712C1EBA00143EA0625EE
:10611000CDF818C0CDF81CC0CDF824C0ADF82A20A9
:10612000ADF828100DF1180CBCE80F0085EAC60583
:106130002DB285F0C80686EA0616274FDCF800C0A7
:1061400084F82CE0F6B2C5F307250FC785EA1615CB
:1061500045EA062585EAC6031BB283F04A0585EAAF
:106160000511C3F307223B46C9B243F810C982EABE
:10617000111242EA01220EF1010E184682EAC1050F
:10618000029314224FF04A0CFE26002384F81EE2EC
:106190004FF0C80E01462585104484F82FC084F8BE
:1061A0002A6084F82B2084F82D3084F82EE015E046
:1061B00008250020D060002088C3E43A44880020ED
:1061C00007250020248A0020000000007488002099
:1061D000D34D621067666666F022002011F8013B1D
:1061E0006B4083EA0313DBB21A0982EA152242EA02
:1061F000032282EAC3031BB29DB281422585EDD101
:1062000083F0140383EA0313DBB24FEA131E8EEA12
:10621000152E8EEA032E8EEAC30E25460FFA8EFE49
:106220001FFA8EF755F82A0FBE4E27854FEA172C16
:106230005FFA8EFE84F844E084F845C06968EB6834
:10624000AA680FC6286969692B8B03C604F2472523
:10625000338004F263272E4684F863C284F862E236
:10626000D4F8040216F8011F03681B689847B74268
:10627000F6D1AD4BAD4A93F8B3321278013B12F030
:106280000400DBB214BFC0224022172B03D8A84958
:106290000B4493F80C80A74B19888E071ABF002374
:1062A00042F01002012311F4027F18BF022311F003
:1062B000100F18BF062311F0200F18BF102300285D
:1062C00041F0BA83032194F81EE206938EF0460350
:1062D00083EA0313D8B2030983F0920343EA00234D
:1062E00083EAC0031BB283EA0310C0B2C3F30723DF
:1062F00083EA101343EA002383EAC0031BB283F04E
:10630000C80686EA0616F6B2C3F3072C032000235C
:106310008DF81C808DF81E208DF81D308DF81F1013
:106320008DF820008CEA161C06AA07CA4CEA062C37
:106330008CEAC60636B2029F84F82F3086EA061C25
:1063400003C75FFA8CFCC6F3072181EA1C1141EAFE
:106350000C2181EACC0194F830C03A700AB28CEA80
:10636000020181EA0111C9B2C2F3072282EA1112C5
:1063700042EA012294F8316094F8320094F833C074
:1063800094F8347084F82D3082EAC10212B256407B
:1063900086EA0616F6B2C2F3072282EA161242EA2B
:1063A000062282EAC60212B2504080EA0010C0B251
:1063B000C2F3072282EA101242EA002282EAC002F5
:1063C00012B28CEA020C8CEA0C1C5FFA8CFCC2F351
:1063D000072282EA1C1242EA0C2282EACC0212B2A2
:1063E000574087EA0717FFB2C2F3072282EA171263
:1063F00042EA072294F8356094F8360094F8371092
:1064000094F838C084F82CE082EAC70212B25640F1
:1064100086EA0616F6B2C2F3072282EA161242EAAA
:10642000062282EAC60212B2504080EA0010C0B2D0
:10643000C2F3072282EA101242EA002282EAC00274
:1064400012B2514081EA0111C9B2C2F3072282EAB5
:10645000111242EA012282EAC10213B28CEA03025B
:1064600082EA0212D2B2C3F3072383EA121343EA89
:10647000022383EAC2031BB283F0320282EA0212D1
:10648000D2B2C3F3072383EA121343EA022383EA57
:10649000C2031BB2284E9AB20EF101014FF0FE0862
:1064A0004FEA122E0927C820DBB284F82A8084F82C
:1064B0002B7084F82E0084F81E12228584F83AE0AE
:1064C00084F8393030687168B268B6F80C8006F22A
:1064D0001E2707C706F22E2687F802C0A7F80080FD
:1064E00084F858E284F85732D4F8040215F8011FF2
:1064F00003681B689847AE42F6D1C4F808A2FFF7BC
:1065000039B80E4B1D682B68DF691646002F00F066
:10651000D98028460A49B847002384F85533FFF745
:1065200093B900BF08250020946100201B8E002035
:10653000CC4F0308C0600020EA220020848900209C
:10654000F8230020684BD4F8D4111B886748D4F88E
:10655000D021DEB21B0A84F8C33184F8B93184F843
:10656000C26184F8B8610E7C01684FF47A738A1AAC
:1065700003FB06F300219A4284F8A61184F8A811BF
:1065800080F088805A4A5B481168D4F89821C4F892
:10659000A0B180FB013680FB0230C917D317C3EBD3
:1065A000A003C1EBA6021012191284F8C42184F8CA
:1065B000C50184F8C03184F8C111FEF751BFDFF87E
:1065C0004C81D8F8000003685B69984700283EF4C6
:1065D000C0AFD8F80000036801219B6998470222E8
:1065E000002386F874203B70FEF7B3BF0CF090FCDC
:1065F000414B1B68C01A40F6B833984200F25682ED
:106600003E4B1A793A2A01F0928000233B70FEF744
:10661000A0BF013BDBB284F8E831D4F8DC01002BE9
:1066200001F0718012F8011B94F8F46194F8F531CF
:106630000768C4F8E42101338A193F6884F8F4211B
:1066400084F8F531B847FEF765BFD4F8DC0103687C
:1066500002219B699847FEF75ABF08F1FF3884F87A
:1066600017824AE7013E84F8166202E5013A84F88F
:106670000F2226E4013B84F80E32FFF704BB05220B
:1066800002EB420201EB82030022C2621A815A60CD
:10669000FEF730BF1A4A03681278C4F8D031032AD3
:1066A0003FF470AF174B1B78934238BF1346013B42
:1066B000012B3FF667AF1022022384F8A62184F84D
:1066C000A8315FE7104F00E02B689B682846984789
:1066D0000028F9D02B6817F8011B1B68284698473B
:1066E000013EF1D118E700BF344500204488002066
:1066F0003045002067666666FC440020E4440020C4
:106700003645002037450020F8230020408900202E
:10671000744B1A6821200023712184F86A03D00089
:1067200084F8683384F8693384F88C1341F11C8150
:106730006D484FF0030E6D4B1B88590501F1FD802C
:10674000DA0701F1A18103F00203694A002B1CBFA3
:106750004FF0030E1046DFF8A0C1013866467123E2
:1067600000216FF02A0710F8012F06F8012B534083
:106770005A0013F0800F82F0D508D2B25FFA88F881
:1067800008BF90464FEA480282F0D50318F0800F08
:106790005FFA83F8D3B218BF43465A0013F0800F54
:1067A00082F0D508D2B25FFA88F808BF90464FEA67
:1067B000480318F0800F83F0D502DBB2D2B208BFD5
:1067C0001A46530012F0800F83F0D508DBB25FFA4F
:1067D00088F808BF98464FEA480282F0D50318F0BF
:1067E000800F5FFA83F8D3B218BF43464FEA4308DD
:1067F00013F0800F88F0D5025FFA88F8D2B208BF94
:106800004246530083F0D50812F0800F01F10101D8
:106810005FFA88F2DBB218BF13468E45A3DC5A003C
:1068200082EA070113F0800FC9B2D3B218BF0B463A
:10683000590081EA070213F0800FC9B2D3B208BF32
:106840000B46590081EA070213F0800FC9B2D2B299
:1068500008BF0A46530083EA070112F0800FDBB23B
:10686000CAB208BF1A46530083EA070112F0800F2C
:10687000DBB2CAB208BF1A46530083EA070112F01E
:10688000800FDBB2CAB208BF1A46530083EA070181
:1068900012F0800FDBB2CAB208BF1A460CEB0E062C
:1068A0001449500080EA0703B71C7F1A12F0800FCA
:1068B000C0B2DBB208BF0346242FA8BF2427A6EB33
:1068C000010800220CF80E20A1F50C7084F86983F1
:1068D0003A46737084F88C332BF0F4FA84F85573CD
:1068E000FEF7CABF148E00200C750308C06000209C
:1068F0001C750308282600202B2600207F4B1B88B0
:10690000D80501F11F80D90601F1C3809A0601F173
:106910008B81580601F19881190701F19C81DA07F2
:1069200001F1938213F0020F0CBF04230C23029396
:10693000734A744B1278DB78C2F380020BB142F0D9
:106940000202306804924FF000033B700368242178
:106950001B6898473068036854211B689847306863
:10696000036853211B689847674B30681B88016890
:1069700003EB830303EB83034FEA83081FFA88F8D2
:106980005FFA88F31A460B68039211469847039AF8
:106990003B78306853403B7003684FEA1828414603
:1069A0001B6898473B78306888EA030887F80080BE
:1069B000036800211B6898473068036800211B6842
:1069C0009847524B52491B883068C3EBC3135B0096
:1069D00081FB032119444FEAE378C8EB612803687F
:1069E0005FFA88F841461B6898473B78306888EA28
:1069F000030887F80080036800211B689847029A03
:106A000030681146049A036841EA02081B6841464F
:106A100098473A78306888EA0202D1B23970036840
:106A20001B68984794F8FC31002B7FF42DA8306840
:106A30003B70036824211B68984730680368542121
:106A40001B689847306803684F211B68984724F0FB
:106A50008FFE24F08DFE24F08BFE30680368012148
:106A60001B6898473B782B4A306892F8008083F087
:106A700001033B70036808F001081B684146984712
:106A80003978306888EA0101397003681B689847D3
:106A900094F8FC31FEF7F8BFD4EDD47A9FED1E7A5E
:106AA000F8EEE77A67EE877AFFF7F4BAB4F8FE31CA
:106AB00000220133A4F8FE313A70FEF74ABDD4F843
:106AC000DC01036801219B699847D4F8DC01FEF7DB
:106AD0002ABF0E460F46084603918E460291049146
:106AE0000A46FFF700B9052303EB430301EB8303D9
:106AF0000021D16219815960FEF700BFC0600020FB
:106B00001B8E00201C8E002034450020A445002050
:106B1000030820804A8E00200AD7233CD4F868015D
:106B200003685E211B689847D4F868010368022156
:106B30001B68984724F03AFE0378FF2B01F06D8024
:106B400090F90130DE17F6B2D8B228F027F93046B6
:106B500028F024F9D4F8680103685E211B6898477F
:106B6000D4F86801036803211B68984724F01EFECF
:106B70000378FF2B01F05480B0F90830D8B2C3F38A
:106B8000072628F00BF9304628F008F94A4AD9F8C8
:106B900000301A4204D0494F3B78002B40F08487E4
:106BA000D4F89431D4F868011A7B0368002A1B6872
:106BB0004FF05E0114BF3C2664269847D4F8680164
:106BC000036813211B689847304628F0E7F8002037
:106BD00028F0E4F8D4F8680103685E211B68984740
:106BE000D4F8680103681B211B689847002028F02F
:106BF000D5F8002028F0D2F8D4F8680103685E21A7
:106C00001B689847D4F86801036823211B689847DC
:106C10004E2028F0C3F8D4F86801036800211B68EF
:106C20009847D4F89431D4F868011A7B0368002A95
:106C30001B684FF05E0114BF3C2664269847D4F8C9
:106C40006801036812211B689847304628F0A6F8AF
:106C5000002028F0A3F8D4F8680103685E211B68BF
:106C60009847D4F8680103681A211B6898470020E8
:106C700028F094F8002028F091F8D4F8680103680F
:106C80005E211B689847D4F86801036822211B68BD
:106C90009847452028F082F8D4F86801036800215D
:106CA0001B689847D4F8680103685E211B68984701
:106CB00094F86431FEF776BD02000008B87E00202B
:106CC000DA4BD4F898211988D94F080A80F0290E98
:106CD0004FEA4E031EF0800F83F0D50EDBB25FFA51
:106CE0008EFE08BF9E464FEA4E031EF0800F83F0D3
:106CF000D50EDBB25FFA8EFE08BF9E464FEA4E030A
:106D00001EF0800F83F0D50EDBB25FFA8EFE08BF57
:106D10009E464FEA4E031EF0800F83F0D50EDBB285
:106D20005FFA8EFE08BF9E464FEA4E031EF0800FAC
:106D300083F0D50EDBB25FFA8EFE08BF9E464FEAA7
:106D40004E031EF0800F83F0D50EDBB25FFA8EFE8D
:106D500008BF9E464FEA4E031EF0800F83F0D50E0B
:106D60005FFA8EFEDBB218BF73464FEA430E13F094
:106D7000800F8EF0D5035FFA8EFEC9B2DBB208BF7A
:106D800073464B404FEA430E13F0800F8EF0D5034D
:106D9000DBB25FFA8EFE18BF9E464FEA4E031EF02E
:106DA000800F83F0D50EDBB25FFA8EFE08BF9E46E1
:106DB0004FEA4E031EF0800F83F0D50EDBB25FFA70
:106DC0008EFE08BF9E464FEA4E031EF0800F83F0F2
:106DD000D50EDBB25FFA8EFE08BF9E464FEA4E0329
:106DE0001EF0800F83F0D50EDBB25FFA8EFE08BF77
:106DF0009E464FEA4E031EF0800F83F0D50EDBB2A5
:106E00005FFA8EFE08BF9E464FEA4E031EF0800FCB
:106E100083F0D50E5FFA8EFEDBB218BF734613F017
:106E2000800F87FB02E74FEA43034FEAE272C2EBAF
:106E3000A70283F0D507FFB2C2F3072EDBB218BF5B
:106E40003B468EEA03035F0013F0800F87F0D50303
:106E5000DBB2FFB218BF1F467B0017F0800F83F034
:106E6000D507DBB2FFB208BF1F467B0017F0800FCB
:106E700083F0D507DBB2FFB208BF1F467B0017F0D7
:106E8000800F83F0D507DBB2FFB208BF1F467B003F
:106E900017F0800F83F0D507DBB2FFB208BF1F46A3
:106EA0007B0017F0800F83F0D507DBB2FFB208BF7D
:106EB0001F467B0017F0800F83F0D507FFB2DBB2CF
:106EC00018BF3B465F0013F0800F87F0D503FFB279
:106ED000D2B2DBB208BF3B4653405F0013F0800FD5
:106EE00087F0D503DBB2FFB218BF1F467B0017F057
:106EF000800F83F0D507DBB2FFB208BF1F467B00CF
:106F000017F0800F83F0D507DBB2FFB208BF1F4632
:106F10007B0017F0800F83F0D507DBB2FFB208BF0C
:106F20001F467B0017F0800F83F0D507DBB2FFB25E
:106F300008BF1F467B0017F0800F83F0D507DBB238
:106F4000FFB208BF1F467B0017F0800F83F0D50704
:106F5000FFB2DBB218BF3B4613F0800F4FEA430786
:106F6000344B84F86B03186884F86C1387F0D503EE
:106F7000D9B2FBB214BF8A469A460A2108230027D9
:106F8000B0F80E8084F86DE384F86E2384F86913FA
:106F900084F86A3384F88CA384F8687318F07AF85C
:106FA0004FEA4A031AF0800F83F0D502DBB2D2B267
:106FB00008BF1A46530012F0800F83F0D502DBB2EF
:106FC000D2B208BF1A46530012F0800F83F0D502E8
:106FD000DBB2D2B208BF1A46530012F0800F83F022
:106FE000D502DBB2D2B208BF1A46530012F0800FAE
:106FF00083F0D502DBB2D2B208BF1A46530012F0BA
:10700000800F83F0D502DBB2D2B208BF1A4653001C
:1070100012F0800F83F0D502D2B2DBB218BF134654
:107020005A0013F0800F82F0D50305E034450020AC
:10703000676666662C450020D2B24FEA1821DBB2A3
:1070400008BF13464B405A0013F0800F82F0D5035F
:10705000DBB2D2B218BF1A46530012F0800F83F091
:10706000D502DBB2D2B208BF1A46530012F0800F2D
:1070700083F0D502DBB2D2B208BF1A46530012F039
:10708000800F83F0D502DBB2D2B208BF1A4653009C
:1070900012F0800F83F0D502DBB2D2B208BF1A46DD
:1070A000530012F0800F83F0D502DBB2D2B208BFDA
:1070B0001A46530012F0800F83F0D502D2B2DBB231
:1070C00018BF13465A0013F0800F5FFA82FE82F059
:1070D000D503DBB25FFA88F208BF734653404FEA2C
:1070E000430E13F0800F8EF0D503DBB25FFA8EFEF5
:1070F00018BF9E464FEA4E031EF0800F83F0D50E58
:10710000DBB25FFA8EFE08BF9E464FEA4E031EF0CA
:10711000800F83F0D50EDBB25FFA8EFE08BF9E466D
:107120004FEA4E031EF0800F83F0D50EDBB25FFAFC
:107130008EFE08BF9E464FEA4E031EF0800F83F07E
:10714000D50EDBB25FFA8EFE08BF9E464FEA4E03B5
:107150001EF0800F83F0D50EDBB25FFA8EFE08BF03
:107160009E464FEA4E031EF0800F83F0D50E5FFA65
:107170008EFEDBB218BF73464FEA430E13F0800F4A
:107180008EF0D5035FFA8EFEDBB208BF7346434034
:107190004FEA430E13F0800F8EF0D503DBB25FFA97
:1071A0008EFE18BF9E464FEA4E031EF0800F83F0FE
:1071B000D50EDBB25FFA8EFE08BF9E464FEA4E0345
:1071C0001EF0800F83F0D50EDBB25FFA8EFE08BF93
:1071D0009E464FEA4E031EF0800F83F0D50EDBB2C1
:1071E0005FFA8EFE08BF9E464FEA4E031EF0800FE8
:1071F00083F0D50EDBB25FFA8EFE08BF9E464FEAE3
:107200004E031EF0800F83F0D50EDBB25FFA8EFEC8
:1072100008BF9E464FEA4E031EF0800F83F0D50E46
:107220005FFA8EFEDBB218BF73464FEA430E13F0CF
:10723000800F8EF0D503DBB25FFA8EFE18BF9E463C
:107240000B4B84F8712384F86F7303F50C7284F888
:10725000720384F8701384F873E307CA83E80700A5
:107260000C2384F88CE384F85533FEF702BB00BF8F
:10727000F8230020D94B9FEDDA6AB3F9022006EE1D
:10728000902AF8EEE66AB3F90020B3F9043066EE0E
:10729000866A07EE102AFDEEE66A07EE903ACDED1B
:1072A000026ABDF90800C0F3072C8CF0FA02530003
:1072B00012F0800F83F0D502DBB2D2B208BF1A46BB
:1072C000530012F0800F83F0D502DBB2D2B208BFB8
:1072D0001A46530012F0800F83F0D502DBB2D2B20F
:1072E00008BF1A46530012F0800F83F0D502DBB2BC
:1072F000D2B208BF1A46530012F0800F83F0D502B5
:10730000DBB2D2B208BF1A46530012F0800F83F0EE
:10731000D502DBB2D2B208BF1A46530012F0800F7A
:1073200083F0D502D2B2DBB218BF13465A0013F075
:10733000800F82F0D503D2B2C0B2DBB208BF1346D1
:1073400043405A0013F0800F82F0D503DBB2D2B273
:1073500018BF1A46530012F0800F83F0D502DBB23B
:10736000D2B208BF1A46530012F0800F83F0D50244
:10737000DBB2D2B208BF1A46530012F0800F83F07E
:10738000D502DBB2D2B208BF1A46530012F0800F0A
:1073900083F0D502DBB2D2B208BF1A465300B8EE72
:1073A000C77A12F0800F83F0D502DBB2D2B227EE9B
:1073B000067A08BF1A46530012F0800FBDEEC77A56
:1073C00083F0D502D2B2DBB28DED037A18BF13463B
:1073D0005A00BDF90C1084F86BC313F0800F82F0D3
:1073E000D503D2B2C1F3072EDBB208BF13468EEA33
:1073F000030313F0800F4FEA430383F0D502D2B2A8
:10740000DBB218BF134613F0800F4FEA430383F03B
:10741000D502D2B2DBB218BF134613F0800F4FEA89
:10742000430383F0D502D2B2DBB218BF134613F088
:10743000800F4FEA430383F0D502D2B2DBB218BF0C
:10744000134613F0800F4FEA430383F0D502D2B204
:10745000DBB218BF134613F0800F4FEA430383F0EB
:10746000D502D2B2DBB218BF134613F0800F4FEA39
:10747000430383F0D502D2B2DBB218BF134613F038
:10748000800F4FEA430383F0D502D2B2C9B2DBB218
:1074900018BF13464B4013F0800F4FEA430383F0AD
:1074A000D502D2B2DBB218BF134613F0800F4FEAF9
:1074B000430383F0D502D2B2DBB218BF134613F0F8
:1074C000800F4FEA430383F0D502D2B2DBB218BF7C
:1074D000134613F0800F4FEA430383F0D502D2B274
:1074E000DBB218BF134613F0800F4FEA430383F05B
:1074F000D502D2B2DBB218BF134613F0800F4FEAA9
:10750000430383F0D502D2B2DBB2F8EEE77A18BFBC
:1075100013465A0013F0800F67EE867A82F0D50387
:10752000DFB2FDEEE77AD3B218BF3B465A0013F044
:10753000800FCDED027A82F0D503D2B2DBB208BF64
:107540001346BDF9082084F86C03C2F307277B407B
:1075500013F0800F4FEA430383F0D5085FFA88F8F1
:10756000DBB218BF434613F0800F4FEA430383F0AA
:10757000D5085FFA88F8DBB218BF434613F0800FD6
:107580004FEA430383F0D5085FFA88F8DBB218BFEF
:10759000434613F0800F4FEA430383F0D5085FFAA8
:1075A00088F8DBB218BF434613F0800F4FEA43035D
:1075B00083F0D5085FFA88F8DBB218BF434613F0B2
:1075C000800F4FEA430383F0D5085FFA88F8DBB2F7
:1075D00018BF434613F0800F04E000BFD0600020C6
:1075E00058A08B414FEA430383F0D5085FFA88FA2D
:1075F0005FFA83F818BFD04618F0800F4FEA4808AA
:1076000088F0D5035FFA88F8D2B2DBB208BF4346F0
:10761000534013F0800F4FEA430383F0D5085FFA1D
:1076200088F8DBB218BF434613F0800F4FEA4303DC
:1076300083F0D5085FFA88F8DBB218BF434613F031
:10764000800F4FEA430383F0D5085FFA88F8DBB276
:1076500018BF434613F0800F4FEA430383F0D50869
:107660005FFA88F8DBB218BF434613F0800F4FEA89
:10767000430383F0D5085FFA88F8DBB218BF4346AE
:1076800013F0800F4FEA430383F0D5085FFA88F8C0
:10769000DBB218BF434613F0800F4FEA430383F079
:1076A000D5085FFA88F8DBB218BF434613F0800FA5
:1076B0004FEA430383F0D50CDBB25FFA8CFC84F80D
:1076C0006DE308BF9C4684F86E1308201E21CD4B45
:1076D00084F86F734FF0000E84F8702384F871C340
:1076E00084F868E384F8690384F86A1393E8070070
:1076F000A3F50C7303C30A2184F88CC31A8084F8A1
:107700005513FEF7B3B894F8F41194F8F531026804
:107710004E1C0133126884F8F46184F8F531904707
:10772000FDF7F8BEC4F8E0B13770FDF7B6BE9A7841
:10773000E2B102F1FF3E5FFA8EFE0EF1010E9E44B1
:107740001E46002116F8012B4A4082EA0212D2B2EC
:10775000090A4FEAC20C41EA0221B6458CEA12122C
:1077600081EA0201EED100297EF44FAFDFF8C0823A
:10777000A549A64EA64AD8F800E00968DEF830C050
:107780001288F164D4F89811F261F162D4F888217A
:10779000B4F8FE11F066F263F165BCF1000F00F081
:1077A0002283DEF84020DCF8041091423BBFDEF873
:1077B0000C008A1AA1EB020A02EB000ABAF1000FD0
:1077C0007DF4C2AEDEF80020029392697046022179
:1077D0009047029B94F80022DB780393642A4FF0D1
:1077E000040386F8743040F04D8294F80132072B80
:1077F00008BF84F801A294F80132029306EB031A41
:10780000DAF804100491084628F0D6F8DAF80830BF
:1078100005935FFA80FA184628F0CEF8C2B2029BB0
:1078200004991046049000EBCA005244A07323F060
:107830000F000832A07203F00F00E271607352462D
:1078400074482AF03FFB059B049A1946724B0AF1D3
:10785000090018442AF036FBE27902F1010AD2B19C
:10786000013A5FFA82FC6C4A6C4B0CF1080C02F195
:10787000010EA44400221EF8010B50408200C108F2
:1078800082EA400201F01801424043FA01F14A4005
:10789000F445D2B2EFD1604B03F80A20E2799DF8AB
:1078A0000C30E37002F03F02911C02F10A0E61718C
:1078B00084F802E05A4C0832A11820464FF0000C20
:1078C00010F8013B83EA0C0383EA0313DBB24FEAAF
:1078D0001C224FEAC30C42EA03228CEA13135A40DB
:1078E00012B288421FFA82FCEAD1A644029B0EF82B
:1078F000022CA27822444FEA1C2C0133002184F888
:10790000013202F801CC84F80012A37853B1D8F800
:107910000000615D03681B6898470135A378EDB2EC
:10792000AB42F4D894F800320322013384F80032D9
:1079300086F874203A70FEF744BE4FF0030E3948C3
:10794000FEF709BF0292FEF7F3BF314BB4F99881FD
:107950001B8803EB830303EB83039E0017F09AFB62
:10796000B6B240B2FEF7D6B8D9F800302E4A2F484A
:1079700003F48003002B0ABF10464FF0030E4FF0B4
:10798000040EFEF7D8BED4F86801DFF8A8A003689B
:107990005E211B689847D4F86801036810211B68B2
:1079A0009847D4F888318AFB0327DB17C3EB6717A6
:1079B000F8B227F0F3F9C7F3072027F0EFF9D4F86E
:1079C000680103685E211B689847D4F86801036862
:1079D00021211B689847D4F888318AFB0312D817F5
:1079E000C0EB6210642202FB103383EAE370A0EB69
:1079F000E370C0B227F0D2F9304627F0CFF9FDF797
:107A000090BE00BF28260020304500203400002012
:107A100034450020CF220020C62200200007090E96
:107A2000C022002010750308047503080C750308B4
:107A3000408900201F85EB518949C97800290CBF76
:107A400004210521FEF73FBCD4F8DC0103680122C4
:107A5000DB68327098470646D4F8DC010368DB68BF
:107A6000984776067DF419AD8E287DF416AD94F80E
:107A7000D831002B7DF40AAF7A4BC4F8E4312D23C2
:107A800084F8E831FDF712BD4FF0040E7648FEF79A
:107A900062BE34230293FEF74BBF164617461046CC
:107AA00003929646FEF71FB9DFF8D4A1B4F89061AF
:107AB000D4F86801BAF800106422360102FB0131E3
:107AC000B6B202685B00B1FBF3F346EA0326126824
:107AD000C3F303235E21B6B21E439047D4F8680176
:107AE000036806211B689847F0B227F057F9300A5F
:107AF00027F054F9B4F89031D4F894013A78867BA1
:107B000001339BB2012E93FBF2F102FB1133A4F877
:107B1000903100F07681BAF800605449C07B6E2342
:107B200003FB06F381FB0361DB17C3EBA10310B179
:107B30009BB293FBF2F3D4F868014D4E02685E21CC
:107B400012689FB29047D4F8680103683A211B6815
:107B50009847A6FB073676091FFA86FA5FFA8AF07D
:107B600027F01CF94FEA1A2027F018F9D4F8680119
:107B700003685E211B689847D4F8680103683B21BD
:107B80001B689847642303FB16739BB2394805337F
:107B900080FB0320DB17C3EBA000C0B227F0FEF888
:107BA000002027F0FBF8D4F8680103685E211B6809
:107BB0009847D4F86801036828211B6898472D4A24
:107BC000D4F89831DE1782FB0323C6EBA306F0B28C
:107BD00027F0E4F8C6F3072027F0E0F8D4F86801AE
:107BE00003685E211B689847D4F868010368042184
:107BF0001B689847204B1B68DB89002B40F00D81E8
:107C00001E4B1E6886F31006F0B227F0C7F8C6F3C5
:107C1000072027F0C3F8FEF7C3BF3046FEF795BF35
:107C200000263046FEF7ADBF24230293FEF780BE48
:107C30000022FEF725BD0322FEF722BD0222FEF739
:107C40001FBD0422FEF71CBD10230293FEF770BE79
:107C50000123FEF749BF20230293FEF769BE00BF50
:107C60001C8E00206424002014750308310CC330DE
:107C70001F85EB51676666662C4500203045002065
:107C80003445002096F875200295130704BF013291
:107C9000D2B2072A28BF01224FEA021A06EB0A03D2
:107CA000002093F810E0784BA07213F80E105FFAE2
:107CB0008AF39C46754B06EB0A004CEA0E0E01292E
:107CC00083F800E0C06803F101050DD90239C9B29B
:107CD00001F1020E9E442B4603F8010B73454FEA57
:107CE0001020F9D101310D44B24401329AF811103B
:107CF00020F06003D2B20B43082A2B7005F1010378
:107D000000F09F804FEA021A06EB0A015F4891F8E3
:107D100010E05D4911F80E10181A45180CF1100CFE
:107D2000132D5FFA8CFCC6DD029DDFF86CA15FFAB3
:107D300080FE0EF10603DBB243F04001E171591CF5
:107D40000291D3B10EF1050E5FFA8EFE0EF1080E10
:107D5000A6440AF1010C00231CF8010B58408300D3
:107D600083EA4003C1084340494801F0180140FA42
:107D700001F14B40E645DBB2EED1029986F8752061
:107D80000AF80130E3799DF80C10E17003F03F032D
:107D9000981C03F10A016071A1703E4C0833E2188F
:107DA00020464FF0000E10F8013B83EA0E0383EAF1
:107DB0000313DBB24FEA1E2E4FEAC30C4EEA032E2A
:107DC0008CEA13138EEA03031BB282421FFA83FE6E
:107DD000E9D121444FEA1E2201F8023CA378234452
:107DE00003F8012C91E5DEF81C10DEF8200081423A
:107DF0003BBFDEF80C205218A1EB000AA2EB000AF0
:107E0000DCE4392026F0F2FFBAF80060F0B226F088
:107E1000C5FF300A26F0C2FFC5E617F03BF926F091
:107E2000BDFF0021D4F8680108F0A2F8FEF7B8BE43
:107E30000423FEF759BE0323FEF756BE0223FEF7C6
:107E400053BE1249029D581A6FE708230293FEF7AA
:107E50006FBD164617461046039296460292FDF7EE
:107E600042BF1646FDF73FBF16461746104603921F
:107E7000FDF739BF16461746FDF735BF16461746BC
:107E80001046FDF730BF00BFCC4F0308CD220020C5
:107E90000007090EC0220020C62200202DE9F0476D
:107EA0000F46B0F908102DED028B3981C9B24B1E77
:107EB00092B01546FD2B00F20081DFE813F0640557
:107EC0005905480539050005FE00FE00FE00FE00CC
:107ED000EF04FE00FE00FE00FE00FE00FE00FE00BD
:107EE000FE00FE00FE00FE00FE00FE00FE00FE00A2
:107EF000FE00FE00FE00FE00FE00FE00FE00FE0092
:107F0000C904FE00C104FE00AE04FE009504FE009C
:107F10009004FE004404FE002C04FE002104FE0038
:107F20001C04FE00C509FE00E002FE004403FE0042
:107F3000D002F302FE003403FE00FE002803FE0020
:107F4000FB02FE00F503C102E103FE00FE00D803C0
:107F5000FE00FB03FE00B803FE0091036103FE0078
:107F60007505FE007E09FE00FE00FE004909FE00C8
:107F70001709FE00E308FE008B08FE007908FE00EA
:107F8000FE00FE0060084E0A1A0A090AF1099E0A5C
:107F9000FE00FE00850A52082108D707BC07FE0034
:107FA000620758071C071007FE00E706AD06FE0033
:107FB000FE00FE007F06630652061406FE00FE0069
:107FC000FE00FE00FE00FE00FE00FE00FE00FE00C1
:107FD000FE00FE00FE00FE00FE00FE00FE00FE00B1
:107FE000FE00FE00FE00FE00D605FE00FE00FE00C4
:107FF000FE00FE00FE00FE00FE00FE00C405FE00C6
:10800000FE00FE00FE00FE00FE00FE00FE00FE0080
:10801000FE00FE00FE00FE00FE00FE00FE00FE0070
:10802000FE00FE00FE00FE00FE00FE00FE00FE0060
:10803000FE00FE00FE00FE00FE00FE00FE00FE0050
:10804000FE00FE00FE00FE00FE00FE00FE00FE0040
:10805000FE00FE00FE00FE00FE00FE00FE00FE0030
:10806000FE00FE00FE00FE00FE00FE00FE00FE0020
:10807000FE00FE00FE00FE00FE00FE00FE00FE0010
:10808000FE00FE00FE00FE00FE00FE00FE00FE0000
:10809000FE00FE00FE00FE00FE00FE00B6058505A7
:1080A000FE00FE00FE00FE00FE00FE00FE00FE00E0
:1080B000FE00FE00FE00FE00D502F529044600F099
:1080C000658194E828000B39ED1AEF2901F2E1816E
:1080D000DFE811F0F409DF09DF09DF09DF09DF0953
:1080E000DF09DF09DF09DF09DF09DF09DF09DF0950
:1080F000DF09DF09DF09DF09DF09DF09DF09DF0940
:10810000DF09DF09AE0ADF09E709DF09050EDF092C
:108110000F0ADF09290ADF09520ADF094B0FDF09BD
:10812000690DDF09800DDF09960DDF09A509DF095B
:10813000C60DDF09DF095301DF09E80DDF09DF099B
:10814000F80DDF09380DDF09DF09DF09DF09DF0975
:10815000DF09E50ADF09EC0ADF09120BDF09DF0995
:108160003B0BDF09550BDF096E0BDF09830BDF09C2
:10817000F000DF09F80BDF092B0CDF094F0CDF09DA
:10818000BD0CDF09DF09DF09DF09DF09DF09DF09CE
:10819000DF09DF09DF09DF09DF09DF09DF09DF099F
:1081A000DF09DF09DF09DF09DF09DF09DF09DF098F
:1081B000DF09DF09DF09DF09DF09DF09DF09DF097F
:1081C000DF09DF09DF09DF09DF09DF09DF09DF096F
:1081D000DF09DF09DF09DF09DF09DF09DF09DF095F
:1081E000DF09DF09DF09DF09DF09DF09DF09DF094F
:1081F000DF09DF09DF09DF09DF09DF09DF09DF093F
:10820000DF09DF09DF09DF09DF09DF09DF09DF092E
:10821000DF09DF09DF09DF09DF09DF09DF09DF091E
:10822000DF09DF09DF09DF09DF09DF09DF09DF090E
:10823000DF09DF09DF09DF09DF09DF09DF09DF09FE
:10824000DF09DF09DF09DF09DF09DF09DF099D0C2D
:10825000DF09200DDF09D20C130D190E270E7B0E3E
:10826000DF098A0E9E0E860FDF09640FDF09DF0922
:10827000720FA70EC10EC90EDE0EDF09DF09DF097E
:10828000DF09DF09DF09DF09DF09DF09DF09DF09AE
:10829000DF09DF09DF09DF09DF09DF09EF0EDF0989
:1082A000DF09FE0EDF09DF09DF09DF09DF09DF096A
:1082B000DF093E0F20460EF079FC054603F005FB72
:1082C000FF285AD012A9002301F8423DEE080DF113
:1082D00005008DF80530013623F0EEF89DF80530E5
:1082E000F6B205F00705B34205F1010503D19DF88B
:1082F0000630AB420ED0AF4B1B685BB11A79B2426D
:1083000008D35A79AA4205D31B68DB6813B1294602
:108310003046984723686268D21A012A2DDD5A1C1C
:1083200012A8226000221D7800F8412D23F0D0F819
:108330009DF80730AB420AD09E4B1B683BB19A793F
:10834000AA4204D31B681B690BB1284698472368CF
:1083500012A85A1C226000221C7800F8402D23F03D
:10836000C3F89DF80830A34207D0924B1B6823B195
:108370001B685B690BB12046984701231A461846D3
:108380007A8112B0BDEC028BBDE8F08794E80C0056
:10839000934241F06E86884BFF2283F823204FF0F2
:1083A0000009864C07F0E8FD49463022844884F8ED
:1083B00000902CF0BEF88DF808909DF808300B2B3B
:1083C00001F26C80DFF814827D4E4A469DF8083039
:1083D00003EB830308EB83031B7BE3B19DF80830B9
:1083E00003EB830308EB830320211B699BB19DF8FA
:1083F000083003EB830308EB8303186946F8220077
:108400000DF07AFB237856F823000DF037FD227823
:108410000132D2B222709DF808300133DBB28DF800
:1084200008309DF808300B2BD0D93B68591C3960B7
:108430001A70002DA1D0634B2B6001231A469EE7D2
:10844000614B03F10B043A6813F8011B501C9C426A
:1084500038601170F7D1002138460EF0B9FB0021C9
:1084600038460EF0B5FB88E7584C04F1080534F89F
:10847000021B38460EF0C4FBA542F8D17DE7544CF0
:10848000544D04F1300694F9DA120023EA568A4278
:1084900003F10C0301F01586482BF7D10834B442E0
:1084A000F1D16AE7396801200A183A6003460246AA
:1084B000087064E7464C3B6894F8B322591C396055
:1084C0001A70A16838460EF083FB3B6894F85C2272
:1084D000591C39601A70B4F8E41138460EF090FB5C
:1084E000B4F8E81138460EF08BFBB4F8EC113846BE
:1084F0000EF086FBB4F8401238460EF081FBB4F85B
:10850000421238460EF07CFB01231A4637E7324B05
:1085100003F108013A6813F8010B541C99423C60BE
:108520001070F7D129E73A68294B501C93F8B21222
:1085300038601170396893F8B1024A1C01233A601F
:108540001A4608701BE73A68214B501C93F8381202
:10855000386011703A6893F83C12501C3860117002
:108560003A6893F83B12501C386011703A6893F8DF
:108570003D12501C38601170396893F83F02DCE7F7
:108580003968134A0123481C38600B70396892F827
:108590007D06CC183C600870396892F87B06CC18D0
:1085A0003C600870396892F87C06CA183A601A462E
:1085B0000870E4E63C870020702600201B5B00204A
:1085C00068580020698F0208C876030814880020C4
:1085D00094610020487E0020E8630020E88C0020A1
:1085E0003B6801241A193A601C701AF0E9FC002853
:1085F00041F08A85C24DC34A03463968481C386039
:108600000B703B6841F2B410591C105C396041F2A8
:108610007811187051583846890A0EF0D9FAE96B6A
:10862000384649080EF0D4FA01231A46A7E6B64E9A
:108630003378002B3FF4A1AEB44C00253B6894F88E
:108640007C22591C39601A7094F87D3203EB830345
:1086500003EB830303F2EE2189B238460EF0D0FA21
:10866000337801359D4204F10204E7DB85E6A84B2F
:108670003846B3F848100EF0C3FA01231A467EE6D6
:108680003B6800245A1C3A6021461C7038460EF0A4
:108690009FFA214638460EF09BFA214638460EF0E6
:1086A00097FA01231A466AE6002D3FF466AE994B0D
:1086B0002B6062E63B68954C591C94F8B6223960F1
:1086C0001A703B6894F8B722591C39601A70B4F8D4
:1086D000B81238460EF094FA3B6894F8BA22591C46
:1086E00039601A70B4F8BC1238460EF089FA39684D
:1086F00094F8BE0221E7854B396893F867021CE7BE
:10870000854C04F1800554F8041F38460EF060FAD9
:10871000AC42F8D131E67D4C04F14005B4F8BC130D
:1087200038460EF06DFA3B6894F8BE23591C396048
:108730001A703B6894F8BF230434591CAC4239606A
:108740001A70EBD119E6714C3B6894F85C22591C05
:1087500039601A70B4F86E1238460EF051FAB4F857
:108760006A1238460EF04CFAB4F86C1238460EF025
:1087700047FA3B6894F86522591C39601A70B4F8BE
:10878000781238460EF03CFAB4F87A1238460EF0F9
:1087900037FA3B6894F87022591C39601A703B68AC
:1087A00094F87222591C39601A70B4F8761238465F
:1087B0000EF026FA3B6894F85F22591C39601A7053
:1087C000D4F8601238460EF003FA3B6894F864223D
:1087D000591C39601A70396894F87302ADE64B4B36
:1087E000396893F8B302A8E6484C3846B4F840120A
:1087F0000EF006FAB4F8421238460EF001FA3B6861
:1088000094F84422591C39601A70B4F8461238465C
:108810000EF0F6F901231A46B1E53C4C3846B4F89F
:10882000E4110EF0EDF9B4F8E81138460EF0E8F96D
:10883000B4F8EC1138460EF0E3F901231A469EE530
:10884000324B384699680EF0C3F901231A4696E573
:108850002E4B324D03F1500493F8D125396802EBC9
:10886000420205EB8202481C92F8382038600A70F8
:108870003A6893F8D215501C386011703A6893F832
:10888000D315501C386011703A6893F8D41504332E
:10889000501CA34238601170DED16EE5204827F0ED
:1088A0008BF8011E7FF769AD1D4B19443A6813F828
:1088B000010B541C8B423C601070F7D15DE5194BE5
:1088C00003F10B043A6813F8011B501C9C423860FA
:1088D0001170F7D1144B03F108013A6813F8010F36
:1088E000541C8B423C601070F7D1104BD91D3A6874
:1088F00013F8010F541C8B423C601070F7D13CE51B
:10890000406100200C6B00206088002094610020F2
:10891000CC890020E5410108CC640020FC4F03080D
:108920001C680020C8760308BB7603085390030830
:10893000AC4B191D3A6813F8010B541C99423C606A
:108940001070F7D1002138460EF05AF915E53B6852
:108950000322591C39601A703A680123D118396012
:10896000137039680720CA183A601A46087006E57D
:108970009D4B191D3A6813F8010B541C99423C6039
:108980001070F7D1F9E43B680022591C39601A7065
:108990003A680123D1183960137039681F20CA184A
:1089A0003A601A460870EAE43A68904B501C01217C
:1089B0003860981D11703A6813F8011F541C8342E7
:1089C0003C601170F7D1D8E4894B03F170043A6828
:1089D00093F80211501C386011703A6893F8031133
:1089E000501C386011703A6893F80411501C3860BC
:1089F00011703A6893F80511501C386011703A688C
:108A000093F80611501C386011703A6893F80711FA
:108A1000501C386011703A6893F808110733501CE5
:108A2000A34238601170D2D1A7E4714C3846B4F833
:108A300022120EF0E5F8B4F8201238460EF0E0F8F5
:108A400001231A469BE46B4B384619680EF0C0F8B8
:108A5000694B384619680EF0BBF8684B3846196800
:108A60000EF0B6F801231A4689E4654B3846B3F890
:108A700058100EF0C5F8002138460EF0C1F8614BD1
:108A80001A68C2F3C003C2F380019B0043EA4103AA
:108A9000C2F340010B43C2F3401143EAC10102F0AB
:108AA0001002114338460EF0ABF80CF0ADFA014657
:108AB00038460EF08DF83B684D4A581C92F8D01598
:108AC000514A38601970118864293846A8BF64215A
:108AD0000EF096F83B684D4A581C03213860197017
:108AE0003968107829E5DFF82CE10025EEB27146EF
:108AF00000233A68501C386016703A68501C386081
:108B000013703A6811F8010F0133541C062B3C60B6
:108B10001070EED10135062D0EF1060EE6D13C495E
:108B200000233A68501C386015703A68501C386051
:108B300013703A6811F8010F0133541C0B2B3C6081
:108B40001070EED13B682A4A581C07213860197012
:108B50003B680021581C38601970396892F82C0461
:108B6000EBE43A68224B501C93F8FC11386011700A
:108B70003A6893F81812501C38601170396893F8ED
:108B80000E02DAE43A681A4B501C93F84C12386023
:108B900011703A6893F84D12501C386011703A68A1
:108BA00093F84E12501C38601170B3F8EE1038462E
:108BB0000EF026F801231A46FFF7E1BB0C4C3846AD
:108BC000B4F8E8100EF01CF8B4F8EA1038460EF0CD
:108BD00017F8B4F8EC1038460EF012F801231A46D4
:108BE000FFF7CDBBC87D0308C07D0308C365002027
:108BF00094610020ACF7FF1FB0F7FF1FB4F7FF1F11
:108C0000A4180020248A0020404200200D8E00205D
:108C1000B36500208F650020B14E00253446B4F8BE
:108C2000721138460DF0ECFFB4F8741138460DF0AF
:108C3000E7FFB4F8761138460DF0E2FF3B6894F890
:108C40007821591C39601A703B6894F87921591CB5
:108C500039601A703B6894F87A21591C39601A708F
:108C60003A6894F87B11C5EBC503501C06EB43032F
:108C700038601170D3F87C11013538460DF0A8FF2B
:108C8000082D04F10E04CAD1FFF777BB954C237869
:108C9000002B3FF472ABDFF854E2E61C0025002302
:108CA00016F8010F904A194604E00133202B10D02A
:108CB00012F80C1C884202F10C02F6D1DBB203EB75
:108CC00043033A680EEB8303511C93F83830396044
:108CD0001370237801359D42E1DBFFF74EBB8349DA
:108CE00052233A68501C3860137011F8013F002B72
:108CF000F7D1FFF742BB7B4C2378002B3FF43DAB11
:108D00007A4E0125DFF8F4914FF00108002319F89D
:108D1000010F754A194605E00133202B01F09C81B3
:108D200012F80C1C884202F10C02F5D1DBB203EB05
:108D3000430306EB8303D3F834A0504626F03CFEF1
:108D4000002D41F0898100280ADD53460AEB000E10
:108D50003A6813F8011B501C9E4538601170F7D11A
:108D6000237843457FF709AB08F10108CEE70123DB
:108D70003A68511C396013700133092BF8D1FFF7A1
:108D8000FCBA574C3846B4F86A120DF039FFB4F803
:108D9000CC1038460DF034FFB4F8CE1038460DF044
:108DA0002FFFB4F8D01038460DF02AFFB4F8B812EF
:108DB00038460DF025FF3A684D490023501C3860B5
:108DC00013703A68501C386013703A68501C386051
:108DD00013703A6894F84502551C3D6010703A686B
:108DE00094F86702551C3D6010703A68501C38605A
:108DF0001370B4F90C3281FB0321DB17C3EBA10123
:108E000089B238460DF0FCFE3B6894F83822591CB4
:108E100039601A703B6894F83C22591C39601A700A
:108E20003B6894F83B22591C39601A70396894F8F1
:108E30003D02FFF782BB2F4E00233A683168501C79
:108E4000C95C38601170326839681A44481C927ADB
:108E500038600A70326839681A440133127D481C40
:108E60000A2B38600A70E8D1FFF787BA224C3B68BA
:108E70002268591C127839601A7023683A68997808
:108E8000531C3B6000231170226839681A44013377
:108E90005279481C032B38600A70F5D13B68226870
:108EA000591C127A39601A703B682268591CD278B2
:108EB00039601A703B682268591C127939601A703F
:108EC0002368384659890DF09BFE3B682268591C7F
:108ED000527A39601A70236839685878FFF72DBBC9
:108EE000946100207026002038500308FC4F0308CE
:108EF000676666668C410020108E00207326002075
:108F0000C84B3A681B88C849FF2BA8BFFF23501CD9
:108F10003860137009684FF6FF74A142A8BF21465C
:108F200021EAE17189B238460DF06AFEBF4B38463E
:108F300019880DF065FEBE4B93F84532002B01F009
:108F4000FA80BC4B1B6803EB83035900A142A8BF06
:108F5000214621EAE17189B238460DF051FEFFF752
:108F60000CBAB54B384619680DF032FEB34B384693
:108F700019880DF045FE01231A46FFF700BA3B6839
:108F8000AB4A581CE721386019703B6892F8B3224D
:108F9000591C39601A703B680022591C39603846E8
:108FA0001A7004210DF014FE01231A46FFF7E7B9E9
:108FB0003A689F4B501C93F81912386011703A6848
:108FC00093F82412501C38601170396893F80F021E
:108FD000FFF7B3BA002138460DF012FE00213846E3
:108FE0000DF00EFE002138460DF00AFE3A68944C52
:108FF0000023511C396013703A682168501C91F8A5
:109000003510386011703A682168501C91F8401092
:10901000386011703A682168501C91F8411038602E
:1090200011703A68511C396013703A68511C3960EC
:1090300013703A68511C39601370236893ED120A5B
:10904000B2EE048A20EE080A29F068F981B23846A7
:109050000DF0D6FD236893ED110A20EE080A29F0E1
:109060005DF981B238460DF0CBFD3B682268591C92
:1090700092F8372039601A702368396893F83800FD
:10908000FFF75BBA6A4C3B6894F801226C4D591C9F
:1090900039601A702B683846198C0DF0B1FD2B68B9
:1090A0003846598C0DF0ACFDB4F8041238460DF07A
:1090B000A7FDB4F8061238460DF0A2FD2B6838461D
:1090C000998C0DF09DFD2B683846D98C0DF098FDDC
:1090D000B4F8081238460DF093FDB4F80A12384679
:1090E0000DF08EFD01231A46FFF749B9504E96F850
:1090F000FF31002B01F025803B680822591C3960A4
:109100001A703B680122991839601A703B6896F80A
:10911000D520591C39601A703B6896F8D420591C28
:1091200039601A70B6F8D21038460DF069FDDFEDDF
:10913000457A96ED360A20EE270A29F0EFF881B23B
:1091400038460DF05DFD396896F80302FFF7F5B972
:1091500002F0BBFBFF28054601F0018012A90024A4
:1091600001F8424D0DF105008DF8054022F0A4F9FB
:1091700012A800F8414D22F0ABF912A800F8404DBA
:1091800022F0B2F93B685A1C3A601D703B689DF8AA
:109190000520591C39601A703B689DF80620591C3F
:1091A00039601A703B689DF80720591C39601A70A5
:1091B00039689DF80800FFF7C0B93B681C4C591C82
:1091C000012239601A703B6894F86C24591C39608C
:1091D0001A703B6894F86A24591C39601A703B680D
:1091E00094F86224591C39601A70B4F86414384633
:1091F0000DF006FDB4F8661438460DF001FDB4F824
:10920000681438460DF0FCFC04F2344504F58C6417
:1092100035F8021F38460DF0F3FCA542F8D1FFF7F0
:10922000ACB800BF3445002030450020A4450020E4
:109230009461002058240020102600202C240020B7
:109240008C4100200000C842BB4B03F15A043A682D
:1092500093F82616501C386011703A6893F821165E
:10926000501C386011703A6893F82216501C386010
:1092700011703A6893F82316501C386011703A68E0
:1092800093F82416501C386011703A6893F825162C
:109290000633501C9C4238601170D8D1FFF76DB86E
:1092A000A64CA74D04F1A00607E014340DF0A8FC6D
:1092B000B44205F102053FF460A8237B3846194605
:1092C000002BF2D028881CF09FFD01463846ECE7C1
:1092D0009C4A3B68146850689168D268DA601C60E8
:1092E000586099603A68012310323A601A46FFF7D5
:1092F00046B8954C2289B2F5007F04F1300594BF41
:10930000012604263C3455F8041B91FBF6F138463F
:1093100089B20DF075FCA542F5D18C4C04F10C0618
:10932000A4F14C05B4EC010AD5ED067A80EE270ACB
:1093300028F0F4FF81B238460DF062FCA642F1D16C
:10934000834C04F10C0554F8041B384689B20DF027
:1093500057FCAC42F7D1FFF710B87E4B3846B3F854
:1093600058100DF04DFC384600210DF049FC7A4BA9
:109370001A68C2F3C003C2F380019B0043EA4103B1
:10938000C2F340010B43C2F3401143EAC10102F0B2
:109390001002114338460DF033FC0BF035FE014648
:1093A00038460DF015FC3B68634A581C92F8D015FE
:1093B0006A4A38601970118864293846A8BF642148
:1093C0000DF01EFCFFF7BEBA654C384621880DF043
:1093D00017FC618838460DF013FCB4F9043061497C
:1093E000DA1781FB0313C2EBA30399B238460DF0E1
:1093F00007FC01231A46FEF7C2BF5B4E3378002BF1
:109400003EF4BBAF594D002435F8021F38460DF02D
:10941000F7FB337801349C42F6DBFEF7AEBF544ACB
:10942000A2FB0512A91A02EB51029208C2EBC2017B
:109430006D1A2ED1D2B2511EC9B2002A3EF49DAF90
:1094400001F101081AE080F8029020460DF0AEFB11
:10945000226830801346511C216013F8021BF17002
:10946000236053783371D31C23609378B371131D39
:109470002360D2787271A8453EF47FAF5A1C2260F7
:1094800093F90090484618F059F90135064600282E
:10949000D9D14FF0FF331A46FEF771BF4A46FEF7A7
:1094A000C4BF254D0023AB6020460DF067FBAA68C2
:1094B00001230243AA601A46FEF761BF2D49102D11
:1094C0004FF000022B4628BF10230A604A608A60D2
:1094D000CA600A74002B3EF450AF22681344013274
:1094E000226012F8010C01F8010B9342F7D1FEF74C
:1094F00044BF20460DF05AFB0F4DA5F84002204610
:109500000DF054FB2368A5F842025A1C22601B7818
:1095100085F8443220460DF049FB0123A5F84602A8
:109520001A46FEF72CBF5A1C2260034A1B7882F8A9
:10953000B332FEF722BF00BF94610020E88C002008
:10954000604900203C6000208C890020188A00209F
:109550005C520020A4180020248A002040420020F1
:10956000D0600020676666666088002072880020F0
:10957000254992241C6800205A1C2260C84E1B7882
:1095800086F85C3220460DF011FBA6F86E022046EC
:109590000DF00CFBA6F86A0220460DF007FB2368CD
:1095A000A6F86C025A1C22601B7886F86532082DDA
:1095B0007EF6E3AE20460DF0F9FAA6F878022046D2
:1095C0000DF0F4FA0C2DA6F87A027EF6D6AE2368DA
:1095D0001A46591C216012F8021B86F8701222608C
:1095E0005B7886F8723220460DF0E0FA102DA6F86E
:1095F00076027EF6C2AE23685A1C22601B7886F87B
:109600005F3220460DF0BAFA2368C6F860025A1C91
:1096100022601A7886F86422162D7EF6AEAE9A1C69
:1096200022605B7886F8733201231A46FEF7A7BEE4
:109630005A1C2260187813283FF62BAF9A1C226020
:1096400000225E789749154605E00132202A3FF452
:1096500020AF11F80C5CAE4201F10C01F5D1D2B291
:10966000914D8F49914E02EB420205EB820500F5C8
:10967000BA7001EB800295F830105170D91C21604E
:1096800099789170191D2160D978D170591D216088
:109690001B793068137121F037FDFEF76EBE20464E
:1096A0000DF084FA01231A46FEF769BE1A46591CCA
:1096B00021607B4D12F8021B85F8B61222605B78A0
:1096C00085F8B73220460DF071FA2368A5F8B80284
:1096D0005A1C22601B7885F8BA3220460DF066FAD3
:1096E0002368A5F8BC025A1C22601B7885F8BE329C
:1096F00001231A46FEF743BE5A1C22601A78112A2B
:109700003FF6C7AE664D02F59E72991C05EB420509
:1097100021605B782B7120460DF048FA40F6CA03B1
:109720009842A8BF184640F2EE239842B8BF1846A8
:109730005F4AA0F2EE2082FB0032C017C0EBE202CB
:1097400001236A711A46FEF71ABE5A4A1278012A94
:109750003EF613AE19465A1C2260514A11F8020B0C
:1097600082F87D062160597882F87B16D91C216029
:109770009B7882F87C3601231A46FEF700BE062D40
:109780007FF487AE4C4A991D0133236013F8010C16
:1097900002F8010F9942F7D1484B93F82530002B7E
:1097A0003EF4EBAD20F080FF01231A46FEF7E7BD43
:1097B0005A1C22601D78FF2D00F00E8520460DF00A
:1097C000F5F9152D3EF6D9AD354A02EB45020123D8
:1097D000A2F836041A46FEF7D2BD5A1C226013F8CE
:1097E000378B0DF107010132226012F8010C01F8EC
:1097F000010F9342F7D1314C94F82650002DFDD142
:10980000DFF8BCA00126082084F8266024F04CFC78
:10981000DAF800000CF02CFB284684F8276024F0CE
:1098200019FC284624F016FC092024F013FC4046BD
:1098300024F010FC0DF1080845460DF13E09A5EB9A
:109840000806F6B20A2024F005FC304624F002FC9B
:1098500015F8016B0B2024F0FDFB304624F0FAFBD9
:1098600024F076FCA945EAD1082024F0F3FBA020DF
:1098700024F0F0FBA02024F0EDFB002024F0EAFB14
:1098800010F02005F6D1DAF800000CF0F7FA02200B
:1098900024F00AFC012384F826501A46FEF76FBD17
:1098A0009461002040500308FC4F03088C410020C5
:1098B0001F85EB5148950020C365002070260020CD
:1098C000708700201A46591C2160C74E12F8021BEF
:1098D00086F8FE1122605A7886F8F821DA1C226098
:1098E0009A7886F8D5201A1D2260DB78082BA8BF4D
:1098F0000823204686F8D4300DF058F9072DA6F835
:10990000D20000F25A84236862689A4207D05A1C37
:1099100022601B78003318BF012386F8033207F05A
:109920009BF901231A46FEF72ABD5A1C2260AF4E4E
:10993000DFF8B4821B78D6F8009088F80132204610
:109940000DF034F9A9F820002046D6F800900DF06B
:109950002DF9052DA9F8220000F2618407F07CF9A9
:109960001AF0C4FA30681CF0BBF801231A46FEF75F
:1099700006BD20460DF01AF920460DF017F92046D5
:109980000DF014F920460DF01DF92368974E9FED58
:10999000988A32681946581C206011F8020B82F828
:1099A00035002160597882F84010D91C21609B78DD
:1099B00082F8413020460DF005F920460DF002F9FD
:1099C00020460DF0FFF82046D6F800900DF0EEF896
:1099D00007EE900AF8EEE77A204667EE887AD6F826
:1099E0000080C9ED127A0DF0E1F807EE900AF8EE6A
:1099F000E77A112D67EE887AC8ED117A00F28D832F
:109A0000306819F0E3F801231A46FEF7B8BCC5F335
:109A10004705122D3FF63DAD002D00F0CB8305F13B
:109A20000043013B0DF1080909EB43080DF106065F
:109A300020460DF0BBF826F8020FB045F8D12946B4
:109A4000484616F0E9F801231A46FEF798BC194675
:109A50005A1C2260644A11F8020B82F81902216034
:109A6000597882F82412D91C21609B7882F80F3231
:109A700001231A46FEF783BC092D7FF60AADDFF8F5
:109A80007C811A46591CD8F80060216012F8021B2C
:109A9000317022605A78B270DA1C22609A78642A97
:109AA00003F10401A8BF642272712160DA78642A8C
:109AB00003F10501A8BF6422B27121601A79F27125
:109AC0009A1D22605A79642A28BF6422D91D3272F5
:109AD00021609A79F27003F108022260DB79337118
:109AE00020460DF063F80A2D708140F04B830BF097
:109AF0000FFB01231A46FEF742BC3E4B1B78590769
:109B00003EF53BAC3C4A4FF4C871012311801A4624
:109B1000FEF735BC354A1068DA1C411E2133951E0C
:109B2000256012F8035C01F8015F551E256012F8EC
:109B3000025C8D72226012F8015C0D7503329A424C
:109B4000EDD15EE75A1C284D22601B7885F8B332B0
:109B50000023AB6020460DF011F82268AB68511C61
:109B60000343AB602160137885F85C3220460DF02A
:109B70001DF8C5F8E40120460DF018F8C5F8E80115
:109B800020460DF013F8C5F8EC0120460DF00EF854
:109B9000A5F8400220460DF009F80123A5F842027D
:109BA0001A46FEF7ECBB5A1C22601E781F2E3FF6A9
:109BB00070AC052D7FF46DAC20460CF0DFFF0A4B36
:109BC00003EB8603C3F83C0310F0EAF901231A46BD
:109BD000FEF7D5BB5A1C2260034A1B7882F8673215
:109BE00001231A46FEF7CBBB946100208C41002074
:109BF000CDCCCC3D1B8E0020488E0020108E002046
:109C00005A1C22601A780E2A3FF643AC991C216038
:109C1000597803293FF63DACC74802EB420200EBFE
:109C20004202D81C82F826162060997882F8211604
:109C3000191D2160D97882F82216591D21601979E1
:109C400082F82316991D2160597982F82416D91DAE
:109C500021609B7982F8253601231A46FEF78FBBD7
:109C600019465A1C2260B44A11F8020B82F83802D5
:109C70002160597882F83C12D91C2160997882F8C9
:109C80003B12191D2160D97882F83D12042D7EF611
:109C900074AB591D21601B7982F83F3201231A46AB
:109CA000FEF76DBB1A46591C2160A34912F8020B3E
:109CB00081F8B20222605B7881F8B13201231A4642
:109CC000FEF75DBB9D4A03F108010133236013F8E1
:109CD000010C02F8010B9942F7D1FEF74EBB20466A
:109CE0000CF064FF944DC5F8E40120460CF05EFFD3
:109CF000C5F8E80120460CF059FF0123C5F8EC0136
:109D00001A46FEF73CBB8E4B1B785A073EF535AB27
:109D10008C490A78012342F004020A701A46FEF7C1
:109D20002EBB20460CF042FF834DA5F86A02204668
:109D30000CF03CFFA5F8CC0020460CF037FFA5F84E
:109D4000CE0020460CF032FFA5F8D00020460CF0E3
:109D50002DFFA5F8B80220460CF034FF20460CF089
:109D600031FF20460CF02EFF23681A46591C216053
:109D700012F8021B85F8451222605B7885F867327D
:109D800020460CF01FFF20460CF010FF236800EB6C
:109D900080001A464100581CA5F80C12206012F8E9
:109DA000021B85F8381222605A7885F83C22DA1CAA
:109DB00022609A7885F83B221A1D2260DB7885F8AC
:109DC0003D3201231A46FEF7DABA5D4B1B7858077D
:109DD0003EF5D3AA07F0E8FB0CF082FC0CF008FB80
:109DE00001231A46FEF7CBBA5A1C226018780506E2
:109DF00000F1BD81524B1B785C073EF5BEAA0328DB
:109E000028BF00200BF016FC01231A46FEF7B7BA54
:109E100020460CF0CBFE4C4A012310801A46FEF778
:109E2000AEBA1A46591C2160434D12F8021B85F840
:109E30004C1222605A7885F84D22DA1C22609B78F9
:109E400085F84E3220460CF0B1FE0123A5F8EE0055
:109E50001A46FEF794BA3D4B186806F0C3FF01237B
:109E60001A46FEF78CBA19465A1C2260324A11F87B
:109E7000020B82F8FC012160597882F81812D91C73
:109E800021609B7882F80E3201231A46FEF777BADA
:109E90001A46591C216012F8020B2260DA1C59780C
:109EA00022609A7810F00EF800287EF466AAFFF778
:109EB000F0BA20460CF07AFE1F4DA5F8220220468B
:109EC0000CF074FE0123A5F820021A46FEF757BADB
:109ED0005A1C226019780F293FF6DBAA164A981CF3
:109EE000C1EBC10120600A44597882F80211D91CE3
:109EF0002160997882F80311191D2160D97882F8C0
:109F00000411591D2160197982F80511991D2160EC
:109F1000597982F80611D91D2160997982F80711C3
:109F200003F108012160DB7982F8083118F016FC92
:109F300001231A46FEF723BA94610020E86300204B
:109F40001B8E00204A8E0020B24700208C4100204A
:109F5000C94B1B785B073FF59CAA0CF0C1FB0CF0CA
:109F600047FA01231A46FEF70ABAC44D05F1400626
:109F700020460CF01BFE2368A5F8BC03591C1A46AA
:109F8000216012F8021B85F8BE1322605B7885F809
:109F9000BF330435AE42EBD1FEF7EFB9B84D05F152
:109FA000100620460CF002FE1BF05CFF25F8020FA5
:109FB000AE42F6D1FEF7E1B920460CF0F7FDAF4D09
:109FC000A5F8E80020460CF0F1FDA5F8EA002046CF
:109FD0000CF0ECFD0123A5F8EC001A46FEF7CFB912
:109FE0000F2D7FF456AA5A1C22601E78072E3FF6CA
:109FF00050AA2046A14D0CF0D9FDC6EBC60605EBD4
:10A000004605A5F8720120460CF0D0FDA5F87401B4
:10A0100020460CF0CBFD2368A5F876011A46591CA2
:10A02000216012F8021B85F8781122605A7885F8B1
:10A030007921DA1C22609A7885F87A211A1D22602B
:10A04000DB7885F87B3120460CF098FD0123C5F8BC
:10A050007C011A46FEF793B923789845FEF684AE44
:10A06000002D3EF48AA90025002B7EF44BAEFEF7AE
:10A0700084B9531C11462360824811F8023B80F8D2
:10A0800023302160527880F82420042B06D9FF2B3E
:10A090003EF485A939680020FEF74FBA072A03D994
:10A0A000022BF7D1FF2AF5D13A680123D118396084
:10A0B0001370002D3EF461A9734A2A601A46FEF718
:10A0C0005EB93B685A1C3A601970B4F8D812384629
:10A0D0000CF096FD3B6894F8DB22591C39601A702D
:10A0E0003B6894F8DC22591C39601A703B6894F87C
:10A0F000DE22591C39601A703B6894F8DD22591C25
:10A1000039601A70FEF7CAB9604D614A95F824307B
:10A11000002B46D12346FEF770BA23683068591CDD
:10A120001A46216012F8021B80F8371022605B7813
:10A1300080F8383065E4574B196801F30F01FEF7DA
:10A140000ABF3B6896F8FE21591C39601A703B68BB
:10A1500096F8F821591C39601A70FEF7D7BF396894
:10A160000123CA183A601A460870FEF708B900F0D1
:10A170007F00032828BF00200BF03CFA01231A4679
:10A18000FEF7FDB82368D8F80020591C2160197823
:10A1900051720B2D3FF4ABAC991C21605B7853706E
:10A1A000A5E45178022961D003290CBF042323467A
:10A1B000FEF723BA0DF1080941E420460CF0F6FC45
:10A1C00007EE900A9FED347AF8EEE77A67EE877A29
:10A1D000C6ED367AFFF797BB9A1C2260274D5A7856
:10A1E00085F86C24DA1C22609A7885F86A241A1D96
:10A1F0002260DB7885F8623420460CF0D7FCA5F8A5
:10A20000640420460CF0D2FCA5F8660420460CF04D
:10A21000CDFC0123A5F868041A46FEF7B0B8204625
:10A220000CF0C4FCA8F8040220460CF0BFFCA8F80F
:10A2300006022046D6F800900CF0B8FCA9F82400DD
:10A240002046D6F800900CF0B1FC0D2DA9F82600A0
:10A250007FF684AB20460CF0A9FCA8F80802204643
:10A260000CF0A4FCA8F80A02FFF778BB042B34BF5B
:10A2700002230323FEF7C1B91B8E00209461002046
:10A280003E58002070260020FD410108406100205A
:10A290000C6B0020582400200AD7233C0279407917
:10A2A00002FB00F0704700BF00207047002070479D
:10A2B0004FF0FF30704700BF00207047002070470C
:10A2C0001E2000FB0212024900208B54704700BF81
:10A2D00098260020F0B41C7884B11E20094F10FB92
:10A2E000021200200E181D2E07EB000600F10105DA
:10A2F000E8B2D8BFB4541C5C002CF3D10020F0BCF1
:10A30000704700BF98260020014B1888704700BF97
:10A31000AA00002008B54FF4F072202102482AF06C
:10A3200008F9002008BD00BF98260020044A054B0C
:10A33000106805490340002013600880704700BF83
:10A34000BC200020BC2FDFFFA6200020437913F0A3
:10A35000020308D00369426A806A013B101A184060
:10A36000C0B2181A704718467047426A806A131ABA
:10A3700058425841704741717047704743799B0775
:10A380000AD5436A8269D154436A01690133B3FB38
:10A39000F1F201FB123343627047437913F001037A
:10A3A0001FBFC369026AC0689B1A1ABF00F1FF3061
:10A3B00018401846704710B5437913F00103014661
:10A3C0000ED0FFF7EAFF60B10B6A4A69CC68D05C37
:10A3D0000133B3FBF4F204FB1233C0B20B6210BDC5
:10A3E000184610BD90F8433830B53BB990F8411885
:10A3F00090F842380124DAB2914200D830BDB0F86A
:10A400004A5804FA03F22A43A0F84A280133F2E733
:10A410002DE9F04118468CB01C460E46154625F035
:10A42000CBFA1E28A8BF1E201A4F8DF80D500246E9
:10A4300003230546214604A800248DF80E608DF8FC
:10A440000C308DF80F40144E27F03CFD07F11E0232
:10A45000B62300970435204601920293335906EB48
:10A4600004082A4603A9CC346BB11B79142B0AD0FB
:10A47000009827F027FD009B00972B444046694633
:10A4800001931EF0AFFAB4F5197FE7D10CB0BDE827
:10A49000F08100BFA0280020AC5800202DE9F04139
:10A4A0008EB0002401A817460D468DF804308DF8B3
:10A4B000054025F081FA1E28A8BF1E201A4E8DF8EF
:10A4C000157002460323074601A906A88DF814302B
:10A4D0008DF816508DF81740DFF8508027F0F2FC09
:10A4E00006F11E02B6230437204602960392049317
:10A4F00058F8043008EB04053A4605A9CC346BB192
:10A500001B79142B0AD0029827F0DCFC029B0296E0
:10A510003B44284602A903931EF064FAB4F5197F60
:10A52000E6D10EB0BDE8F081A0280020AC58002094
:10A53000F0B5114E114D85B006F11E02B623002470
:10A54000019602920393204602272B592A19CC34F4
:10A5500063B11B79142B09D0019B1F70019B0196DD
:10A560000133104601A902931EF03CFAB4F5197F9D
:10A57000EBD105B0F0BD00BFA0280020AC580020F2
:10A58000F0B5114E114D85B006F11E02B623002420
:10A59000019602920393204601272B592A19CC34A5
:10A5A00063B11B79142B09D0019B1F70019B01968D
:10A5B0000133104601A902931EF014FAB4F5197F75
:10A5C000EBD105B0F0BD00BFA0280020AC580020A2
:10A5D000F0B5114E114D85B0002406F11E02B623D0
:10A5E000019602920393204627462B592A19CC3410
:10A5F00063B11B79142B09D0019B1F70019B01963D
:10A600000133104601A902931EF0ECF9B4F5197F4D
:10A61000EBD105B0F0BD00BFA0280020AC58002051
:10A62000F0B5114E114D85B0002406F11E02B6237F
:10A63000019602920393204627462B592A19CC34BF
:10A6400063B11B79142B09D0019B1F70019B0196EC
:10A650000133104601A902931EF0C4F9B4F5197F25
:10A66000EBD105B0F0BD00BFA0280020AC58002001
:10A670000B4B1B7810B504460BB9FAF77DFC094B60
:10A68000094A9B78126813F0400F517814BF1023C9
:10A690000D230B44237113781E33637110BD00BF6B
:10A6A00096260020AA0000206087002073B590F84D
:10A6B0005338032B04460D461ED10023124E8DF84D
:10A6C00007309DF8073094F854289A4201D802B018
:10A6D00070BD9DF8073006EBC303D3F8280245B1DF
:10A6E0000BF0CCFB9DF807300133DBB28DF807305F
:10A6F000E7E70BF0BDFBF5E7406B11B10BF0BEFBDC
:10A70000E5E70BF0B5FBE2E7982600202DE9F04FD6
:10A71000654F3B7883B013B9644B1C781CB10020A3
:10A7200003B0BDE8F08F012308203B7023F0BCFC90
:10A730005F4B604E1868DFF88C810BF099FB80202E
:10A7400023F088FC204623F085FC594B044618680A
:10A750000BF094FB022023F0A7FCB378D8F800207C
:10A76000A3423DD0FAF762FC534DB6F80080B5F82D
:10A770009032002214464FF0050B4FF0060A4FF0BE
:10A780000709EE18E85C96F89412814203F1010E75
:10A7900004F1050113D005EB010C291986F8940288
:10A7A0001E0A81F874B481F876A481F8773481F8B0
:10A7B000789481F87564013206348CF874041FFAB9
:10A7C0008EF3984502F1010234D9632AD9DDA5F848
:10A7D00090329CBB002300203B7003B0BDE8F08F9B
:10A7E000364B354D1C78002CBFD1D5F88832D31AA2
:10A7F000B3F57A7FB9D90820019223F055FC2C4B90
:10A8000018680BF035FBA02023F024FC204623F031
:10A8100021FC274B814618680BF030FB022023F007
:10A8200043FC19F0040F019A21D0C5F88C42C5F8F9
:10A8300088229AE70023A5F89032CAE7082023F07F
:10A8400033FC1B4B18680BF013FB1D4B013C1D190F
:10A850005C1E14F8010F23F0FDFBA542F9D1144B47
:10A8600018680BF00BFB022023F01EFCB2E709F086
:10A870000503012B11D0002BD9D1B3785B06D6D5B7
:10A88000D5F88C12D8F8003059B15B1A642BCED9A8
:10A890000192FAF7CBFB019AC9E7B3785906EFD5D5
:10A8A000C5E7C5F88C32C2E796260020972600201F
:10A8B00070870020AA0000209826002074870020BE
:10A8C0000C2B00204488002064292DE9F84328BF80
:10A8D00064212F4B11FB00F983FB09235B09074619
:10A8E0005FFA83F89BB12B4D00262B4C14F8012BFB
:10A8F00040213C2023F080F9AC42F7D10136002200
:10A9000040213C2023F078F9F3B29845EDD8474533
:10A910001ED808F10103DBB29F4217D9023FA7EB13
:10A920000807FFB21D4D013700261D4C14F8012BFE
:10A9300040213C2023F060F9A542F7D101360022E6
:10A9400040213C2023F058F9BE42EED1BDE8F88307
:10A95000144C154A84FB0934E408C8EB8813663CA0
:10A96000C8EB83031C44E4B2203C04EB8404651D63
:10A970001544144414F8012B40213C2023F03CF9E9
:10A98000AC42F7D1002240213C2023F035F9C0E74A
:10A990001F85EB511857030813570308FF56030888
:10A9A000FA56030867666666985403089E4B1B6850
:10A9B00023B193F90830002B00DD70472DE9F04FEB
:10A9C0009A4CD4F8E4362DED028BC31A002B87B0D5
:10A9D0002CDB974B94F8E8261B7803F00403002B3C
:10A9E000059300F5433314BF0121002103F5A07343
:10A9F00084F8E816C4F8E4361DD0012A16D08D4F2D
:10AA000001237A783B707B70FB78BA708A4D23F013
:10AA100002030544AE2280213C20FB70BD6023F080
:10AA2000EBF8002840F01C81844B187007B0BDEC97
:10AA3000028BBDE8F08F7F4FFB7822B1BA787A7035
:10AA400043F00203FB709D071BD4BA68821A002AE8
:10AA500002DBD90700F160810023DFF8E0813B7061
:10AA600098F80030002BE1D07B78072B4DD8DFE839
:10AA700013F056014C009C015504D70393021F02AA
:10AA8000CA0101223A70DA07C0D53A796C496D4D96
:10AA90000132D2B2A1FB0261890801EB4101A2EBB4
:10AAA0004102D2B23A71AA5C7A70AFE703462344FE
:10AAB0000022284683F8CC2602F0F1FC94F8CC66FC
:10AAC000CEB1614F614D203E06EB860606F10509C9
:10AAD000A9442E4416F8012B40213C2023F08CF889
:10AAE000B145F7D1002240213C2023F085F817F82A
:10AAF000016F002EE7D114F0CDFA0546404602F072
:10AB0000CEFC29461520FFF7DFFE059B002B8DD1DB
:10AB10004F4B4E4D93F82030052B9CBF494A9B1854
:10AB20004FF0800198BF93F834604FF0B0024FF0BF
:10AB30003C0094BF203E1F2623F05EF80C228021AB
:10AB40003C2023F059F8162280213C2006EB860693
:10AB500023F052F8771D2F442E4416F8012B402184
:10AB60003C2023F049F8BE42F7D1002240213C208E
:10AB700023F042F8B02280213C2023F03DF802224D
:10AB800080213C2023F038F8172280213C2023F03C
:10AB900033F8304A304B12781B78002A14BF522603
:10ABA0000126002B18BF322606EB8606771D2F44A0
:10ABB0002E4416F8012B40213C2023F01DF8B7420B
:10ABC000F7D1002240213C2023F016F8B02280214A
:10ABD0003C2023F011F8082280213C2023F00CF8BF
:10ABE000172280213C2023F007F894F8E9261B4B1C
:10ABF000D35C203B03EB83035E1D2E441D4415F8FC
:10AC0000012B40213C2022F0F7FFB542F7D1002272
:10AC100040213C2022F0F0FF94F8E936013303F0A4
:10AC2000030384F8E93601E75087002098260020C6
:10AC30001B8E002054870020404B4C004087002092
:10AC4000ABAAAAAAAC510308642D002098540308AB
:10AC50001C8E0020D88D0020704600202080030824
:10AC600002F06AFBDFF8248388F8000000283FF434
:10AC7000DDAEB02280213C2022F0BEFF40228021A8
:10AC80003C2022F0B9FF002280213C2022F0B4FFBA
:10AC9000102280213C2022F0AFFF4FF48065013D5F
:10ACA000002240213C20ADB222F0A6FF002DF6D1BB
:10ACB000B02280213C2022F09FFF2A4680213C20A8
:10ACC00022F09AFF102280213C2022F095FF9E4B1B
:10ACD0007A7803EB8203D3F8089099F80060002E8D
:10ACE0003FF4BEAE994D203E06EB860606F1050AFE
:10ACF000AA442E4416F8012B40213C2022F07CFF70
:10AD0000B245F7D1002240213C2022F075FF19F80E
:10AD1000016F002EE7D1A3E601223A70B5E68C4B15
:10AD20008C4A8D498D480CF081F8012002F0B7FB68
:10AD300094F8CC66002E00F07185884F834D203E3C
:10AD400006EB860606F10508A8442E4416F8012BEA
:10AD500040213C2022F050FFB045F7D10022402195
:10AD60003C2022F049FF17F8016F002EE7D10220A6
:10AD700002F095FB7A4F5626203E06EB860606F13A
:10AD80000508A8442E4416F8012B40213C2022F04F
:10AD900033FFB045F7D1002240213C2022F02CFFA8
:10ADA00017F8016F002EE7D1AFE66E4F3B689A07A8
:10ADB00000F1DC844FF0020801251F057FF5A5AEE8
:10ADC000694B6A481B686A4A0068009082FB03204E
:10ADD000DA17C2EB6012642000FB123365495F484A
:10ADE0000CF024F85D4824F0E7FDC0B214283FF6CB
:10ADF0005DAE2021431CDBB22218152B184682F8C9
:10AE0000CC16F7D153E6DFF888A1DFF850914FF068
:10AE100000083AF9023B5849424648460CF006F809
:10AE2000484624F0C9FDC0B2142800F2AB832021AB
:10AE3000431CDBB22218152B184682F8CC16F7D12A
:10AE40002344A8F14F020025D2B280213C2083F890
:10AE5000CC5622F0D1FE2A4680213C2022F0CCFEA6
:10AE6000102280213C2022F0C7FE94F8CC56CDB1B0
:10AE70003A4F364E203D05EB850505F1050BB344F1
:10AE8000354415F8012B40213C2022F0B5FE5D45EC
:10AE9000F7D1002240213C2022F0AEFE17F8015FDE
:10AEA000002DE7D108F10108B8F1040FB1D12CE66B
:10AEB000012002F0F4FADFF8DC80244D5426203E15
:10AEC00006EB8606771D2F442E4416F8012B4021F1
:10AED0003C2022F091FEB742F7D1002240213C20D5
:10AEE00022F08AFE18F8016F002EE8D1234B9FED67
:10AEF000248A186837464FF001094FF0020AA84625
:10AF0000204BFAB23426002806FB02360FDD1E4B1A
:10AF10001B68B34200F080821B49002304E051F813
:10AF2000045FAE4200F0748201338342F7D1B9F17D
:10AF3000130F3FF6EAAD114B186809F101095FFAEA
:10AF400089F90137DCE700BFAC51030898540308C6
:10AF5000549003087C7603084C7F0308642D00207E
:10AF6000B0760308B47E002058240020304500202D
:10AF70001F85EB51707F030814800308A045002053
:10AF800000247449A41800203C450020408700207C
:10AF900014880020347F0308D14BD24993F8D02580
:10AFA000D1480BF043FF012002F079FA94F8CC6607
:10AFB000CEB1CD4FCD4D203E06EB860606F10508FD
:10AFC000A8442E4416F8012B40213C2022F014FE08
:10AFD000B045F7D1002240213C2022F00DFE17F8A9
:10AFE000016F002EE7D1C24BDFF820B31B684FF092
:10AFF000B20803F1FF3919F8013F5BF8042B99F807
:10B000001410019199F80A100091B748B9490BF052
:10B010000DFFB54824F0D0FCC0B2142800F2FC8328
:10B020002021431CDBB22218152B184682F8CC16BF
:10B03000F7D123440025424680213C2083F8CC569A
:10B0400022F0DAFD2A4680213C2022F0D5FD102294
:10B0500080213C2022F0D0FD94F8CC56CDB1A24FF7
:10B06000A24E203D05EB850505F1050AB2443544A5
:10B0700015F8012B40213C2022F0BEFDAA45F7D156
:10B08000002240213C2022F0B7FD17F8015F002D7F
:10B09000E7D108F101085FFA88F8B8F1B50FAAD135
:10B0A000954B964993F800908F484A460BF0BEFEA8
:10B0B000052002F0F4F994F8CC66CEB18A4F8B4D9E
:10B0C000203E06EB860606F10508A8442E4416F835
:10B0D000012B40213C2022F08FFDB045F7D100220A
:10B0E00040213C2022F088FD17F8016F002EE7D1A7
:10B0F00074237B4A82497C4803FB09F31A4492F883
:10B10000C0844FEA480A0AEB080203EB8203744A40
:10B110001A4492F8C23492F8C4240BF087FE7248A5
:10B1200024F04AFCC0B2142888BF034608D8202166
:10B13000431CDBB22218152B184682F8CC16F7D127
:10B1400023440022062083F8CC2602F0A8F994F8C4
:10B15000CC36D3B1644F654D1E46203E06EB8606C5
:10B1600006F1050BAB442E4416F8012B40213C2080
:10B1700022F042FDB345F7D1002240213C2022F0CD
:10B180003BFD17F8016F002EE7D17420544B5D4949
:10B19000D04400FB09F000EB8800184490F8C83454
:10B1A00090F8C72490F8C90400904F480BF03EFE79
:10B1B0004D4824F001FCC0B2142888BF034608D8CB
:10B1C0002021431CDBB22218152B184682F8CC161E
:10B1D000F7D123440022072083F8CC2602F05FF940
:10B1E00094F8CC66002E3FF490AC3F4F3F4D203E8C
:10B1F00006EB860606F10508A8442E4416F8012B36
:10B2000040213C2022F0F8FCB045F7D1002240213B
:10B210003C2022F0F1FC17F8016F002EE7D174E416
:10B22000DFF8ECA09AF80030002B3FF46EAC4FF042
:10B23000410BDFF8E090DFF8E0802C4D00265F4600
:10B2400072084F3AD2B280213C2022F0D5FC002275
:10B2500080213C2022F0D0FC203F102280213C2085
:10B2600007EB870722F0C8FC07F1050BAB442F441E
:10B2700017F8012B40213C2022F0BEFCBB45F7D142
:10B28000002240213C2022F0B7FC38F9023C1E4944
:10B29000B3F5FA6FA8BF4FF4FA63B3F57A7FB8BF7E
:10B2A0004FF47A73A3F57A7381FB0321DB17C3EBA9
:10B2B000A101C9B20920FFF707FB9AF80030B34299
:10B2C00000F21D810236F6B29E42BFF41EAC0E2E75
:10B2D00008F104083FF419AC19F8027FB0E700BF89
:10B2E00094610020A47F0308642D00209854030873
:10B2F0008C410020B07F03080D8E0020C87F03081A
:10B30000DC7F0308F07F030867666666D451030894
:10B3100060880020D85D030876880020012002F0B4
:10B32000BEF8C14FC14D2026203E06EB860606F131
:10B330000508A8442E4416F8012B40213C2022F099
:10B340005BFCB045F7D1002240213C2022F054FCA8
:10B3500017F8016F002EE7D1DFF8FC82D8F8003033
:10B360009E0700F17B814FF003090227D80700F107
:10B370000B81190700F1B681AD48AE49B0F9042040
:10B38000B0F90030B0F90200009081FB0201D21741
:10B39000C2EBA10212B20192A749A84AA8480BF039
:10B3A00045FDA74824F008FBC0B2142800F23982FA
:10B3B0002021431CDBB22218152B184682F8CC162C
:10B3C000F7D123440022384683F8CC2602F067F8F0
:10B3D00094F8CC66002E3FF498AB994F203E06EBD4
:10B3E000860606F10508A8442E4416F8012B4021D4
:10B3F0003C2022F001FCB045F7D1002240213C2046
:10B4000022F0FAFB17F8016F002EE7D1FFF77DBBA2
:10B410008C49342303FB02139E6AD3F82CE093ED8E
:10B42000097A052A4FEA56163FF487ADB8EE477AF7
:10B4300041F2883CC8EE077A7346009682498048FC
:10B44000FDEEE77A17EE905A06FB05C60EFB05CE19
:10B450007E4DA5FB06567D4DA5FB0EE5760B6D0BCF
:10B46000029601950BF0E2FC754824F0A5FAC0B2F3
:10B47000142800F285802021431CDBB22218152BF2
:10B48000184682F8CC16F7D12344AAF150020025C1
:10B49000D2B280213C2083F8CC5622F0ADFB2A4664
:10B4A00080213C2022F0A8FB102280213C2022F0A9
:10B4B000A3FB94F8CC660AF1010A5FFA8AFAC6B1D6
:10B4C0005F4D203E06EB860606F1050BC34446445D
:10B4D00016F8012B40213C2022F08EFBB345F7D11A
:10B4E000002240213C2022F087FB15F8016F002E3E
:10B4F000E7D1BAF1080F7FF61AADFFF706BB4B4F45
:10B5000007F1050B17F8012B40213C2022F074FBBA
:10B51000BB45F7D1002240213C2022F06DFB99F879
:10B520000170203F07EB870707F1050BAB442F4461
:10B5300017F8012B40213C2022F05EFBBB45F7D1E0
:10B54000002240213C2022F057FBB8F90030394955
:10B55000B3F5FA6FA8BF4FF4FA63B3F57A7FB8BFBB
:10B560004FF47A73A3F57A7381FB0321DB17C3EBE6
:10B57000A101C9B20920FFF7A7F99AF80030A1E6A6
:10B58000034681E703465BE4314E96ED130A26F04D
:10B59000C5FE96ED140A824626F0C0FE96ED150A09
:10B5A000834626F0BBFE534601902A4A2249CDF835
:10B5B00000B023480BF03AFC214824F0FDF9C0B25A
:10B5C000142800F234812021431CDBB22218152BF1
:10B5D000184682F8CC16F7D123440022384683F867
:10B5E000CC2601F05CFF94F8CC66C6B1144F203E27
:10B5F00006EB860606F1050AAA442E4416F8012B2E
:10B6000040213C2022F0F8FAB245F7D10022402137
:10B610003C2022F0F1FA17F8016F002EE7D1D8F89C
:10B6200000304F46A5E600BF1C7F0308985403086E
:10B63000D0600020676666668C7F0308A07F0308E1
:10B64000642D0020A4180020048003085917B7D1E6
:10B65000CC8900209C7F0308248A00207649774A01
:10B660000B6B886B496B00910190754975480BF025
:10B67000DDFB744824F0A0F9C0B2142800F2D58094
:10B680002021431CDBB22218152B184682F8CC1659
:10B69000F7D123440022022083F8CC2601F0FFFEDC
:10B6A00094F8CC66C6B1674F203E06EB860606F1DD
:10B6B0000509A9442E4416F8012B40213C2022F014
:10B6C0009BFAB145F7D1002240213C2022F094FAA8
:10B6D00017F8016F002EE7D1D8F800304FF00409B9
:10B6E000032743E65849594ACB68486909690091DC
:10B6F0000190534953480BF099FB524824F05CF9F0
:10B70000C0B2142800F28F802021431CDBB2221823
:10B71000152B184682F8CC16F7D1234400217A1C49
:10B72000384683F8CC16D7B201F0B9FE94F8CC664F
:10B73000002E3FF421AEDFF80C81203E06EB86069A
:10B7400006F10509A9442E4416F8012B40213C209E
:10B7500022F052FAB145F7D1002240213C2022F0DC
:10B760004BFA18F8016F002EE7D105E6384B39483F
:10B770001B88394A00780090A2FB0302D20802EB32
:10B780008200A3EB400335492E489BB20BF04EFBE1
:10B790002C4824F011F9C0B214284AD82021431CA7
:10B7A000DBB22218152B184682F8CC16F7D12344A9
:10B7B0000022012083F8CC2601F071FE94F8CC66BB
:10B7C000D6B1DFF88080264D203E06EB860606F1D6
:10B7D0000509A9442E4416F8012B40213C2022F0F3
:10B7E0000BFAB145F7D1002240213C2022F004FAA7
:10B7F00018F8016F002EE7D113F04CFC054602202B
:10B8000001F04DFE29461520FFF75EF84FF00408C1
:10B810003B680325FFF7D1BA03460AE4104DFFF752
:10B82000A6BA0346CDE5034677E7034631E703466C
:10B83000D2E60346BBE700BF8C890020887F03085F
:10B840008C7F0308642D0020505200204C94030884
:10B8500034450020B87E0020CDCCCCCC587F0308E6
:10B860009854030810B50C4604F01CFF03228271A3
:10B870000022C2712146BDE810400AF03DB910B562
:10B880000446007910B10121FFF7ECFF63792168CC
:10B890009A0802239340C868DB439BB20340CB6005
:10B8A00010BD10B50446007910B12221FFF7DAFF70
:10B8B00063792268990802238B40D94389B21161C8
:10B8C000D1689BB20B43D36010BD044B1B681BB106
:10B8D0001B685B6803B11847FF2070473C87002056
:10B8E0001FB50123ADF80830ADF80410002301A9FD
:10B8F000ADF80A30ADF80C30ADF8062017F036FC84
:10B9000005B05DF804FB70B5A0F6580494F845380E
:10B91000C3B1B4F84C3801339BB2082BA4F84C38AF
:10B9200040F29180002384F84538A4F84C38A36B8A
:10B93000022259791868FFF7D3FF94F84538002B95
:10B9400040F08180404D95F8EA361BB90121204630
:10B95000FEF7ACFE94F8443853BBA36A626A9A427D
:10B9600003D1002385F8EA3670BD95F8EA26022A4D
:10B9700012D802F1010214BFFF237F2385F8EA26C3
:10B98000A4F84838082384F84638012384F844385A
:10B99000A06BBDE8704072E75A1CA169A262CB5C43
:10B9A00021698A4228BF0022DBB228BFA262E7E7F2
:10B9B00094F94638002B3CD094F8481811F0010156
:10B9C00027D095F8EB66012E03D801212046FEF71B
:10B9D0006DFE023E012E03D800212046FEF766FED2
:10B9E00095F8EB360133DBB2032B85F8EB362AD919
:10B9F000B4F848385B08A4F8483894F84638013B56
:10BA00005BB2002284F8463885F8EB26002BA4D0E0
:10BA100070BD95F8EB3613F0FD0304D101212046EB
:10BA2000FEF744FEDCE7012BDAD12046FEF73EFEAE
:10BA3000D6E7616AA26A914205D184F84438A06BC6
:10BA4000BDE870402DE770BD982600202DE9F04F2D
:10BA5000164685B080460C4622F088FB04F08CFA2E
:10BA6000022E09D0042E0AD0022E4FF4964508D19A
:10BA7000FF2C06D1032629E04FF41645F8E744F6DB
:10BA8000C0150023C6498DF80D3014209DF80D30E7
:10BA9000072B01D900230AE09DF80D3000FB0313AA
:10BAA000DB79DA0740F1A1809DF80D30DBB2611E31
:10BAB0001944C9B2072900F20582032E06D0B84BFB
:10BAC00001EB810103EB8101B64B9963B54CB64B99
:10BAD000B34A236004F13C0003234FF48061637197
:10BAE0006061002304F588600127032E84F8536801
:10BAF000C4F83C24A560A371E362E1602362E361C2
:10BB0000A0612161A362636284F8443884F84078BC
:10BB100084F84138A4F84E38A4F85038A4F84C38CA
:10BB200084F8523891460DD0D4F838A09AF8040021
:10BB300004F0B8FD60635046FFF7B3FE3946204677
:10BB4000FEF7B4FD322006F045FC002E54D1D4F8A7
:10BB50003C54286817F0EAFB28460122222106F00F
:10BB60004FF8924BC4F8583832469149284605F0B0
:10BB7000A1FFA56B286817F0D9FB01224FF6FF71D2
:10BB8000284606F03DF8022269792868FFF7A8FEEA
:10BB9000884BC4F85C3832468749284605F08AFF4E
:10BBA000864D4FF0060AC5F8EC464FF0050B022E05
:10BBB0000FD0D5F8EC0604F0D7F950B122F0E6FA30
:10BBC000D5F8EC0604F0D0F9002840F0B18022F05E
:10BBD000CDFA404604F0C8F9002840F07681042EE2
:10BBE000E7D0052006F0F6FBE1E79DF80D200132D5
:10BBF000D2B28DF80D2049E7012E08D1D4F83C04CB
:10BC000029461FF008FCA06B1FF034FCC8E7022E89
:10BC100008D1A06BFFF733FE2946D4F83C041FF08F
:10BC2000FAFBBDE7032E7CD1002784F8547860220C
:10BC300039466348DFF88CA128F07BFC8DF80E7044
:10BC40009DF80E200B2A09D901215648FEF72EFD3A
:10BC50002946D4F83C041FF0DEFBA1E79DF80E2036
:10BC600002EB82020AEB8202127B002A4BD09DF883
:10BC70000E2002EB82020AEB82021269002A42D0F5
:10BC800000228DF80F204FF0140B9DF80F20072A8B
:10BC900028D89DF80E709DF80F20FFB20BFB029282
:10BCA00007EB870710790AEB870704F0FBFC3A697A
:10BCB00082422FD19DF80F0000EB800009EB80003D
:10BCC000FFF7DDFD9DF80F200BFB029B9BF8072083
:10BCD000930707D594F85428384B03EBC20201218F
:10BCE00082F82C129DF80E2094F85418334B02EB76
:10BCF00082020AEB820203EBC1001269C0F828221B
:10BD0000013184F854189DF80E200132D2B28DF81A
:10BD10000E2095E79DF80F200132D2B28DF80F204A
:10BD2000B3E7042E7FF43CAFA06BFFF7A8FD65E7F7
:10BD3000D5F8EC0604F014F90146404604F018F971
:10BD40003EE7404604F00CF995F8FE360746ABB9DD
:10BD5000242802D1012385F8FE36012E03D139466D
:10BD6000404604F005F93946D5F8EC0604F000F930
:10BD7000404604F0F9F80028E3D130E7012B06D162
:10BD80004D280CBF0223002385F8FE36E5E7022B81
:10BD90001AD13C280CBF0323002385F8FE36DCE7CC
:10BDA00044740308DC7E0020E851030807B900084A
:10BDB00034870020D1BE0008388700209826002054
:10BDC000C0280020E88C0020032B10D10A2802D9BB
:10BDD00085F8FE96C1E7042385F8F10685F8F0960C
:10BDE00085F8F39685F8F20685F8FE36B5E7042B5C
:10BDF00009D195F8F23685F8FF06434085F8F2360A
:10BE000085F8FEB6A9E7052BA7D195F8F03695F889
:10BE1000F12695F8F216934209D25A1C2B44414060
:10BE200085F8F21685F8F02683F8F40695E7814246
:10BE3000CED195F8FF3685F8FEA6F42B8DD1002AD9
:10BE40008BD12421404685F8FE26019204F090F81B
:10BE50004D21404604F08CF83E21404604F088F81D
:10BE6000019A4046114604F083F8F421404604F05C
:10BE70007FF8F421404604F07BF8032E18D0A26B23
:10BE800053791168980802238340DB439BB20B610E
:10BE9000C8680340CB60107910B12021FFF7E2FCA5
:10BEA000A06B00211EF0DEFDA36B186817F03EFAB0
:10BEB000D4F83C0400211EF0D5FDD4F83C341868B9
:10BEC00017F034FA05B0BDE8F08F4FF000094FE7E6
:10BED00038B5A0F65C04A1F12905A36B186800220F
:10BEE000302D4262324D31D895F800370133DBB244
:10BEF000012B89BFB4F84A3885F800375B08A4F8ED
:10BF00004A3881BF95F8013785F80027013385F855
:10BF1000013795F801270023082AA4F84C3814D1DA
:10BF200085F80137B5F8023701339BB2032BA5F82A
:10BF3000023707D96379DB0704D5E36A94F84A0826
:10BF400053B398470023A4F84A3838BD5B396C29AD
:10BF50000ED8B4F84A3885F800275B0843F0800310
:10BF6000A4F84A3895F80137013385F80137D0E74E
:10BF700094F84528002ACCD1012184F8451885F889
:10BF800001178021A4F84A18597985F80027A5F8E7
:10BF90000227FFF7A5FCBCE7E3696269D054E369B7
:10BFA000E1680133B3FBF1F201FB1233E361C9E74E
:10BFB0009826002038B5A0F65C046379DB074AD5E3
:10BFC000A57994F8403805F0010503B3D4F83C3462
:10BFD0001A68D36A5B08536294F8443823B1B4F802
:10BFE0004E380133A4F84E38A36B6A0059791868AB
:10BFF000FFF776FC012384F84338002384F84138A6
:10C0000084F8423884F84038A4F84A3838BD94F8A7
:10C010004338012B04BF94F8413884F84238204655
:10C02000FEF7E0F994F84328A36B4AB9012284F89B
:10C0300043285979186805FA02F2BDE838404FE400
:10C04000002284F8432895425979186808BF0222D3
:10C05000BDE8384044E438BD10B5A0F6580494F863
:10C0600045381BBB94F844288ABBA36A616A99428D
:10C070001CD0591CA069A162C35C2069DBB25B00C3
:10C0800043F40073A4F848380A2384F8463801239F
:10C0900084F8443894F85338814228BFA262012BB7
:10C0A00001D0042B02D1A06BFFF7E9FB94F84038D4
:10C0B000002B73D194F841380133DBB2092B84F89B
:10C0C000413827D12046BDE81040FEF78BB994F9DE
:10C0D00046387BB1B4F848184B08A4F8483801F04A
:10C0E00001012046FEF7E2FA94F84638013B84F855
:10C0F0004638DBE784F84438626AA36A9A42D5D1AD
:10C1000094F85338012B01D0042BCFD1A06BFFF74B
:10C11000C8FBCBE70A2B41D194F843382BB9B4F8CC
:10C120004A3843F00103A4F84A386379D9070AD59D
:10C13000B4F84A08820501D4C3071DD4B4F85038B6
:10C140000133A4F85038012284F8402894F8432899
:10C150000023012A84F8413820D1A27984F8433899
:10C16000A36B12F0010F0CBF02220022597918684C
:10C17000BDE81040FFF7B4BBE36AC0F347000BB162
:10C180009847E0E7E3696269D054E369E168013305
:10C19000B3FBF1F201FB1233E361D4E710BD00BF42
:10C1A0002DE9F04F7F4BDFF818E293F8048793F8FE
:10C1B00005A793F806777C4EDFF808924FF0000C45
:10C1C00001259EF802309EF80320C3F1FF039BB2C5
:10C1D000002B00F0DD80BEF80010C3F1FF03A9FBC7
:10C1E000014002FB03F340091B121446052800F22C
:10C1F000D580DFE800F0BDA48F765E03A9FB014087
:10C200004009C0EB0010A1EB800189B2D71AC1F13F
:10C210003C0107FB01F75FFA83FAA9FB07170AEB5A
:10C2200057179046FFB21C463A4643461B0243EA64
:10C23000044414431723624605FA03F1214214BF54
:10C2400011200920511C013BB0548AB2591CF3D172
:10C25000564B0EF1040E0CF1180C73451FFA8CFCB2
:10C26000AFD1534B4F4A4F4C52481B7882F804874A
:10C270004FF44071202284F805A784F806770570F2
:10C28000A4F80817A4F80A278BB14B4B4B4A19683E
:10C290001268002340F22A3050604B620B889BB238
:10C2A00043F001030B80136843F001031360BDE802
:10C2B000F08FA9FB01404009C0EB0010A1EB800802
:10C2C0001FFA88F8D11A08FB01F85FFA83FAA9FB74
:10C2D00008180AEB58185FFA88F81C4617464346B8
:10C2E000A4E7A9FB01404009C0EB0010A1EB8001CD
:10C2F00089B2C1F13C01A2EB030A0AFB01FAA9FBD6
:10C300000A1A5FFA83F808EB5A1A5FFA8AFA174694
:10C3100054468BE7A9FB01704009C0EB0010A1EB6C
:10C320008007BFB2D11A07FB01F7A9FB07175FFA15
:10C3300083F808EB5717FFB292463A4676E7A9FB17
:10C3400001704009C0EB0010A1EB800189B2A2EBA3
:10C350000308C1F13C0108FB01F8DFB2A9FB081892
:10C3600007EB58185FFA88F892461A4643465DE78D
:10C37000A2EB030A01FB0AFADFB2A9FB0A1A07EBD8
:10C380005A1A90465FFA8AFA1A46544643464DE7CF
:10C390001746144692469046134647E7544643468E
:10C3A0003A4643E798260020503E0020243E0020D5
:10C3B000884100202E3E00207C4100208441002046
:10C3C000A43D002089888888074B9FED087A1B7858
:10C3D00007EE903AF8EEE77A054B67EE877A002091
:10C3E000C3ED367A704700BFA42D0020CDCCCC3DE4
:10C3F00094610020074B084AD3ED367AB2EE047AF6
:10C4000067EE877A0020FCEEE77A17EE903A137019
:10C41000704700BF94610020A42D002030B1007946
:10C4200010F1FF3018BF4FF0FF3070474FF0FF3072
:10C430007047064B5A7832B9054A528802F0010219
:10C440009A7001225A700020704700BFA42D00206E
:10C45000B47E0020094A0A49D378742000FB0313F4
:10C460009188A3F89414D188A3F89814118952895B
:10C47000A3F89A14A3F8962400207047A42D002056
:10C4800094610020094A0A49D378742000FB031301
:10C490000020B3F894149180B3F89814D180B3F8C5
:10C4A0009A14B3F89634118153817047A42D00205B
:10C4B000946100200D4B0E491A7B30324A70DA78B5
:10C4C0000C49742000FB0212002092F8B514597335
:10C4D00092F8B414997392F87B14D97392F8851476
:10C4E00092F88F2419745A74704700BFA42D00204D
:10C4F000B0000020946100200C4A0D49137BD078D5
:10C5000030330B71937C30338B7192F8203074216F
:10C5100041430C2000FB031306490B44002019681B
:10C520005161596891619968D1617047A42D0020CB
:10C53000B0000020566600200B4BD87893F82010EE
:10C54000742242430C2000FB01220849114453F895
:10C55000142FC1F8C2245A68C1F8C6249A68C1F8D9
:10C56000CA240020704700BFA42D00209461002041
:10C5700010B50C4A0C49137BD07830334B700B4903
:10C58000742300FB03132132002113F8010F885498
:10C5900050189C7A447003311C7D84700929F4D1B1
:10C5A000002010BDA42D0020B00000200766002050
:10C5B000034A937C013B82F820300020704700BF83
:10C5C000A42D0020024A137B013BD370002070474A
:10C5D000A42D0020064A0749D37881F8D03574206D
:10C5E00000FB031392F8202083F8C024002070473A
:10C5F000A42D0020946100200849094A91F8D03503
:10C60000D370581C1073742000FB0313002093F8A0
:10C61000C03482F820300133937470479461002055
:10C62000A42D00200023044A194699540133072BF6
:10C63000FBD10020704700BFCE2D002070B5194BF4
:10C640001B78012B18D8184B93F83150174B93F8DF
:10C650007B1683F87D5621B193F87C260AB191426E
:10C660000CD3012283F87B2683F87C2625B1022D8A
:10C670001CBF002283F87D26002070BD14460846AA
:10C6800034B190FBF4F604FB160620463446F7E777
:10C6900091FBF0F192FBF0F283F87B1683F87C2695
:10C6A000E4E700BF48950020A42D002094610020FD
:10C6B00030B50D4B5A6B002115794C1C0E2DE4B290
:10C6C0000ED1027883F83810501E8842DCBF023A3F
:10C6D00083F8382093F83820013A83F8382030BDA9
:10C6E00014322146E8E700BFA42D002070B544694C
:10C6F000054623790E2B04D12B694BB1BDE8704060
:10C700001847032B02D1E068FFF7F0FF1434F0E77D
:10C7100070BD064B30B11A69186001321A610522EA
:10C720001A75704704221A75704700BF3C7D0020BF
:10C7300008B5084B5A7832B19B7833B1064A9368F2
:10C7400043F480339360002008BD4FF4803009F03B
:10C7500017FEF8E7A42D00209461002008B5094BCE
:10C7600093F839203AB193F83A3033B1064A9368D6
:10C7700043F400239360002008BD4FF4002009F02B
:10C78000FFFDF8E7A42D00209461002070B50F4C48
:10C790000F4DE278637B742606FB025282F8B534B3
:10C7A000A37B82F8B4340B4B186816F00FFAE378C9
:10C7B000E27B06FB0353002083F87B24227C83F872
:10C7C0008524627C83F88F2470BD00BFA42D0020D7
:10C7D000946100208C41002010B50C490C4AC878A7
:10C7E000742300FB032321310022505C03F8010F66
:10C7F00088180332447880789C72092A1875F4D11D
:10C80000044B186816F0E2F9002010BDA42D00209A
:10C81000076600208C410020F7B5344E96F87D362F
:10C82000022B5AD116F0CCFB044640BB30493148AC
:10C83000314D27F0F6FE2346304F314A009508214E
:10C8400007F1430027F07EFE234600952C4A08217D
:10C8500007F14B0027F076FE96F87D3687F83130E9
:10C8600097F8393043B9274B1B68C3F3C04387F8A7
:10C870003A30012387F83930002003B0F0BD224D53
:10C8800095F8244034B921491A481B4D27F0C9FEB8
:10C890002346D1E71E4C6378022B14D0032B1AD108
:10C8A0001C49144827F0BDFE41F278134FF4FA6298
:10C8B000E4584FF47A23B4FBF3F4EB6B0E4DB3FB67
:10C8C000F2F31B1BB8E714490A480B4D002427F06C
:10C8D000A8FE2346B0E70D49F6E710490548104D7C
:10C8E000002427F09EFE2346A6E700BF94610020A7
:10C8F0006D800308DF2D00206A800308A42D00202E
:10C9000086800308B47E0020406100207580030803
:10C910000C6B00207B800308818003082C860308B1
:10C920006B800308244B5A6DD2682DE9F04105460F
:10C930001C4692BB94F8583063B3284609F0B8FB04
:10C9400094F85830013BDBB204EB830284F8583092
:10C950002344D76D93F884607B69636304354FFA91
:10C9600086F82846676584F85980FFF7A1FE94F899
:10C97000383098450EDD7A69C4F89020142103FB05
:10C980000111DB430A4433442846626384F859307A
:10C99000FFF78EFE0020BDE8F08193F959005B6B34
:10C9A00000EB800003EB800090470028C2DA4FF0D4
:10C9B000FF30BDE8F08100BFA42D0020F8B505468A
:10C9C00051B3164C606D81421AD094F85820144F20
:10C9D000616504EB8203A618D8654069636B1B1A76
:10C9E00094F859009B1007FB030386F8843000235A
:10C9F00084F859308B68013284F8582003B1984785
:10CA0000636D5B69636328460023C4F8903009F0C6
:10CA10004FFB281DFFF74CFE0020F8BDA42D002081
:10CA2000CDCCCCCC2DE9F04FBD4A81461068002812
:10CA300089B050DBBB4DD5F8942002F5434250320B
:10CA40004A4548D895F89880C5F894904FF47A7282
:10CA5000B9FBF2F20192B44AB8F1000F3ED1D3888B
:10CA6000A3F2E3439BB2B3F5F97F31D8B2F90410D6
:10CA700040F2E14399422BDCB2F9022040F2D66346
:10CA80009A4225DDA9490B7813F0040420D148B15E
:10CA9000A74A10680028B8BF1460126805EB82022C
:10CAA000D2F89C00C5F8AC0070B1012285F898203E
:10CAB00023F001039F4A0B706A6509F0EBFA696D78
:10CAC000D5F8AC00FFF77AFF9B4B4FF4FA721A844B
:10CAD000019BC5F8B03009B0BDE8F08FD188964F02
:10CAE000A1F2E34189B2B1F5F97F10D8B2F904009F
:10CAF00040F2E14188420ADCB2F9020040F2D6611C
:10CB0000884204DD89490978480740F18F83B2F9EA
:10CB1000020040F2D661884200F3AE8340F2E14465
:10CB2000A04240F3AB83B2F90000A04240F3A883D7
:10CB3000884200F3A7839288A2F2E24292B2B2F551
:10CB4000FA7F00F2A18301220024BA62C5F8B44042
:10CB50006FE3002C00F07983BA6AD5F8AC600292DA
:10CB600004F1FF3B4FF0000A5FFA8BFB029A52453B
:10CB700024DC033C012C3B8400F267837A6A142A8C
:10CB800040F36383A2F1140193FBF1F31BB2322B48
:10CB90003B8400F35A83D5F8B4300BB9C5F8B42000
:10CBA000D5F8B430D21A644B986A052192FBF1F2A1
:10CBB00002448A42C8BF0A469A6246E36B6D0BB9CB
:10CBC000FA238CE0052C05D13046FFF7ABFE4FF47D
:10CBD000FA7384E0022C46D195F9593095F8382043
:10CBE00093422DDA013385F85930BBF1010FE7D9B3
:10CBF00095F959306A6B03EB830302EB83031A79CF
:10CC0000013A0C2ADCD801A151F822F0C9CB000866
:10CC100005CD0008CDCC0008E5CC00083DCD0008CE
:10CC200011CE000893CD00083DCE00086DCE00085F
:10CC3000C1CB000893CD00085FCD0008D9CD000816
:10CC4000D5F890305BB1304609F032FAD5F8903023
:10CC50006A6BC5F89020301D6B63FFF729FD002338
:10CC600085F85930C1E7012CBFD195F859106A6B8E
:10CC70004B1E5BB203EB830002EB800085F859305A
:10CC8000007920B9002BC4BF023985F8591095F9F5
:10CC90005930591C06D003EB830302EB83031B7945
:10CCA000002B8DD1D5F890305BB1304609F000FAF9
:10CCB000D5F890306A6BC5F89020301D6B63FFF794
:10CCC000F7FC95F8383085F859308EE7042C7FF45E
:10CCD00077AFD9683046FFF771FE4FF4FA730AF167
:10CCE000010A43E79A68002A3FF46AAF042C7FF4F4
:10CCF00067AFD9683046904701303FF465AF4FF4D5
:10CD0000FA73ECE79A68002A3FF45AAF042C7FF4D8
:10CD100057AFD968304690474FF4FA73DFE700BF4A
:10CD2000C4300020A42D0020748800201B8E002019
:10CD3000B0170020B8000020B0000020DA68002AF8
:10CD40003FF43EAFA4F1040CDCF1000141EB0C0117
:10CD500011701A7C42F001021A74FA23BFE7D968F5
:10CD600000293FF42DAF042C0A8809D142F4006257
:10CD700092B20A801A7C42F001021A74FA23AEE7DA
:10CD800040F6010092FBF0F000EBC020121A92B2C4
:10CD9000EFE7DA68002A3FF413AF1168042C087833
:10CDA00012D192F805E0864502D9927910440870B4
:10CDB0001A7C42F001021A749A68002A3FF400AF0C
:10CDC000194630469047FBE692F804E08645EFD2DC
:10CDD0009279801A0870EBE7D8680268042C117801
:10CDE00011D10079884201D9013111709A6822B1BC
:10CDF000D968039330469047039B1A7C42F00102A6
:10CE00001A74FA236BE70029F0D001391170EDE7AD
:10CE1000DA68002A3FF4D4AE1168042C91F90000BE
:10CE200007D192F905E08645C2DD927902440A7085
:10CE3000BEE792F904E08645BADAC9E7DA68002A63
:10CE40003FF4BEAE1168042C088807D1B2F806E0A2
:10CE50008645ADD9128910440880A9E7B2F804E0EC
:10CE60008645A5D21289801A0880A1E7DA68002ACF
:10CE70003FF4A6AE1168042CB1F9000004D1B2F958
:10CE800006E0864594DDE5E7B2F904E086458FDAF1
:10CE9000E8E795F838203B799B1A022293FBF2F3DE
:10CEA000013BDBB20293D5F8BC3003F5C333A033AA
:10CEB00099453B6888BFC5F8BC909B6A384698BFC7
:10CEC0004FF000089847BB791FFA80F9002B00F05B
:10CED0009180686B002201460B790E2B02F1010450
:10CEE00040F081803B79D2B2591E91420BDC142272
:10CEF00002FB0303283BC5F890301B790E2B04BFBF
:10CF00000023C5F890300023BB71686B95F8593049
:10CF100059B201EB810200EB820201331279DBB2DC
:10CF2000002AF5D097F9072085F85910002A0BDB65
:10CF30008A4220D0029B1A44D2B2B74B0121384614
:10CF400009F0A0F8A9EB0009B9F11D0F40F28381A7
:10CF500095F9592097F90730934210D0029B1A4453
:10CF6000D2B2AE4B0121384609F08CF895F8593011
:10CF7000FB71A9EB0009B9F11D0F40F26C816C6BDC
:10CF8000002614343B79F2B2023B9A4247DB6E6BC7
:10CF90004FF0000B14363B795FFA8BF8023B984553
:10CFA00080F2598116F8103C0E2B00F0548116F8CF
:10CFB000042CD10740F19280029988445FFA88F8E6
:10CFC0000D2B00F22481DFE813F018012201220169
:10CFD0005B005B009100CD00BD00D600D6004E0086
:10CFE000DE00B000A6000A7C42F003020A7414318D
:10CFF000224671E7B8F1000F87D095F838306A6B98
:10D0000003EB830302EB83039A423FF67EAF117C6E
:10D010004C0744BF41F0010111741432F4E714F8D5
:10D02000103C0E2BB3D014F8041C880718D5002B25
:10D03000029B1A4418BF032154F8143C08BF022174
:10D04000D2B2384609F01EF814F8043CA9EB0009E6
:10D0500023F00203B9F11D0F04F8043C40F2FB80F9
:10D06000013614348EE756F8083C002B00F0CF80D0
:10D07000797908394246C9B2384609F003F843E0E5
:10D0800097F805A0032BAAF1080A2BD156F80C0C2F
:10D0900050B312F008040DD080475FFA8AF10346BE
:10D0A00003904246384608F0EDFF0446039822F00C
:10D0B00083FC82445A4B42465FFA8AF1384608F0B4
:10D0C000E1FF16F8043C23F00103204406F8043C79
:10D0D000A9EB0009B9F11D0F40F2BD800BF1010B66
:10D0E000143658E70024E5E70446E3E756F8080C51
:10D0F0000028EDD07979037808390BB3494B4246C3
:10D10000C9B2384608F0BEFF16F8043C23F001030C
:10D1100006F8043CDCE756F8083C79791A689B6805
:10D120001278083953F82230A4E756F8080C002882
:10D13000CED00388797913F4006FA1F10801DDD115
:10D14000394B97E756F8080C0028C1D003681878C7
:10D1500005A91DF027FE05A81DF012FE797905AB83
:10D16000083987E756F8080C0028B1D0036805A9EC
:10D1700093F90000EDE756F8080C0028A8D00368E2
:10D1800005A91888E5E756F8080C0028A0D0036820
:10D1900000891B78584300F5C33005A9A0301DF065
:10D1A00001FE9DF816209DF815308DF815202E22D1
:10D1B0008DF816209DF819208DF81430302A01D0F2
:10D1C0002E2A0DD14FF000028DF819209DF818205D
:10D1D000302A01D02E2A03D14FF000028DF81820FA
:10D1E000302B08BF202305A808BF8DF814301DF090
:10D1F000C7FD797905AB09393CE756F8084C44B1CD
:10D2000056F8140C22F0D8FB2346C11C32E700204C
:10D210005EE720465CE700BF8C8003088F80030830
:10D2200090800308928003089680030806247A6A97
:10D2300001327A62B7F92020002A7FF78AACD5F84C
:10D24000B0301344019A9B1A3B846B6BD5F8AC70D9
:10D25000002B7FF41EAED5F8B830019A03F5FA73AF
:10D260009A427FF635ACD5F8AC0003681B6A984744
:10D27000019BC5F8B8302BE40124D8E70224D6E797
:10D280000324D4E70424D2E70524D0E7F8B5044604
:10D290000E461A4DE1B108F00BFF03220521184B91
:10D2A000204608F0EFFE236820465B6A98471AF094
:10D2B00025FC1AF075FBC82005F08CF81148FFF723
:10D2C00015FA6B6DDB680BB10020984708F0C6F9C2
:10D2D000236800275B6885F8987020469847237A72
:10D2E0006F65013B237216B1074B084ADA60084AA2
:10D2F000137843F0010313700020F8BDA42D002023
:10D300009A800308B800002000ED00E00400FA0550
:10D310001B8E002050B110B5064C60601DF0EEFC75
:10D3200002234FF6FF722375A28110BD014A1075CA
:10D33000704700BF3C7D002010B5D42280213C20E6
:10D3400020F05AFC802211463C2020F055FCA822F7
:10D3500080213C2020F050FC3F2280213C2020F006
:10D360004BFCD32280213C2020F046FC002280216F
:10D370003C2020F041FC402280213C2020F03CFC5D
:10D380008D2280213C2020F037FC142280213C207B
:10D3900020F032FCA12280213C2020F02DFCC8226C
:10D3A00080213C2020F028FCDA2280213C2020F043
:10D3B00023FC122280213C2020F01EFC81228021AF
:10D3C0003C2020F019FCCF2280213C2020F014FCCE
:10D3D000D92280213C2020F00FFCF12280213C202A
:10D3E00020F00AFCDB2280213C2020F005FC4022BA
:10D3F00080213C2020F000FCA42280213C2020F051
:10D40000FBFBA62280213C2020F0F6FBAF228021EE
:10D410003C2020F0F1FBA62280213C2020F0ECFBF8
:10D42000AE2280213C2020F0E7FB202280213C20FE
:10D4300020F0E2FB002280213C2020F0DDFBB02226
:10D4400080213C2020F0D8FB402280213C2020F08D
:10D45000D3FB002280213C2020F0CEFB1022802133
:10D460003C2020F0C9FB4FF48064013C00224021A5
:10D470003C20A4B220F0C0FB002CF6D181228021F8
:10D480003C2020F0B9FBC82280213C2020F0B4FBD6
:10D49000AF2280213C2020F0AFFB012010BD08B559
:10D4A000A0F15002D2B280213C2020F0A5FB002246
:10D4B00080213C2020F0A0FB102280213C20BDE8F0
:10D4C000084020F099BB074B1A68042A08D0511C69
:10D4D0001960054B03EB8203C3F89C0001207047E1
:10D4E00000207047C4300020A42D002070B50446F1
:10D4F000006800F120033F2B4BD800F108030F2BED
:10D500002BD8811C032994BF00210121636803F1FA
:10D5100020023F2A00F2B28003F108020F2A1ED82F
:10D520009A1C032A02D9002908BF0121A26802F12E
:10D5300020053F2D2FD802F108050F2D11D900F03D
:10D540003F0040F08000F4F721FD2079F4F71EFD44
:10D55000207ABDE87040F4F719BD0221D6E7022118
:10D56000E4E7951C032D00D911B1012940F0888012
:10D5700000F00F0040F04000F4F708FDA068636879
:10D5800000F00F0040EA0310C0B2BDE87040F4F7AD
:10D59000FDBC6368A26802F18001FF2944D902F54D
:10D5A0000041B1F5803F64D302F50002B2F1807F03
:10D5B00034BF0225032503F18002FF2A4FEA8505C7
:10D5C0000DD903F50042B2F5803F54D303F50003B3
:10D5D000B3F1807F2CBF45F0030545F0020500F153
:10D5E0008003FF2B4FEA850506D900F50043B3F50C
:10D5F000803F34D245F0010565F03F00C0B2F4F73A
:10D60000C5FC04F10C0605F00303022B20781DD0A5
:10D61000032B11D0012B09D0F4F7B8FC0434B44229
:10D620004FEAA505EFD170BD0025C4E7F4F7AEFCC5
:10D630006078F4F7ABFCF1E7F4F7A8FC6078F4F756
:10D64000A5FCA078F4F7A2FCE078E5E7F4F79EFCEF
:10D650006078F4F79BFCA078F4F798FCDEE700F51F
:10D660000000B0F1807F34BF45F0020545F00305AE
:10D67000C2E701259FE745F00105B0E7A2688AE708
:10D6800002293FF45CAF01019B0003F00C0301F0A1
:10D6900030010B4302F0030243EA0200BDE8704090
:10D6A000F4F774BCF0B5C41784EA40047F2C83B04F
:10D6B00046D9434D434E95F87D36434F08E03068D8
:10D6C00003681B68984795F87D36E4097F2C3AD9A2
:10D6D00064F07F01022BC9B2F1D1DFF8F0E0DEF88F
:10D6E000000040F2FF1C90F91A308DF806105A1C09
:10D6F00016D04268C2F30802624502EB43230FD002
:10D70000D9554368E40901337F2C436064F07F01FD
:10D710002BD990F91A30C9B25A1C8DF80610E8D1ED
:10D72000037E13F0060F02D090F82830ABB1E40965
:10D730007F2C64F07F0118D9C9B2DEF80000D2E76F
:10D740001F4B93F87D36022BE1B235D01D4B186884
:10D7500003681B68984703B0F0BD01220DF1060174
:10D7600017F004F995F87D36AFE7E1B2DEF8000076
:10D770008DF8071090F91A20531C0FD0436840F21F
:10D78000FF14C3F30803A34208D003EB42230E4A5D
:10D79000995443680133436003B0F0BD037E13F036
:10D7A000060FD8D090F82830002BD4D101220DF1EB
:10D7B000070117F0DBF8CEE7DFF810E0D6E700BF8F
:10D7C00094610020547D0020246B00203C7D0020CB
:10D7D000F0B57F2883B0044646D9434D434E95F8B3
:10D7E0007D36434F08E0306803681B68984795F81A
:10D7F0007D36E4097F2C3AD964F07F01022BC9B24F
:10D80000F1D1DFF8F0E0DEF8000040F2FF1C90F903
:10D810001A308DF806105A1C16D04268C2F308025E
:10D82000624502EB43230FD0D9554368E409013325
:10D830007F2C436064F07F012BD990F91A30C9B274
:10D840005A1C8DF80610E8D1037E13F0060F02D0A3
:10D8500090F82830ABB1E4097F2C64F07F0118D92F
:10D86000C9B2DEF80000D2E71F4B93F87D36022BD9
:10D87000E1B235D01D4B186803681B68984703B0A8
:10D88000F0BD01220DF1060117F070F895F87D3614
:10D89000AFE7E1B2DEF800008DF8071090F91A202A
:10D8A000531C0FD0436840F2FF14C3F30803A34294
:10D8B00008D003EB42230E4A995443680133436076
:10D8C00003B0F0BD037E13F0060FD8D090F82830D7
:10D8D000002BD4D101220DF1070117F047F8CEE754
:10D8E000DFF810E0D6E700BF94610020547D0020EF
:10D8F000246B00203C7D00200FB42DE9F04FDFF8B1
:10D90000F49299F87D368BB0022B149C00F00981BB
:10D91000B44B1868036848211B68984799F87D360E
:10D92000022B00F05781AF4B1868036820211B6859
:10D93000984715AF0025DFF8C0A20497A84607AEA8
:10D94000631C0593217849B3252948D1A31CCDF840
:10D95000188005936078302863D04FF0000BA0F159
:10D960003003DBB2092B57D96C282DD0642800F086
:10D97000C2803AD8252831D079D9582800F0A6801D
:10D98000632830D139780020F3F770FC059C631CC4
:10D9900005932178043701350029D5D199F87D36D2
:10D9A000022B6AD08F4B186803680A211B689847BE
:10D9B0008D4AD2F8C03003355D1BC2F8C0500BB0A1
:10D9C000BDE8F04F04B07047059B5C1C05941A78C5
:10D9D000642A00F0F0802AD8252A6DD12521002064
:10D9E0000135F3F743FC059CAAE7732833D05CD9D3
:10D9F000752869D13C1D3868334600220A21274624
:10DA000009F084F8069A00965B465146002009F01A
:10DA100001F9059C054493E706AA05A91CF074FFCB
:10DA2000A2E7E31C0593A0784FF0010B97E7732A58
:10DA300011D040F2CB80752A54D0782A80D1A2F13F
:10DA40005802B2FA82F2386852093346102104377C
:10DA500009F05CF8D6E73B6800930023069A184665
:10DA6000514609F0D7F804370544059C68E70028BB
:10DA7000B9D199F87D36022B94D15C4B0A221868F3
:10DA80008DF81C2090F91A104B1C3BD0436840F2D3
:10DA9000FF14C3F30803A34234D003EB41235449DA
:10DAA0005A5443680133436082E76E289BD1059C3A
:10DAB0003B6804371D6043E740F28480582ABED09B
:10DAC000632A3FF45FAF3BE778288CD1A0F158027E
:10DAD000B2FA82F2386852093346102109F016F87A
:10DAE00004378FE73C1D3868334600220A21274659
:10DAF00009F00CF886E73B1D386831461F4608F0F0
:10DB0000D7FF7FE7037E13F0060F3FF451AF90F885
:10DB10002830002B7FF44CAF012207A916F026FF16
:10DB200046E7324B186890F91A10436848224E1C99
:10DB3000C3F308038DF80E2040F2FF151DD0AB4251
:10DB40001BD003EB41232A495A54436890F91A1019
:10DB500001334360C3F3080320224D1C8DF80F20CE
:10DB600019D040F2FF15AB4215D003EB41232049F9
:10DB70005A54436801334360DBE6027E12F0060F1D
:10DB8000EAD090F82820002AE6D101220DF10E01FA
:10DB900016F0ECFEC2E6037E13F0060F3FF4C9AEAA
:10DBA00090F82830002B7FF4C4AE01220DF10F0154
:10DBB00016F0DCFEBDE63B1D386831461F4608F016
:10DBC00077FF1FE7002A3FF4E9AEB9E66E2A3FF47B
:10DBD0006FAFB5E6054B1868426890F91A10C2F3AA
:10DBE0000803B9E7547D0020A42D00203C7D0020CF
:10DBF000246B0020946100206D1200080FB42DE901
:10DC0000F04389B010AE002556F8043BDFF8888158
:10DC100002962F4605AC5A1C0392197839B3252970
:10DC200035D19A1C049703925878302852D04FF07F
:10DC30000009A0F13003DBB2092B46D96C281CD0B7
:10DC4000642800F0948028D825281FD067D9582848
:10DC500077D063281FD131780020F3F707FB039BAF
:10DC60005A1C03921978043601350029D7D1284669
:10DC700009B0BDE8F04304B07047039A531C039306
:10DC80001278642A7AD02BD8252A52D12521002057
:10DC90000135F3F7EBFA039BBDE7732833D041D985
:10DCA00075284CD106F1040E3068234600220A2163
:10DCB000764608F02BFF4B46049A0094414600201C
:10DCC00008F0A8FF039B0544A5E704AA03A91CF0DC
:10DCD0001BFEB3E7DA1C039298784FF00109A8E71E
:10DCE000732A10D055D9752A37D0782A93D1A2F14A
:10DCF0005802B2FA82F230685209234610210436E3
:10DD000008F004FFD7E73368009300231846049A0D
:10DD1000414608F07FFF04360544039B7BE700285B
:10DD2000A5D0B8E76E28B6D1039B326804361560DB
:10DD300071E72AD9582ADAD0632A8CD06BE7782881
:10DD4000A9D1A0F15802B2FA82F2306852092346F2
:10DD5000102108F0DBFE0436ADE706F1040E306852
:10DD6000234600220A21764608F0D0FEA3E7331DA1
:10DD7000306821461E4608F09BFE9CE7331D306844
:10DD800021461E4608F094FE95E7002A3FF46FAF47
:10DD900041E76E2AC9D03EE76D120008104B93F997
:10DDA0000030002B17DD0F4B1B88B3B1192B0CD99A
:10DDB000642B0CD9C82B0CD9B3F5C87F94BF0323AF
:10DDC000042301330370012070470023F9E7012386
:10DDD000F7E70223F5E7002070470120704700BFF6
:10DDE000C0300020682E0020074B93F90030002B34
:10DDF00007DD064B1B780370054B1B780B70012069
:10DE000070470020704700BFC03000201C880020F1
:10DE10001D880020034B93F900000028D4BF002088
:10DE200001207047C030002004207047034B1A784F
:10DE30000AB901221A700020704700BF4411002067
:10DE4000064B5A784AB19B783BB103EBC203093BBE
:10DE5000034A32F81320034B5A80704744110020C4
:10DE6000D8700308682E002008B5144B1B780BB13E
:10DE7000134A5370134B1B780BB1114A9370FFF781
:10DE8000DFFF114B114A1B780133137113886BB1FB
:10DE9000192B0DD9642B0DD9C82B0DD9B3F5C87F1B
:10DEA00094BF03230423064A01331370002008BDE6
:10DEB0000023F8E70123F6E70223F4E71C8800209B
:10DEC000441100201D880020C1300020682E002051
:10DED00008B5054B9A781AB901229A70002008BD3E
:10DEE000FFF7AEFFFAE700BF4411002008B5054B6D
:10DEF0005A781AB901225A70002008BDFFF7A0FF16
:10DF0000FAE700BF44110020044B93F900000128F8
:10DF100006BF02221A700020704700BFC0300020E8
:10DF200058B1064B013833F81020054B1989DA80B7
:10DF300091421CBF02229A72E6E7704728520308FA
:10DF4000682E002070B169B101EBC0010939064BA0
:10DF500033F81120054B1969DA608A421CBF02228E
:10DF60001A75D1E7704700BFD8700308682E0020EB
:10DF700008B5104A51789378127803EBC103093B36
:10DF80000D4931F813100D4B1869D96081421CBF3F
:10DF900002211975013A0A4931F812201989DA80EB
:10DFA00091421CBF02229A72FFF7AEFF4FF0FF3082
:10DFB00008BD00BF44110020D8700308682E00205F
:10DFC00028520308054A117E537E03EBC103093B27
:10DFD000034931F81330D382704700BF682E002008
:10DFE000D8700308094A0A4B917E51B1D27E22B9FA
:10DFF00003F11C029A610020704703F1E4029A6168
:10E00000F9E703F5C2729A61F5E700BF682E0020B8
:10E0100044110020024BDA8B9A834FF0FF30704797
:10E02000682E0020024B9A8BDA830020704700BFD5
:10E03000682E0020024B5A8C1A840020704700BFC3
:10E04000682E0020064B93F9E821022A06D193F8A6
:10E05000EB31C3F340030370012070470020704789
:10E06000441100200F4A92F9E831C3B1012B11D1BC
:10E0700092F9EA31272B09DC182B09DC0F2BD4BFCE
:10E080000023012301330370012070470323F9E7C4
:10E090000223F7E792F8EA310133DBB2F3E71846DF
:10E0A000704700BF441100200B4A92F9E8318BB150
:10E0B00092F9E931082293FBF2F2013202705A42DE
:10E0C00002F0070203F0070358BF534201330B70FD
:10E0D000012070471846704744110020034B93F904
:10E0E000E801003018BF0120704700BF4411002034
:10E0F0000320704730B5084A92F8243092F8255032
:10E100005C1C04F00304AC4205D002EBC30382F8AC
:10E1100024409862D96230BD682E002010B50246B6
:10E120000023141AA14201DC184610BD12F8014B5D
:10E130006340082413F0800F4FEA430318BF83F0B5
:10E14000D503013CDBB2F5D1EBE710B50E4C94F9E9
:10E15000E831BBB1032815D8012B0C4B4FEAC000A6
:10E1600003444FF005010CBF1B7C9B7C084884F8DE
:10E17000F431FFF7D3FF84F8F50106210448BDE828
:10E180001040B7E710BD00BF44110020285203081B
:10E190003413002008B50B4B93F9E8210A4B1AB948
:10E1A00083F84820002008BD93F8480008B90122F0
:10E1B000F6E793F84930012BF4D10138C0B2FFF7EC
:10E1C000C4FFEFE744110020682E002010B1013891
:10E1D000C0B2BAE7704738B5094C00F03F0004F50B
:10E1E000FB7540F0080084F8FA0105212846FFF786
:10E1F00095FF062184F8FB012846BDE8384079E701
:10E200004411002008B5064B93F84A3023B9012089
:10E21000FFF7E1FF002008BD0220FFF7DCFFF9E770
:10E22000682E0020094B93F9E821022A0CD158B935
:10E2300093F8EB3113F0040F0CBF042005201B07EB
:10E2400048BF40F00200C6E7704700BF44110020FD
:10E2500038B5094C01EBC00104F5FE7584F80012D5
:10E2600028460521FFF75AFF062184F801022846B7
:10E27000BDE838403EE700BF4411002008B5074B19
:10E2800093F9E821064B12B95A76002008BD5A7E50
:10E290000AB90122F8E7FFF795FEF6E744110020DE
:10E2A000682E002008B5074B93F9E821064B12B9F8
:10E2B0001A76002008BD1A7E0AB90122F8E7FFF796
:10E2C00081FEF6E744110020682E002028B121B11C
:10E2D00001390138C9B2C0B2BAE7704738B5094C44
:10E2E00004F20225030A84F807020621284684F86E
:10E2F0000632FFF713FF072184F808022846BDE81D
:10E300003840F7E64411002008B5054B188C6FEA39
:10E3100040406FEA504080B2FFF7E0FF002008BDA8
:10E32000682E002010B5174C94F84930022B1AD1F2
:10E33000617E207E01390138C9B2C0B2FFF788FF83
:10E3400094F84A305BB90520FFF745FF94F8480080
:10E350000138C0B2FFF7F9FE4FF0FF3010BD0620C4
:10E36000FFF739FFF2E7E37E43B9617E207E013992
:10E370000138C9B2C0B2FFF76BFFE7E7A08BFFF728
:10E38000ADFFE3E7682E002008B50D4BDA7E5AB9E1
:10E39000597E187E01390138C9B2C0B2FFF758FF63
:10E3A000FFF720FE002008BD93F84920012A03D181
:10E3B000988BFFF793FFF3E70022DA76F0E700BFD0
:10E3C000682E0020F8B50E4C94F84930012B064613
:10E3D0000F4604D10020FFF7FEFE0020F8BD022BFF
:10E3E0000AD1002584F84A50FFF70CFF3946304621
:10E3F000E576FFF7C9FFF0E7012384F84930ECE741
:10E40000682E0020074A084992F84B3009780133FA
:10E41000DBB2994282F84B3004BF002382F84B30C4
:10E42000704700BF682E002088870020F8B55F4B3A
:10E430005F4A1B68A2FB0020DBB15E4C94F84C30B5
:10E44000012B4FEA901003D014D3022B1AD0F8BD41
:10E45000594D94F84B10594E2D782065582202FBE7
:10E46000016202200D2D84F8543084F84C0013739F
:10E470006AD0F8BD41F287339842FAD9012384F873
:10E480004C30F8BD236D643398421FD394F84B3061
:10E490004B4903EB83035B00CA5CFF2A04D00132C3
:10E4A0004848CA5401230370FFF7ACFF424B1B7866
:10E4B00001220D2B84F84C20DBD1B4F86430424AA1
:10E4C00001339BB2A4F864305380F8BD94F8542013
:10E4D00002F0FF03002ACCD104F1570104F16005DA
:10E4E00011F8010F0822434013F0800F4FEA430355
:10E4F00018BF83F00703013ADBB2F5D1A942EFD18F
:10E5000094F86110994294F84B3021D003EB8303C7
:10E510002B495B00CA5CFF2A04D001322948CA5447
:10E5200001230370FFF76EFF234B1B7801220D2B95
:10E5300084F84C209DD1B4F86230234A01339BB259
:10E54000A4F862309380F8BD1F4B01311980F8BDEB
:10E5500003EB83031A4E94F8591094F85A5094F828
:10E560005BE094F85C0094F85D705B0045EA01257F
:10E57000F254334494F8582094F85E1094F85F6095
:10E580005A7094F860205D8040EA0E2041EA07212D
:10E5900042EA06220B4D9880D98001201A8128700A
:10E5A000FFF730FF84F84C00F8BD00BF08310020B1
:10E5B000D34D6210682E002010880020C85B002018
:10E5C00098870020911E0020148800200A4B93F8A1
:10E5D00054204AB193F866209918092A81F8580006
:10E5E00003D0013283F866207047002283F866204A
:10E5F00083F85420704700BF682E002010B5054BEB
:10E6000005499A8B03F16704204608F00FFC204669
:10E6100010BD00BF682E00201586030810B5054BFD
:10E6200005495A8C03F16C04204608F0FFFB204694
:10E6300010BD00BF682E00201586030810B54D4C94
:10E6400094F9E821002A00F093804B4B997E01B9A0
:10E650009A765A8C1AB9B4F8EE2102B15A849A8B80
:10E660001AB9B4F8EC2102B19A8394F8EB2143482B
:10E67000C2F3C00183F84A1093F84910DB7E415C75
:10E6800084F80912002B35D194F9E9313C4808216E
:10E6900093FBF1F1405C594201F0070103F00703DD
:10E6A00058BF4B423133DBB284F80C3202F00A031C
:10E6B0000A2B84F80B0233481FD1B4F8EE213249FB
:10E6C00008F0B4FB202384F8123294F8EB319A0757
:10E6D00031D513F0040F14BF49234F2384F81432AB
:10E6E0005223502284F81532002384F8132284F830
:10E6F000163210BD46235520D6E7D10705D5B4F80C
:10E70000EC21214908F092FBDCE794F9E931594208
:10E7100001F007014FF0080293FBF2F203F0070348
:10E7200058BF4B4203EBC203184A174932F8132073
:10E7300008F07CFBC6E794F9E831154A022B94F9FE
:10E74000EA3108D102EBC3031249DA681248BDE886
:10E75000104008F06BBB272B06DC182B06DC0F2BB8
:10E76000D4BF00230123EDE70323EBE70223E9E70E
:10E7700010BD00BF44110020682E00201986030838
:10E780001D8603085213002015860308D87003085D
:10E79000285203082686030857130020F8B5154BA6
:10E7A0001E6807460D461EB3134C1022002104F1CB
:10E7B000710025F0BEFE0F2384F873502D0A84F8F3
:10E7C000713084F8727084F874500023012204F1CF
:10E7D0007100115C01320B440E2ADBB2F9D184F8CE
:10E7E0007F30304610220549BDE8F84001F098BB63
:10E7F000F8BD00BF10310020682E0020D92E002067
:10E8000008B5074B197919B901221A71002008BD02
:10E810004B1E594259414920FFF7C0FFF6E700BFA0
:10E82000682E0020B0FA80F149094920B6E7034B71
:10E83000002183F88110C3F88410AFE7682E002010
:10E840002DE9F0479C4D95F900300133064600F064
:10E8500031819A4B9A4C1A689846002A40F09B8066
:10E8600095F90030032B00F2E580DFE803F09A9A77
:10E87000B6DD0F281DD1012384F88130D8F80000BF
:10E8800001F072FB0028EBD0D8F8000001F068FB23
:10E89000D4F884305A1C2344C4F8842083F88800B8
:10E8A00094F88130012B07D0E3D3022B0DD084F8EC
:10E8B0008170C4F88470E1E7A0F17203012B01D9E3
:10E8C0007628F4D184F88190D8E7102AD6D1002395
:10E8D000012212F80A1001320B440E2ADBB2F8D1E1
:10E8E00094F8962084F881709A42C4F88470C5D157
:10E8F00094F89730002BC1D194F88930732B3DD018
:10E90000762B0FD0722BABD194F88B2094F88A30F1
:10E9100053EA0223A4D095F90030002BA0DC012398
:10E920002B709DE794F88B3094F88A0050EA03200E
:10E9300096D094F88D2094F88C30206143EA02231D
:10E940002380604B94F88F201A7094F8912094F8EB
:10E95000903043EA0223238123F060FAE3680BB985
:10E960002369E360E3880BB92389E38095F90030DC
:10E97000032B7FF475AF02232B7071E794F88F207F
:10E9800094F88E3043EA02231BB2002B3FF468AFA9
:10E99000A4F8983064E74FF00209002704F1880AD0
:10E9A0006CE7D4F89C204849B21A8A4242DD2BB960
:10E9B0007220FFF73CFFC4F89C603BE0D4F8A03025
:10E9C0005A1CDB07C4F8A02003D47620FFF72FFFE2
:10E9D000F1E77320FFF72BFFEDE7E168A1B1237D9D
:10E9E00093B1236999420FD089B24620FFF7D6FE32
:10E9F000237D013B237506F59226032306F57876E1
:10EA00002B70C4F89C6015E0E188002948D0A37AF7
:10EA1000002B45D023888B4242D05020FFF7BEFE0A
:10EA2000A37A013BA372E6E7D4F89C30274AF31A95
:10EA30009342CADC26482A2380F82832254B1978CD
:10EA4000254B0B44202293F82C3080F82A32234B9C
:10EA500080F829221978224B53F821301B7880F84E
:10EA60002C22226980F82B3200F22D207AB11D4928
:10EA700008F0DCF923891C486BB122881B499A42B3
:10EA80000CBF20222A22BDE8F04708F0CFB9184970
:10EA900008F0CCF9EEE71749BDE8F04708F0C6B931
:10EAA00001232B702369E3602389E3800023A37291
:10EAB0002375BFE7BDE8F087C0300020103100208B
:10EAC000682E0020C130002040420F00400D03009E
:10EAD000441100201C880020285203081D880020B3
:10EAE00014530308158603087513002023860308B2
:10EAF0002B8603082A86030838B5114C94F8253074
:10EB000094F824209A4216D004EBC3030D499A6A64
:10EB1000D86A002398420FDC9378C4F8A4005B08FD
:10EB200084F8A8301CF0AEFE94F82530013303F0D1
:10EB3000030384F8253038BDD55C5D540133E9E723
:10EB4000682E0020248800202DE9F843BF4E33684A
:10EB50000746002B40F03A81BDE8F883306801F0A9
:10EB6000FFF994F8A9308046052B09D8DFE803F0B7
:10EB700003324046606DAA2802D1012384F8A930EF
:10EB8000306801F0F1F90028E8D1B14B1988092962
:10EB90001D460BD9B3F802E0642202FB0EF292FB91
:10EBA000F1F2452A40F315811880588094F8C4305A
:10EBB000002B40F03D810521A648FFF79BFA4FF45A
:10EBC0008040FFF78BFBFFF797FF012384F8C430E9
:10EBD000BDE8F883552803D1022384F8A930CFE794
:10EBE0009B4A938801339380002384F8A930C7E7B8
:10EBF000032384F8AA0084F8A930C1E7092884F81F
:10EC0000AB00C4F8BC0007DD914AD3880133D38040
:10EC1000002384F8A930B3E718B9052384F8A93094
:10EC2000AEE70023C4F8C030042384F8A930A7E776
:10EC3000D4F8C030E218013382F8AC00D4F8BC201C
:10EC4000C4F8C03093429BD1E7E7D4F8BC30824887
:10EC500003F102094FFA89F1FFF760FA804540F0AD
:10EC6000AB8094F8AA2094F8A830DFF8E4819A42A7
:10EC70001FD1002384F8A830531ED9B208290AD81E
:10EC800001238B4013F0160F3AD140F201110B42D1
:10EC900019D1180767D4B8F80C300133A8F80C3034
:10ECA000B8F802300133A8F80230002384F8A93004
:10ECB00066E7092A01D1012BDBD0B8F80A3001330D
:10ECC000A8F80A30D8E7B9F1060F19DD012A0CBF00
:10ECD0000123022385F8E83194F8AC3085F8E93156
:10ECE00094F8AD3085F8EA3194F8AE3085F8EB3120
:10ECF00094F8AF2094F8B03043EA0223A5F8EC3141
:10ED000094F8493053BB95F8EB3113F0020F03F040
:10ED1000010314BF02220122E37695F9E93184F858
:10ED20004920082293FBF2F2511C2176594201F04E
:10ED3000070103F0070358BF4B42591C03EBC20302
:10ED4000464A617632F81330E38295F9E831022BB6
:10ED500020D195F8EA31013384F84830FFF76EFC92
:10ED6000FFF76CFC9CE7B9F1040FC9DD94F8AC30F7
:10ED700094F8AD2042EA032212B293B2590404D5AA
:10ED8000C3F30D03A5F8EE31BAE7002AF8DBA5F8C6
:10ED9000EC31B5E795F9EA31272B09DC182B09DCB2
:10EDA0000F2BD4BF00230123013384F84830D5E76B
:10EDB0000323F9E70223F7E794F8AA30DB073FF5CE
:10EDC00074AF234A1389013313816EE7244C254D18
:10EDD000D6E6244BD3F84822012A1ED1B3F84C12B0
:10EDE00041F25632914203D14FF0FF32C3F848222C
:10EDF000D3F84812B3F84C22306801EB810101EBE3
:10EE0000810102EB410189B2A3F84C1203681B692E
:10EE1000984700232B806B80C8E60132E8D1B3F815
:10EE20004C22B2F5965F04BF0122C3F84822DFE707
:10EE300094F8A830D3B10C4B1B68FB1A782B15D96A
:10EE4000D4F8A400BDE8F8431CF01CBD20880020C5
:10EE50004C88002092130020122F0020D870030845
:10EE6000682E0020441100204888002094F82420B7
:10EE700094F825309A4202D0BDE8F8433CE6064BB0
:10EE80001B68FF1AB7F57A7F04D305210348FFF703
:10EE900031F9F1E7BDE8F88348880020921300209B
:10EEA0002DE9F043C24CC34D94F814312E6883B061
:10EEB0003BB1D4F8180120B194F81C31013B012B6F
:10EEC00002D903B0BDE8F083BB4F4FF001094FF00A
:10EED000000809E01B2B00F074820D2B00F0578214
:10EEE00087F85392D4F8180103685B6898470028A4
:10EEF0003AD0D4F818010368DB68984783B27E2BB8
:10EF00002A682AD097F853120029EBD194F81D21D2
:10EF1000002ADFD07D2B00F0518294F822E1BEF16F
:10EF2000000F04D080F02003DBB284F82211511CC2
:10EF3000C9B22244092984F81D1182F8C83000F0B2
:10EF400033820829CED8B4F82021134403EB1323CD
:10EF500003F0FF03A4F82031C4E784F81D8184F88E
:10EF60001E8187F85382BDE794F8233133B194F8BA
:10EF7000C93084F82301302B00F0F58294F81EE1AB
:10EF80008E4A8F49DFF850C28E4F94F8348294F83D
:10EF90004632BEF1000F94D0B8F1000F40F01C8251
:10EFA0002868801B012847D802EB4300808E002888
:10EFB0003CD00133B0F5826FDBB200F0CE8143D993
:10EFC000B0F5E26F00F00A816BD9B0F5046F00F084
:10EFD0002181B0F5116F00F0A581B0F5E46FDFD1AC
:10EFE000794A84F84632916B1289642303FB01F35A
:10EFF000202593FBF2F307224FEA132E1F0C1E0E5F
:10F00000694610208DF802308DF803E08DF8047009
:10F010008DF805608DF800508DF801201FF06EFE10
:10F02000002384F81E3103B0BDE8F0832868801BFC
:10F0300001284FF00103B7D9002284F8463284F842
:10F040001E2103B0BDE8F083B0F5007F00F04381DE
:10F0500052D8B0F5807F00F0EC80B0F5887F9FD16A
:10F06000386884F8463243078FD5584B1B688DF8B3
:10F07000023010221F0A23FA02F61B0E1046012549
:10F0800069468DF803708DF804608DF805308DF8B1
:10F0900000208DF801501FF031FE002384F81E314E
:10F0A0000FE7B0F5C06F00F02C81B0F5E06F7FF492
:10F0B00077AF454A84F84632116B1289642303FB0B
:10F0C00001F3002593FBF2F307224FEA132E1F0CE6
:10F0D0001E0E694610208DF802308DF803E08DF881
:10F0E00004708DF805608DF800508DF801201FF038
:10F0F00005FE84F81E51E4E6B0F5047F00F0B98007
:10F10000B0F5806F7FF44CAF94F8502284F846320B
:10F11000531CDAB2032A00F2418142F2107384F8E0
:10F12000502203FB02F32A4A1278D70748BF013363
:10F13000960748BF02335507264A128848BF043352
:10F14000D00748BF0A33910748BF1433170648BF9A
:10F150002833D60548BF2833550748BF6433100706
:10F1600048BFC833910548BF03F5C873970648BF29
:10F1700003F57A73D60648BF03F5FA63550648BF10
:10F1800003F57A6300251E0A0422694610208DF8D3
:10F1900002308DF803608DF800508DF804508DF822
:10F1A00005508DF801201FF0A9FD84F81E5188E656
:10F1B000682E0020448800204411002028520308B3
:10F1C000B47E0020248A00208C8900202C2400207A
:10F1D0001B8E0020C0600020B87E0020CD4A84F83D
:10F1E0004632506B11896423102203FB00F393FB1A
:10F1F000F1F34FEA132E23FA02F71E0E10460725ED
:10F200008DF8023069468DF803E08DF804708DF8B2
:10F2100005603CE7C04A84F84632B2F9043003EB9B
:10F2200083035B004FEA132E1F0C1E0E402508229D
:10F23000E6E6386884F8463240077FF5A6AEB74B5D
:10F240009B698DF802301F0A1E0C00251B0E01223F
:10F25000694610208DF803708DF804608DF8053034
:10F260008DF800508DF801201FF048FD84F81E51E4
:10F2700027E6086884F8463283077FF586AE9CF857
:10F28000000000283FF481AED4F84C32DB7B002B29
:10F2900000F0ED80A24B1B8893FBF0F303EB83039C
:10F2A0005B0010224FEA132E23FA02F710460226C3
:10F2B000002569468DF802308DF803E08DF8047062
:10F2C0008DF800208DF801608DF805501FF016FDB7
:10F2D00084F81E51F5E5086884F8463210F0082FCE
:10F2E0003FF453AE8F4A9049126881FB0231D31725
:10F2F000C3EBA1034FEA132E1F0C1E0E00250222A2
:10F30000E7E6086884F8463210F0082F3FF43DAE77
:10F31000864B1B688DF802301F0A1E0C00251B0E41
:10F32000062295E7086884F8463283077FF52DAEFC
:10F330009CF80080B8F1000F3FF427AE784B1B8893
:10F34000102203EB83035B00104693FBF8F30926BE
:10F350004FEA132E23FA02F7AAE7386884F84632F8
:10F3600010F020087FF411AE0B68180600F1E6805B
:10F37000D4F84C325B7C002B3FF407AE94F851324A
:10F38000032B00F27B81DFE803F0BAB0A17884F8A8
:10F390001D9184F8C830A4F82021A3E5012384F846
:10F3A000503242F21073BEE6B4F82021C2F1FF02DF
:10F3B00093427FF495AD84F8239191E584F82291EE
:10F3C00090E5D4F8180103685B68984700287FF43B
:10F3D00087AD84F81E9185E52A68961B012E3FF6BD
:10F3E0002BAED4F82832DFF8509194F847224B45E1
:10F3F00000F01481511C94F84852D4F82C7284F80F
:10F40000471202F00F028DF800200DF10102F91AE7
:10F4100000296E460DF1060E02DC12E0002829DDFF
:10F420000133C4F8283213F8011C02F8011B72459D
:10F43000A7EB030085EA0105F0D384F8485200F0F9
:10F440003681501C7045157005D202AB9A1A033AEA
:10F45000002125F06EF8314632201FF04FFC4FF0AE
:10F460000008002384F8348284F81E3129E52C4BEF
:10F470001B8813E784F84852E3E72D4B1A68537949
:10F480009179D27903F1407303EB012303EB02433B
:10F49000002284F8512210221F0A23FA02F61D0EC0
:10F4A0004FF0040E104669468DF802308DF80020AA
:10F4B0008DF801E08DF803708DF804608DF805502B
:10F4C0001FF01CFC002384F81E31FAE4194A11686D
:10F4D0008A7D487D097D120402EB00220A44591CF2
:10F4E00084F8511202EB0363D5E7124A11680A7BD4
:10F4F000C87A897A120402EB00220A44EFE70D4A27
:10F5000011688A7848780978120402EB00220A44CC
:10F51000E5E700BF8C890020D06000203024002067
:10F520003445002058240020676666663045002078
:10F53000108E00208C410020902F002010230422E8
:10F54000184669468DF802808DF803808DF8048096
:10F550008DF805808DF800308DF801201FF0CEFB6E
:10F5600084F81E81ADE494F8CA305A09012A74D196
:10F5700003F00F0C13F0100300F08A80684F94F82A
:10F58000CB3094F8CCE0A4F84202F9188EEA0300DC
:10F5900084F824213B46C4F83872C4F83C12FA1FA0
:10F5A00084F84402A4F840E294F84402DFF880E1D1
:10F5B00003E0D4F83C12D4F83832994203F1010741
:10F5C00008D012F8011BC4F83872724580EA0100B5
:10F5D0001970EED3724584F8440208BF84F845C21E
:10F5E0003FF4CCAC127894F844329A4264D04D4B3C
:10F5F000B4F84002C4F828320122013300274FF644
:10F60000F671C4F82C3284F82471A4F8300284F81E
:10F61000282184F83422A4F83212AFE4D4F82C72F2
:10F62000B4F9321294F83052501CA7EB090902F0D9
:10F630000F0242F01002002989EA0505B8BF42F026
:10F640002002EDB28DF8002084F847028DF8019079
:10F6500084F848520DF10202D9E6324B324984F85F
:10F6600024015F1C012284F82801C4F82832C4F860
:10F670002C72C4F8301284F834227FE45A1CD2B2BF
:10F68000042A84F851224FEA03637FF404AFFFE6B3
:10F6900094F82421002A3FF471AC94F845220132F9
:10F6A00002F00F0262452DD084F8243166E4314621
:10F6B00032201FF023FBD4E6194BD4F83822C4F8CB
:10F6C0003C22002703F5AA72114603F15409C4F83D
:10F6D0002C2203F5B2703A46C4F82892C4F83832A6
:10F6E00084F82471C4F83072F8F7D8FB01300FD0D9
:10F6F000D4F82832C4F82C320123C4F8289284F8B4
:10F7000034323BE4D4F83C12D4F83832074A4BE7A1
:10F71000D4F828320222591CC4F828121A70E7E7DC
:10F720003C2F0020902F00200000F6FF332F0020F8
:10F73000382F0020044B93F90020002AC3BF5B78C8
:10F740000370012000207047C030002003682DE9BD
:10F75000F041DF691FB13B46BDE8F0411847002A80
:10F76000164611DD04460D460E4400E023689B68F2
:10F77000204698470028F9D0236815F8011B1B681C
:10F7800020469847AE42F1D1BDE8F08170B410F840
:10F790000E3C50F8044C002B40D030F80C2C20F8D4
:10F7A0000A1C8C4D10F80F6C8B4B891A89B2002201
:10F7B00020F8081C25F8161000F80E2C1D78617929
:10F7C0002368012D75D0154616461446002958D0D9
:10F7D000042900F09380082900F0AA80196A4EF6E7
:10F7E000FF7421401962DC69196A40F6FF452C401C
:10F7F00045F6FF7544F480742940224341F480515A
:10F80000DA611962DA694FF2FF310A40DA61DA69C6
:10F81000DA61002300F8063C70BC704701256E4A8F
:10F8200000F80E5C20F80C1C107861792268A84260
:10F830005ED01C461D461846002940D0042900F021
:10F840009380082900F0AA80116A4EF6FF700140EB
:10F850001162D169106A40F6FF44214045F6FF74F9
:10F8600041F4807120400B4340F44050D36110625A
:10F87000D3694FF2FF310B40D361D369D36170BCC0
:10F8800070471A6A22F001021A6299691A6A21F015
:10F89000F30141F0010122F00A0242F0010221438A
:10F8A00099611A629A6922F00C029A619A699A61C6
:10F8B000AFE74FF44052302516462C4686E7136AD0
:10F8C00023F0010313629169136A21F0F30141F0FF
:10F8D000010123F00A0343F0030301439161136222
:10F8E000936923F00C0393619369936170BC704733
:10F8F0004FF4405330241D4620469DE71A6A4FF6C8
:10F90000EF710A401A629A69196A22F473424FF63B
:10F910005F7442F480722140164341F010019E61F1
:10F9200019629A6922F440629A619A699A6170E751
:10F930001A6A4FF6FF610A401A62DA691C6A92B2CB
:10F9400022F0F3024FF2FF5142F001022140154331
:10F9500041F48071DD611962DA694FF6F3710A4092
:10F96000DA61DA69DA6154E7136A4FF6EF710B4036
:10F9700013629169136A21F473414FF65F7041F489
:10F980008071034043F030030D4395611362936926
:10F9900023F440639361936993613DE7136A4FF6E3
:10F9A000FF610B401362D369106A9BB223F0F3032B
:10F9B0004FF2FF5143F0010301401C4341F44071F9
:10F9C000D4611162D3694FF6F3710B40D361D369EF
:10F9D000D36121E7A0430020888A002010F80A3C68
:10F9E0000133DBB20A2B00F80A3C07D9044A10F8AD
:10F9F000131C002322F8113000F80A3C704700BFA6
:10FA0000A0430020F8B56C4F6C4B38786C4C01303B
:10FA1000A3FB00231B096568226CA66803EB830324
:10FA2000A0EB8303A9423B7001EB020330D294F8B0
:10FA30004820002A50D0634A03F580331078B3FB86
:10FA4000F0F39E422DD39A1B4FF4803595FBF0F0D6
:10FA50000244E26040F68C2000258242A36061608F
:10FA600084F8485025D9237894F94520934245D00D
:10FA7000002294F9441084F846205DB28B424BD0AA
:10FA80000023012284F84550237084F84720F8BDF4
:10FA90004C4A1078B3FBF0F39E42D4D294F848203D
:10FAA00002B34FF4803292FBF0F09A1B121AE2601C
:10FAB000D0E794F8473073B1A2F2EF2140F2DA5365
:10FAC000994211D823780B2B0ED8191D01332370BE
:10FAD00044F82120F8BDF8BD3A480078B3FBF0F3B4
:10FAE0009E42B0D21046E0E70023194684F8473022
:10FAF00030223548BDE8F84024F01BBD1A1F082A03
:10FB0000B6D894F84620182A51D8013284F84620F5
:10FB10005DB294F94410B1E794F84720002AAFD0C1
:10FB20002A48002B34D022690280012B30D0626930
:10FB30004280022B2CD0A2698280032B28D0E2695C
:10FB4000C280042B24D0226A0281052B20D0626A55
:10FB50004281062B1CD0A26A8281072B18D0E26A50
:10FB6000C281082912D0226B028209290ED0626B51
:10FB700042820A290AD0A26B82820B2908D0E36B49
:10FB8000C382134A13780133137079E70B2BF8DC27
:10FB9000C3EBC3720B2B4FEA420202F1180200EBD7
:10FBA0004100C8BF0222002124F0C3FCE9E75DB296
:10FBB00084F84450294661E714310020CDCCCCCCE8
:10FBC0009C8C0020981E0020AC8C0020A0430020BC
:10FBD0009D43002030B40E4D0E4B2A780E4C01325E
:10FBE000A3FB02031B09206C03EB8303A2EB83033B
:10FBF0004FF6FF72914200F101002B70084408BFDC
:10FC00000123206408BF84F8483030BC704700BF2F
:10FC100014310020CDCCCCCC9C8C0020002854D0BA
:10FC20002DE9F04F294DDFF8B080294FDFF8AC9077
:10FC3000DFF8ACA0DFF8ACB000EB800005EB800E85
:10FC400050264FF0000C05E055F8143B7545C3F8FD
:10FC500000C026D02B7A002BF6D06C68A30A43454F
:10FC60002FD022D94B452AD0534526D05B451AD0F8
:10FC7000FE23EFF3128286F31288606A616903EB58
:10FC8000830307EBC303013041F001015862D2B294
:10FC9000616182F3118855F8143B7545C3F800C0C3
:10FCA000D8D1BDE8F08F0023E3E7B3F5801F0AD079
:10FCB000084A9342DCD10223DBE70523D9E704237A
:10FCC000D7E70323D5E70123D3E77047E88C00206B
:10FCD000587D002001001000020010004D001000AF
:10FCE000500010004B001000704700BF00EB800078
:10FCF000024B53F820301960704700BFE88C002099
:10FD000010B400EB8000094C094A80002318A1F5CB
:10FD10007A715B8920585DF8044B03FB01F182FB8B
:10FD20000132C917C1EBA21101607047E88C0020B5
:10FD3000D34D6210704700BFF0B5046D8160236839
:10FD400023F001032360827912F0040395B0054685
:10FD50000E4679D012F0020F14BF4FF4005100216B
:10FD60004FF4A057206895F805E020F001002060CE
:10FD7000606820F440500143616023680EF0010286
:10FD8000002A23F4B0530BBF08220C2200210421C7
:10FD900023F00C031EF0020F08BF0A463B43134337
:10FDA0002360A36823F44073A360684613F06EFCDD
:10FDB0002D4B9C424FD02D4B9C424ED02C4B9C4205
:10FDC0004DD02C4B9C420CBF0F9A109A23681F04F5
:10FDD00048BF5200B2FBF6F306FB1322B2EB560FFC
:10FDE000226828BF0133160405D54FF6F0721A4079
:10FDF000C3F3420313439BB2A38168792B6DA979A6
:10FE000000F00202002A15BF4FF440324FF4803256
:10FE10004FF40034002410F0010F586808BF224648
:10FE2000CC074CBF024320EA02025A609A680907D5
:10FE30004CBF42F0080222F008029A601A6842F0B1
:10FE400001021A6015B0F0BD12F0020209D01F467F
:10FE50004FF4005186E70C9AB8E70D9AB6E70E9A70
:10FE6000B4E7174611467DE70038014000440040E2
:10FE700000480040004C0040A1F57A7107EE901A4E
:10FE80009FED087A9FED080A084BF8EEE77A10B567
:10FE900000EB8000A7EE870A53F8204022F03EFADC
:10FEA000206010BDEC51B83F0000B443E88C002046
:10FEB00001EB4101C90007EE101ADFED087A084B8B
:10FEC000B8EEC70A10B500EB800020EE270A53F801
:10FED000204022F023FA206010BD00BFABAA2A3DCB
:10FEE000E88C0020CA0000EE102A10B500EB80005C
:10FEF000044BBAEEEE0A53F8204022F00FFA2060CD
:10FF000010BD00BFE88C002003685B6A03B118478E
:10FF1000704700BF03681B6A03B11847704700BFF2
:10FF200003682DE9F041DF691FB13B46BDE8F041B0
:10FF30001847002A164611DD04460D460E4400E01F
:10FF400023689B68204698470028F9D0236815F855
:10FF5000011B1B6820469847AE42F1D1BDE8F081F5
:10FF60000368DB68184700BF03685B68184700BF79
:10FF700003681B68184700BF1C4B1A680AB10021B0
:10FF800011605A690AB1002111609A6A0AB1002110
:10FF90001160DA6B0AB1002111601A6D0AB10021FB
:10FFA00011605A6E0AB1002111609A6F0AB10021E6
:10FFB0001160D3F88C200AB100211160D3F8A02081
:10FFC0000AB100211160D3F8B4200AB100211160F8
:10FFD000D3F8C8200AB100211160D3F8DC300BB18E
:10FFE00000221A60024B00221A707047E88C002031
:10FFF0002C6000202DE9F04F0C68DFF814C3C04FCF
:020000040801F1
:100000002588C04E85B00CFB02F2BC42B6FBF2F66E
:1000100003F1FF3C06F1FF36BDF838E0B6B2AAB2F4
:100020001FFA8CFC5ED0B84DAC425BD0B4F1804F6F
:1000300058D0A5F59835AC4254D005F58065AC4252
:1000400050D0B24DAC4253D005F58065AC424FD094
:1000500022F4407205F58C3592B2AC422280C4F88D
:100060002CC026850ED0A84A94420BD002F54062DF
:10007000944207D002F58062944203D002F5806278
:10008000944201D10022228601256561CE79497909
:1000900016F0040731D016F0020F4FF040054FF074
:1000A00000060CBF4FF00809B146B0460296B246B2
:1000B000B446324601964FF4806703954FF0040B27
:1000C0000C2900F2E280DFE811F0AF00E000E00070
:1000D000E0008A00E000E000E0006300E000E000F3
:1000E000E0002A00894D22F07002AC4292B2ABD1FE
:1000F0002280C4F82CC02685C6E701954FF48065A0
:1001000006F002020397BB46B9464FF480464FF40F
:10011000805802954FF0100A4FF4807CD0E7256A92
:10012000DFF8DCC125F480552562256A6768D4F8BC
:100130001C9025F4005545EA0808644529F4E64575
:1001400048EA023245F4C04500F0F0800CF5006C3E
:10015000644500F0EB806760E561C4F840E022622E
:10016000E26942F40062E261626C42F4004262645D
:100170002288254692B242F0010225F8342B002253
:100180006E184381446006606A5005B0BDE8F08F88
:10019000256A5B4E25F480752562D4F820B0656829
:1001A000D4F81CA02BF4007B4BEA0C0C2AF0730A49
:1001B000B4424CEA02224AF0600A00F0AB8006F535
:1001C0000066B44200F0A6806560C4F81CA0C4F8C4
:1001D0003CE02262E26942F00802E261C4E7256A7B
:1001E000474F25F010052562D4F820C06668A56940
:1001F0002CF0200C25F080754CEA0A0A25F4E6451F
:10020000BC424AEA021245F4C0456AD007F50067CD
:10021000BC4266D06660A561C4F838E02262A2697B
:1002200042F40062A2619FE7266ADFF8D480019D54
:1002300026F001062662D4F820A06768A66926F495
:1002400080362A432AF0020A26F07306444542EA21
:100250000A0246F0600639D02B4DAC4236D005F587
:100260004065AC4232D005F58065AC422ED005F534
:100270008065AC422AD06760A661C4F834E022628F
:10028000A26942F00802A2616EE70C293FF66CAF4A
:1002900001A252F821F000BF8102010869010108A2
:1002A00069010108690101081F02010869010108CB
:1002B0006901010869010108D50101086901010806
:1002C00069010108690101086101010822F00C02BD
:1002D00042EA090227F4407742EA0B0247EA0C0798
:1002E000C9E722F08002039F42EA091222F040028D
:1002F0003A43029F26F4406637433E468AE700BFF2
:10030000002C014000A24A040034014000100040CB
:1003100040420F0022F4006242EA092222F4806285
:1003200025F440553A4348EA05054DE727F4804750
:10033000374310E7036803F138422DE9F04F920A82
:10034000584DAA5C02F01F0552090124022A04FA42
:1003500005F400F08C80032A00F08E80012A3CD046
:1003600001F003077A1E012AC1F3810CC1F30018C2
:100370008088C1F3411135D9C60700F19780850700
:1003800000F1A380440700F1B180020700F1BF80B3
:10039000C60600F1CD80850600F1DB80440600F141
:1003A000E980020600F1F780C60500F105818505A8
:1003B00000F11381440500F12181020500F12F8134
:1003C000C60400F13D81850400F14B81440400F135
:1003D0005981020455D4BDE8F08F334A55692C4346
:1003E0005461BDE7002422464FF0010E4FF003098F
:1003F00004E00132102A04F10204ECD00EFA02F6F5
:1004000036EA0005F5D1D3F808A009FA04F5ED4362
:100410000AEA050AC3F808A0D3F808B00CFA04FAEF
:100420004AEA0B0AC3F808A0B3F804A01FFA8AFA34
:100430002AEA06069E80B3F804A008FA02F646EA05
:100440000A06B6B29E801E682E401E60D3F800A039
:1004500007FA04F646EA0A061E60D3F80CA001FA71
:1004600004F605EA0A0A46EA0A05DD60C1E70E4A13
:1004700095692C43946173E70B4AD5692C43D46189
:100480006EE71A6822F040421A601A6842EA8777DB
:100490001F60DA6822F0404242EA8171D960BDE80B
:1004A000F08F00BF3C740308001002401A6822F06D
:1004B00003021A601A683A431A60DA6822F00302EB
:1004C0000A438507DA607FF55DAF1A6822F00C02F7
:1004D0001A601A6842EA87021A60DA6822F00C028F
:1004E00042EA81024407DA607FF54FAF1A6822F0D2
:1004F00030021A601A6842EA07121A60DA6822F0BB
:10050000300242EA0112DA6002077FF541AF1A6851
:1005100022F0C0021A601A6842EA87121A60DA688A
:1005200022F0C00242EA8112C606DA607FF533AFDC
:100530001A6822F440721A601A6842EA07221A60A6
:10054000DA6822F4407242EA01228506DA607FF519
:1005500025AF1A6822F440621A601A6842EA8722BC
:100560001A60DA6822F4406242EA81224406DA60C4
:100570007FF517AF1A6822F440521A601A6842EAEF
:1005800007321A60DA6822F4405242EA0132DA6035
:1005900002067FF509AF1A6822F440421A601A6811
:1005A00042EA87321A60DA6822F4404242EA813233
:1005B000C605DA607FF5FBAE1A6822F440321A6095
:1005C0001A6842EA07421A60DA6822F4403242EAC4
:1005D00001428505DA607FF5EDAE1A6822F440220B
:1005E0001A601A6842EA87421A60DA6822F44022E6
:1005F00042EA81424405DA607FF5DFAE1A6822F4F0
:1006000040121A601A6842EA07521A60DA6822F445
:10061000401242EA0152DA6002057FF5D1AE1A6853
:1006200022F440021A601A6842EA87521A60DA68B5
:1006300022F4400242EA8152C604DA607FF5C3AE7A
:100640001A6822F040721A601A6842EA07621A6059
:10065000DA6822F0407242EA01628504DA607FF5CE
:10066000B5AE1A6822F040621A601A6842EA8762E0
:100670001A60DA6822F0406242EA81624404DA6079
:100680007FF5A7AE1A6822F040521A601A6842EA53
:1006900007721A60DA6822F0405242EA0172DA60A8
:1006A00097E600BF10B50409013C052C17DC0D4B83
:1006B00033F8142000F00F0042FA00F313F00103A6
:1006C0000DD0012303FA00F0013810401FF0C2FEE4
:1006D000054A064B125D104403EBC00010BD00201C
:1006E00010BD00BFBC710308B47103086C8B0020FF
:1006F0002DE9F047B04C96B0A0429DF878608A464C
:1007000090461F4600F02981AC4B984200F066816C
:10071000AB4B984203D0002016B0BDE8F087A94A41
:10072000A94CD369A94DC4F8B48043F48023D361A4
:1007300004F5A06104F5C0624FF48073C4F8FC00B6
:100740002A20C4F8C010C4F8C420C4F8B830C4F8D3
:10075000BC30C4F8AC50FFF7A5FF05462B20FFF7CF
:10076000A1FF032301460093284633463A460DF184
:1007700058091DF0EFFA964B49F8503D48461DF0D8
:100780004FFAAC34256D6771A6712A68C4F82CA0A5
:1007900000232362E361A362636222F0010201216C
:1007A00016F00403C4F8088084F844102A6000F0AE
:1007B000CA8016F0020F14BF4FF4005000204FF40F
:1007C000A0512B6823F001032B606A6822F4405289
:1007D00002436A602B6807F00106002E23F4B05331
:1007E0000BBF0022042208200C2023F00C0317F07A
:1007F000020718BF02460B4313432B60AB6823F478
:100800004073AB60484612F041FF6B4B9D4200F0D5
:10081000A2806A4B9D4200F01081694B9D4200F01E
:100820000E816C4B9D420CBF119B129B2A681204D7
:1008300048BF5B00B3FBF8F108FB1133B3EB580F73
:100840002B6828BF01311B0405D54FF6F0730B4010
:10085000C1F34201194389B2A9816079216DA2795E
:1008600000F00203002B15BF4FF440334FF48033E8
:100870004FF40035002510F0010F486808BF2B46E3
:10088000D5074CBF034320EA03034B608B68120774
:100890004CBF43F0080323F008038B600B6843F060
:1008A00001030B601EB3206B002800F0CF80D4F84A
:1008B0004C80E568666912F0FBFD236B216D1A68B8
:1008C00022F4FF4222F0700242F48552ADB21A6067
:1008D0005D60C3F80880DE601A6842F001021A60A9
:1008E0008A6842F040028A605B689BB2236417B357
:1008F000606B002800F0A580A66C256912F0D8FD79
:10090000636B216D1A6822F4FF4222F0700242F4F8
:100910008452002042F01002ADB21A605D609E6009
:10092000D8601A6842F002021A60586058608B68FA
:1009300043F080038B600B68204643F001030B609B
:1009400016B0BDE8F08716F0020600F08680194662
:100950004FF4005035E70E9B68E71A4A1A4C93692A
:100960001A4DC4F80C8043F48043936104F5807100
:1009700004F500724FF4807360651920A161E26193
:10098000236163616560FFF78DFE05461A20FFF75E
:1009900089FE012301460093284633460DF158098C
:1009A0003A461DF0D7F90C4B49F8503D48460434FF
:1009B0001DF036F9E6E600BF003801400044004073
:1009C000004800400010024014310020505303083A
:1009D00027010001004C004025010001204A214C64
:1009E000D369214DC4F8608043F40033D36104F52A
:1009F000407104F580624FF48073C4F8A8001E2093
:100A0000E16622676366A366A565FFF74BFE0546B0
:100A10001F20FFF747FE0223014600932846334676
:100A20000DF158093A461DF095F9104B49F8503D23
:100A3000484658341DF0F4F8A4E60F9BF6E6109BE8
:100A4000F4E60B6843F080030B6074E720230B622D
:100A50000B6843F020030B6049E731463046B0E6AF
:100A600000100240143100205053030826010001F9
:100A70002DE9F04F4A484B4B4B4C4FF090414FF013
:100A8000010A4FF002094FF004084FF0080C4FF034
:100A9000100E20274026802530F8022B12F0010F7F
:100AA00003D01960A3F804A0083312F0020F03D09A
:100AB0001960A3F80490083312F0040F03D01960F2
:100AC000A3F80480083312F0080F03D01960A3F8CC
:100AD00004C0083312F0100F03D01960A3F804E02B
:100AE000083312F0200F02D019609F80083312F0F3
:100AF000400F02D019609E80083312F0800F02D0A0
:100B000019609D80083312F4807F05D04FF4807BFC
:100B10001960A3F804B0083312F4007F05D04FF435
:100B2000007B1960A3F804B0083312F4806F05D07D
:100B30004FF4806B1960A3F804B0083312F4006F0F
:100B400005D04FF4006B1960A3F804B0083312F419
:100B5000805F05D04FF4805B1960A3F804B00833C0
:100B600012F4005F05D04FF4005B1960A3F804B0E5
:100B7000083312F4804F05D04FF4804B1960A3F86E
:100B800004B00833D20B04D04FF4004219609A80AD
:100B9000083301F58061A1427FF47EAFBDE8F08F9C
:100BA000BC7103086C8B0020001800482DE9F04749
:100BB0000569C3681D4028D00F4606464FF000481F
:100BC0004FF00009B5FA85F328FA03F2D2431B3B34
:100BD00032611540042B16D8DFE803F031292119C2
:100BE00003007B6A002B32D003F1FF3A1FFA8AFA26
:100BF000C7F824903C6A34B1236820465146984790
:100C00006468002CF8D1002DDCD1BDE8F08738688D
:100C1000716B036889B29847002DD3D1F5E77868E6
:100C2000B16B036889B29847002DCBD1EDE7B86866
:100C3000F16B036889B29847002DC3D1E5E7F868E6
:100C4000316C036889B29847002DBBD1DDE7F36AA8
:100C50001FFA83FACEE700BF10B54B4CB4F804324C
:100C6000B4F806229A4224BF0023A4F80432B4F850
:100C70000A22B4F808329A4224BF0023A4F80832AA
:100C800094F8FF31A3B1072B12D094F8D42001239C
:100C90000021062A84F8F83184F8FE3184F8031222
:100CA00058D994F8D530DFED396A002B3FD110BD0B
:100CB00094F80332002B53D094F8FE3194F8F811D5
:100CC000DFED326A042B38BF042307EE903AB8EE0A
:100CD000E77A07EE901A27EE267AF8EEE77A84F89C
:100CE000FE3167EE877A94F8D420062A2FD8284B55
:100CF00003EB8203D3ED006AF4EEE76AF1EE10FA3B
:100D000011DDC6EE877AFDEEE77A17EE903A102BEA
:100D1000A8BF1023012BB8BF0123DBB28B4228BF31
:100D20000B4684F8F83194F8D530002BBFD0013A47
:100D3000032ABCD8B7EE000A80EE260A21F0EEFAAC
:100D4000B4F8D230984238BFA4F8D20010BDDFED1D
:100D50000F6AD1E7DFED0F7A1946B0EE677AC6E782
:100D600094F8FE3194F8F811DFED0B6A07EE103AB3
:100D700007EE901AB8EEC77AF8EEE77A27EE267AF1
:100D800067EE877AAFE700BF946100206F120338E7
:100D9000785303086F12833A6F120339F8B534227F
:100DA0000746002123F0C5FB642252233A8687F8C8
:100DB00032300B483B4607F130061421052204254A
:100DC000002401E010F9011F9970DA701D719C7107
:100DD0005A710833B342F5D101233B80F8BD00BFFF
:100DE000806F03082DE9F0411E212C243A2223268E
:100DF0004FF02D0E14270F252223047001750E24A9
:100E00003521427046751922212680F80CE087753D
:100E10004FF0530E4B270571437128253223C473BD
:100E20004176827100216422067480F81AE0372628
:100E30004FF07C5E4777857201270572C372C370DD
:100E4000C371437480F8283046241D46A02346729F
:100E5000C674C0F82CE04FF0000C4FF48278847018
:100E60004173C175817301764184C276C0F830E068
:100E7000DFF880E0877780F8367080F837603C27AD
:100E800080F83860C3844FF4AF76194B80F8417016
:100E9000C0F844E04687C363028480F8351080F8C8
:100EA0004020A0F82480C0F848C0034600F1240E7A
:100EB0000A2740F2726683F84E2083F84F2083F8A9
:100EC000501083F8515083F8521083F8567083F80D
:100ED0005710A3F8586083F8534083F8544083F8C0
:100EE00055400C337345E6D180F84C10BDE8F081D5
:100EF00000004040000020412DE9F04704464FF437
:100F0000D4620021162740F6761523F012FBDD4B44
:100F1000A4F8367440F60C0140F6961240F66C10B8
:100F20008127A4F840546F25A360A4F838144FF427
:100F3000C6736121A4F84224A4F844044222A120EB
:100F4000A4F84874A4F84E544FF4B1774FF4D17517
:100F5000A4F84634A4F84C144FF4A1732F21A4F83C
:100F60005024A4F85404142240F69800A4F85874AD
:100F7000A4F85E5440F6C8074FF4C175A4F856347F
:100F8000A4F85C140023C82184F86224A4F8640443
:100F90000A226420A4F83C74A4F83E74A4F85254C5
:100FA0009D27A4F85A5440F6C415A4F84A14A4F88E
:100FB0006014A4F8662484F86F3484F8703484F8DC
:100FC000713484F8723484F86C3484F86D3484F8A5
:100FD0006E34A4F86804A4F80812A4F80A020421E4
:100FE0005A202770A4F8F0514FF496773025A64E7A
:100FF00084F8F81184F801026E212B20A4F80672FF
:1010000084F8FD512127232584F8381284F83B0207
:1010100001214FF4C87084F83C7284F83D523727A0
:10102000242584F83922A4F8040284F8D035A4F8E1
:10103000F23184F8FF3184F8003284F8F931A4F8F1
:101040001C32A4F81A32A4F81E3284F8FC3184F859
:10105000183284F80E3284F8193284F8FE1184F8BC
:10106000FA1184F8501284F80F1284F8241284F8CC
:101070003A1284F83E12A4F8400284F84B2284F815
:10108000487284F83F32A4F84232A4F8463284F819
:10109000441284F8491284F84A3284F8245306F141
:1010A0008C003746324602E0072B0BDC917989072A
:1010B00004D5E118157981F825530133824202F1F4
:1010C0001402F1D1002105234FF010091125C4F8B5
:1010D0001013C4F8141384F81C333F21984640F2CF
:1010E000DC5300224FF0010EDFF8A0C184F82F93EB
:1010F00084F8335340F24C4940F26C7584F836134F
:10110000A4F86A3240F2753140F64303C4F808C0CF
:10111000A4F86E52A4F87A3284F80DE384F80EE352
:1011200084F82EE384F832E384F837E384F85DE250
:1011300084F866E284F80C2384F8182384F81923D1
:1011400084F81A2384F81B2384F81D2384F8382399
:1011500084F8732484F85C2284F85E2284F85F2289
:1011600084F86522A4F86C92A4F8781225462346E8
:101170004FF01E0C03E0013202330EF1010E032A80
:10118000CCBF0121002183F87C1200F0F881BEF170
:10119000120F83F87DC2EED100234FF0130E40F200
:1011A00046524FF002080E2184F868C284F8673274
:1011B00084F8693284F8713284F8733284F872E208
:1011C000A4F8762284F8708284F8741204F52973E6
:1011D00004F52D724FF47A7E4FF4FA6C23F804EC88
:1011E00023F802CC04339A42F8D10523A4F8D0E0C6
:1011F0004FF0190E84F8B23284F8F4E1032340F280
:101200002E4E0122002184F8B332A4F8CCE04FF432
:10121000F073DFF87CE0A4F8D230A4F8CEC084F8F4
:101220002D1384F8B01284F8B12284F8B52284F822
:10123000B42284F8D420144BC4F8D8E002E00B297F
:101240000CDC9A79520705D5621893F804E082F80D
:10125000DCE00131834203F11403F0D14FF4C87E86
:1012600040F2DC5301210022A4F8FEE04FF0320EE0
:10127000A4F8F03084F8FC1084F80021024BA4F8A4
:10128000F2E00AE003090C004474030803098C002F
:1012900000009040072A0CDC9979090705D5A118B0
:1012A00093F804E081F8F4E00132834203F114037F
:1012B000F0D1322340F2EA5140F2B45240F27E5073
:1012C000A4F8EE30A4F8E800A4F8EA10A4F8EC20A2
:1012D00004F56F7004F54F7808F0DCFD80220021E2
:1012E000404623F026F92422A64904F57F7020F019
:1012F000E9FD0B22A44904F5846020F0E3FD0323FB
:10130000002284F82C3484F82B24012300E0B379E4
:1013100013F0100306F1140640F029810132082A67
:10132000F5D184F82D3404F2CB22104604F2BF2309
:10133000002102F8011F03F8011F8342F9D1934BEA
:101340000020591D4FF02B094FF02A084FF01F0CB9
:101350004FF01E0E1A27192699424DD013F9012F6E
:101360001F2AF9D80FF2040A5AF822F05B15010877
:1013700051150108471501085913010859130108AF
:101380005913010859130108591301085913010889
:101390005913010859130108591301085913010879
:1013A0005913010859130108591301085913010869
:1013B0005913010859130108591301085913010859
:1013C0005913010859130108591301085913010849
:1013D0005913010859130108591301085913010839
:1013E0005913010865150108ED130108994284F8A5
:1013F000D70284F8CB02B1D104F5367004F27446FA
:10140000FFF7CCFC3046FFF7EDFC614B614A6249C7
:10141000C4F8283200274FF001084FF00A094FF0B6
:10142000280A1523C4F82C12C4F83022A4F820721C
:10143000A4F82272A4F80C7284F8F58184F825329D
:1014400004F515715548A4F8169284F8F6A184F8AD
:10145000F7A10EF07DF94FF448734FF47A706421D0
:1014600084F84C7284F84D7284F84F8284F8367296
:1014700084F8BA7284F8BE82A4F8343284F84EA29A
:1014800084F8B69284F8B792A4F8B802A4F8BC1213
:1014900004F1700823464FF4FA6C40F2DC5E5A22E5
:1014A000FF27A3F87201A3F874C1A3F876E183F8CB
:1014B000781183F8792183F87A2183F87B710E33D0
:1014C0009845EED10423002184F8E331002284F80A
:1014D000E21104F1C003EA6010359D42FBD1304DAA
:1014E000304A297984F89D1692E80300A368C4F86D
:1014F000300443F400222868A4F8341400230121A6
:1015000002272325C4F89906A26084F87B1684F884
:101510007C1684F87D76314684F87E3684F8213353
:1015200084F8223384F8233384F82053742204F59A
:101530009D6020F0C7FC314604F25C507422BDE887
:10154000F04720F0BFBC84F8CE9284F8C28203E753
:1015500084F8CDC284F8C1E2FEE684F8CC7284F847
:10156000C062F9E684F8D60284F8CA02F4E602EB17
:10157000820207EB8202137984F82D34D3E683F8D4
:101580007D82F8E594530308B8530308806F03087D
:101590009A99193F3D0A773FF6287C3F0088030857
:1015A000C87D0308C453030810B50B4C2046FFF751
:1015B000A3FC0A4894F8C0340370094A09490C2076
:1015C00000FB034304F2744403F2C2431460BDE819
:1015D00010400B6008F0E4BC946100200D8E0020E8
:1015E0008C410020108E0020F0B50C292BD8DFE8AC
:1015F00001F06F2A2A2A4C2A2A2A2B2A2A2A070093
:10160000046AB2F80CE097881668674D24F4805499
:101610000462036A4468C16923F4005343EA0E3349
:1016200021F4E641A84243EA073341EA062100F0EB
:10163000B58005F50065A84200F0B080926844606E
:10164000C16102640362F0BD046A96899588D2F88C
:1016500000E0554F24F480740462036A4468C16951
:1016600023F4007343EA062321F07301B84243EAEE
:10167000052341EA0E017ED04C4DA8427BD09268F2
:101680004460C161C2630362F0BD046A96899588B3
:10169000D2F800E0444F24F010040462036A446866
:1016A000816923F0200321F0807143EA061321F4BD
:1016B000E641B84243EA051341EA0E2148D03B4DCA
:1016C000A84245D092684460816182630362F0BDA4
:1016D000046A9389B2F804E01768334E24F00104D9
:1016E0000462056A4468816943EA0E0321F480318B
:1016F00025F002059BB221F07301B04243EA0503D5
:1017000041EA070114D0294DA84211D005F54065E2
:10171000A8420DD005F58065A84209D005F5806581
:10172000A84205D092684460816142630362F0BDC3
:10173000D689158A578A23F0080333433D43D68858
:1017400024F4407423F00403ADB233432C43E9E79F
:10175000D589178AD68823F0800343EA051324F439
:101760004064558A23F0400344EA870443EA0613A1
:1017700044EA8504A6E7D589178AD68823F400634E
:1017800043EA052324F44054558A23F4806344EA51
:10179000071443EA062344EA051470E7158A24F483
:1017A000804444EA851449E7002C0140003401409C
:1017B0002DE9F84FF02200218E488F4CDFF860921F
:1017C0008E4D8F4E8F4FDFF85C8222F0B2FE8E4836
:1017D0008E49DFF854E2DFF854C2002213598342E5
:1017E00000F0F880B3F1804F00F0F680AB4200F0DB
:1017F000F580B34200F0F480BB4200F0F380734503
:1018000000F0F280634500F0F180434500F0F08085
:10181000DFF81CA2534500F0A7800AF5806A534503
:1018200008BF092300F0A1801432A02AD6D1DFF826
:10183000C881774F774D08F1A0064FF0030A4FF0AB
:10184000020998F804301C09013C052C03F00F0331
:1018500000F3838037F8140040FA03F2D2077CD5F6
:101860004FF0010B0BFA03F3013B18401EF0F2FDA1
:10187000694B1B5D184415EBC0046ED055F8303031
:10188000664898F8081003F13842920A825C02F028
:101890001F005209022A0BFA00FB00F09480032A71
:1018A00000F08A80012A05D1584A584852694BEA0B
:1018B00002024261B4F804E0BEFA8EF2C2F11F02E5
:1018C00092B2D00803EB800002F00702046A920093
:1018D0004FF00F0C0CFA02FC24EA0C040462046AB8
:1018E00001FA02F22243002402624FF0010C224668
:1018F00003E0102A04F102042FD00CFA02F030EABF
:101900000E0102F10102F4D1D3F808B00AFA04F191
:10191000C9430BEA010BC3F808B0D3F808B0C3F809
:1019200008B0B3F804B01FFA8BFB2BEA00009880D4
:10193000988880B29880186808401860D3F800B082
:1019400009FA04F040EA0B001860D868102A01EA8E
:101950000001D96004F10204CFD108F11408464512
:101960007FF46FAFBDE8F88F082309EBC3034FF096
:10197000010B93F804A00AF01F034FEA5A1ABAF1B8
:10198000020F0BFA03F311D0BAF1030F08D0DA45B6
:101990007FF44AAFD1F814A043EA0A034B6143E74E
:1019A000D1F81CA043EA0A03CB613DE7D1F818A0A7
:1019B00043EA0A038B6137E7144A1448D2694BEAB9
:1019C0000202C26176E7114A104892694BEA0202AC
:1019D00082616FE70023C8E70123C6E70223C4E75B
:1019E0000323C2E70423C0E70523BEE70623BCE7C1
:1019F0000723BAE7587D0020447403080004004020
:101A00000008004000100040002C0140001002407F
:101A1000BC7103086C8B0020B47103083C7403088C
:101A2000C871030800400140001400400034014028
:101A30000044014001490248FFF7B8B8207E002069
:101A40000040014001490248FFF7B0B8F87D00208E
:101A50000034014001490248FFF7A8B8F87D002092
:101A60000034014001490248FFF7A0B8D07D0020B2
:101A70000008004001490248FFF798B8A87D0020FF
:101A80000004004002494FF08040FFF78FB800BFCC
:101A9000807D002001490248FFF788B8587D00206A
:101AA000002C014001490248FFF780B8587D002012
:101AB000002C01402DE9F04104684E4DA30AAB42D1
:101AC0007AD00AD94C4DAB425FD00335AB4277D0C8
:101AD000053DAB425DD0BDE8F081B3F5801F67D016
:101AE000013DAB4259D14FF0700E022647794FEAC3
:101AF000970C002968D0B000634685190227D4F8F6
:101B00000C809F400CEB4503BFB23C4D03F1040C2D
:101B100047EA080745F8231045F82C20E760EFF363
:101B20001281502282F31288821905EBC2021369D6
:101B3000002B34D013620433821905EBC2025769BB
:101B400017B11F6053690433821905EBC20297690C
:101B500017B11F6093690433821905EBC202D7697C
:101B600017B11F60D36904330027CAB21F6082F324
:101B70001188304405EBC000036A9BB9E3684FF657
:101B8000FE721340E360BDE8F0814FF0C00E042602
:101B9000ACE74FF0200E0026A8E7BDE8F08105EB8A
:101BA0000E03C9E7E36843F00103E360BDE8F08199
:101BB0004FF0480E012699E74FF0980E032695E75F
:101BC0004FF0E80E052691E7BF08022306FA03F05E
:101BD000BB40DB43E768094D9BB23B4087190CEBE8
:101BE000470CE3600CF1040345F82C1045F8232062
:101BF00095E700BF020010004D001000587D002046
:101C000070B503685E4D5F4E18885F4C05FB02F2AD
